:100000000C9445060C948B060C948B060C948B0672
:100010000C948B060C948B060C948B060C948B061C
:100020000C948B060C94C9180C948B060C948B06BC
:100030000C9448320C948B060C948B060C948B0613
:100040000C948B060C948B060C949D150C948B06CB
:100050000C94CB0B0C948B060C94950B0C948B0688
:100060000C94851B0C948B060C94CE2D0C948B0653
:100070000C940A780C948B060C946F72AC1BB11B19
:10008000B61BBF1BD61BED1BFD1B0D1C2A1C161E11
:10009000ED1BD81CE91C181D361D531DAD1D081E77
:1000A0000F20B9204821C8210022A322AA24142508
:1000B0008E25D72521264F267C26DF262927732744
:1000C0006C28ED2D212E642ED42EEC2E2D2FE42F16
:1000D000AB30AB30AB30AB30AB30AB30AB30AB3048
:1000E000AB30AB30AB306030623067307F30813066
:1000F0000A0D426174743A002025642043656C6CDB
:10010000732000204C6F77207761726E696E6720D4
:100110006C6576656C3A2025642E2564000A0D46D0
:100120006F756E6420424C2D4374726C3A2000252A
:1001300064000A0D0A0D2121204D495353494E47B1
:1001400020424C2D4354524C3A202564202121005A
:100150000A0D3D3D3D3D3D3D3D3D3D3D3D3D3D3D32
:100160003D3D3D3D3D3D3D3D3D3D3D3D3D3D3D3DBF
:100170003D3D3D3D3D000A0D43616C696272617415
:10018000696E672070726573737572652073656E32
:10019000736F722E2E004F4B0A0D000A0D466C69CC
:1001A0006768742D74696D65202575206D696E20F2
:1001B00020546F74616C3A2575206D696E000A0DCC
:1001C000436F6E74726F6C3A200048656164696EAB
:1001D00067486F6C64004E6F726D616C20284143FC
:1001E000432D4D6F646529000A0D3D3D3D3D3D3D6C
:1001F0003D3D3D3D3D3D3D3D3D3D3D3D3D3D3D3D2F
:100200003D3D3D3D3D3D3D3D3D3D3D3D3D0A0D00BE
:10021000416E676C654E69636B2020202020202092
:10022000416E676C65526F6C6C202020202020206E
:100230004163634E69636B20202020202020202012
:10024000416363526F6C6C202020202020202020EE
:100250005961774779726F202020202020202020AC
:100260004865696768742056616C75652020202098
:100270004163635A2020202020202020202020209D
:1002800047617320202020202020202020202020B3
:10029000436F6D706173732056616C75652020200B
:1002A000566F6C74616765205B302E31565D20207F
:1002B0005265636569766572204C6576656C2020B1
:1002C0004779726F20436F6D706173732020202017
:1002D0004D6F746F7220312020202020202020209C
:1002E0004D6F746F7220322020202020202020208B
:1002F0004D6F746F7220332020202020202020207A
:100300004D6F746F72203420202020202020202068
:1003100031362020202020202020202020202020B6
:1003200031372020202020202020202020202020A5
:100330003138202020202020202020202020202094
:100340003139202020202020202020202020202083
:10035000536572766F20202020202020202020202E
:10036000486F76657267617320202020202020204E
:1003700043757272656E74205B302E31415D2020B2
:100380004361706163697479205B6D41685D202011
:1003900048656967687420536574706F696E74206E
:1003A0003235202020202020202020202020202026
:1003B0003236202020202020202020202020202015
:1003C000436F6D7061737320536574706F696E74E1
:1003D0004932432D4572726F722020202020202048
:1003E000424C204C696D6974202020202020202060
:1003F0004750535F4E69636B20202020202020202F
:100400004750535F526F6C6C20202020202020200A
:1004100021212120494E434F4D50415449424C45E2
:1004200020212121002E000A0D20444143206F721B
:1004300020493243204552524F5221204368656380
:100440006B204932432C2033567265662C20444180
:100450004320616E6420424C2D4374726C005B2516
:10046000695D005B25695D002B204D696B726F4BE8
:100470006F70746572202B0048573A5625642E25FC
:10048000642053573A25642E256425630053657410
:1004900074696E673A2564202573004D697865722A
:1004A000204572726F7221004861726477617265D3
:1004B000204572726F7220313A2564202121004D4F
:1004C000697373696E6720424C2D4374726C3A25D0
:1004D0006421210021204E432D4552523A202532DD
:1004E0006420212000493243204552524F5221219D
:1004F00021004865696768743A20202535690053F2
:100500006574706F696E743A253569005072657351
:10051000737572653A253569004F66667365743A7E
:1005200020202535690048656967687420636F6E0F
:1005300074726F6C0044495341424C4544006163FE
:10054000742E2062656172696E67004E69636B3A52
:1005500020202020202025356900526F6C6C3A2025
:10056000202020202025356900436F6D7061737352
:100570003A202020253569004B25693A2534692029
:10058000204B25693A25346920004E693A253469A3
:100590002020526F3A253469200047733A25346988
:1005A000202047693A253469200050313A253469C2
:1005B000202050323A253469200050333A253469DE
:1005C000202050343A25346920004779726F202D5D
:1005D0002053656E736F72004E69636B253469201A
:1005E000282533692E25692900526F6C6C253469E2
:1005F00020282533692E256929004769657225342D
:1006000069202825336929004E69636B20253469E8
:1006100020282533692E25782900526F6C6C2025FF
:10062000346920282533692E2578290059617720DF
:1006300020253469202825336929004E69636B2001
:100640002534692028253369292825336929005252
:100650006F6C6C20253469202825336929282533BF
:1006600069290059617720202534692028253369BC
:1006700029282533692900414343202D2053656EE5
:10068000736F72004E69636B20253469202825330F
:10069000692900526F6C6C20253469202825336944
:1006A00029005A2020202025346920282533692953
:1006B00000566F6C746167653A2020202533692EDF
:1006C000253169560043757272656E743A20202098
:1006D0002533692E2531694100506F7765723A20C4
:1006E00020202020253469570044697363686172B3
:1006F00067653A202535696D416800526563656913
:100700007665720052432D525353493A20202020DF
:100710002534690052432D5175616C6974793A2012
:100720002534690052432D4368616E6E656C733ADF
:1007300025346900436F6D70617373004D61676E9E
:1007400065743A202020253569004779726F3A2078
:100750002020202025356900536574706F696E7400
:100760003A2025356900506F746925693A202025A3
:10077000336900506F746925693A20202533690078
:10078000536572766F202000536574706F696E74C4
:10079000202025336900506F736974696F6E3A20A9
:1007A0002533690052616E67653A2533692D25331B
:1007B0006900424C2D4374726C204572726F7273E3
:1007C000200025336420253364202533642025331D
:1007D000642000424C2054656D70657261747572BE
:1007E00065002533642025336420253364202533B8
:1007F000642000424C2D4374726C20666F756E64E9
:100800002000202563202020256320202025632030
:100810002020256320002025632020202563202020
:100820002025632020202563200020256320202010
:100830002D2020202D2020202D200031300031318E
:1008400000313200466C696768742D54696D65200B
:100850002000546F74616C3A2535756D696E0041E6
:1008600063743A20202535756D696E0028726573B2
:10087000657429000A0D47656E65726174696E675B
:100880002064656661756C7420506172616D657479
:10089000657220536574202564000A0D5573696ED6
:1008A0006720506172616D657465722053657420B4
:1008B0002564000A0D47656E65726174696E672074
:1008C00064656661756C74204D6978657220546149
:1008D000626C65000A0D4D697865722D436F6E6616
:1008E00069673A202725732720282575204D6F74C6
:1008F0006F727329000A0D3D3D3D3D3D3D3D3D3D3F
:100900003D3D3D3D3D3D3D3D3D3D3D3D3D3D3D3D17
:100910003D3D3D3D3D000A0D414343206E6F742037
:1009200063616C69627261746564210D0A00000084
:100930008F001E01AD013B02CA025803E603740496
:1009400002058F051B06A7063307BE074808D20815
:100950005B09E3096B0AF20A780BFD0B810C040DAD
:10096000860D070E870E060F840F00107B10F51002
:100970006E11E5115B12CF124213B31323149214BC
:10098000FE146A15D3153B16A11605176717C8176D
:1009900027188318DE1837198E19E319361A871AA3
:1009A000D61A231B6E1BB61BFD1B411C831CC31CCC
:1009B000001D3C1D751DAB1DE01D121E421E6F1E4D
:1009C0009A1EC31EE91E0D1F2E1F4D1F691F841F77
:1009D0009B1FB01FC31FD31FE11FEC1FF51FFB1F81
:1009E000FF1F002003010000BA6B00020101A96C87
:1009F000010302023D6D020003039A6D2532692E48
:100A00002531695600253364256320253033646D14
:100A1000256300537461747573004552524F523A06
:100A2000202532642000253469202532693A25309A
:100A30003269002534696D2563002533692025332B
:100A40006920253369202533690025336920253342
:100A50006920253369202533690054656D706572FE
:100A60006174757265732020202000256343202067
:100A7000202020002532692E25316956202025337B
:100A8000692E253169410025346957202536696D65
:100A90004168002532756D2F73205361743A2564C7
:100AA000200020203344004E6F46780044475053C6
:100AB00000486F6D653A2533646D202533642563E6
:100AC000202563004E6F204E6176694374726C215D
:100AD000000A0D7777772E4D696B726F4B6F7074CC
:100AE00065722E64652028632920486953797374E0
:100AF000656D7320476D6248000A0D746865207546
:100B00007365206F66207468697320736F667477ED
:100B1000617265206973206F6E6C79207065726DEB
:100B20006974746564200A0D6F6E206F726967695D
:100B30006E616C204D696B726F4B6F707465722DB6
:100B400048617264776172650047726175706E65A5
:100B50007220486F5454004143542044534C004A7F
:100B600065746920736174656C6C69740053706599
:100B70006B7472756D20736174656C6C6974202878
:100B80004C6F77207265736F6C7574696F6E290096
:100B90005370656B7472756D20736174656C6C69EC
:100BA0007420283230343829005370656B747275A4
:100BB0006D20736174656C6C6974004D756C74693B
:100BC0007369676E616C2050504D000A0D52656369
:100BD00065697665723A2000756E6B6E6F776E2E62
:100BE000205573696E672050504D2E2E2E006E6F6B
:100BF0007420737570706F727465642062792068F8
:100C00006172647761726521000A0D3D3D3D3D3D95
:100C10003D3D3D3D3D3D3D3D3D3D3D3D3D3D3D3D04
:100C20003D3D3D3D3D3D3D3D3D3D3D3D3D3D000A64
:100C30000D466C69676874436F6E74726F6C0A0D51
:100C400048617264776172653A25642E25640A0DE5
:100C5000536F6674776172653A5625642E25642554
:100C60006320000A0D3D3D3D3D3D3D3D3D3D3D3D4B
:100C70003D3D3D3D3D3D3D3D3D3D3D3D3D3D3D3DA4
:100C80003D3D3D3D3D3D3D3D000011241FBECFEFAC
:100C9000D0E1DEBFCDBF11E0A0E0B1E0EEEAF5EFBC
:100CA00002C005900D92A63AB107D9F718E0A6EA5E
:100CB000B1E001C01D92AC3DB107E1F76AEAE2E0A4
:100CC000F0E081E2809357007491AE014F5F5F4F77
:100CD00020EF37EFDA019FE0F9012F5F3F4F84915A
:100CE0008D93915097FFF8CF773911F40000FECF24
:100CF000FA019EE0819168276095915097FFFACFA5
:100D00008889681721F0773911F40000FECF0E941E
:100D10004C070C94D67A0C94000080912106E82FA1
:100D2000FF27EE0FFF1FE15BF84F808191818D5E01
:100D30009F4F14F010920301808191818A5B9F4F35
:100D4000CCF4809103018823A9F481E0809303010E
:100D5000809114048F5F80931404853038F088EEFE
:100D600093E09093DB018093DA0104C066E970E0C0
:100D70000E94C6358091140499279093A205809310
:100D8000A10508951F93CF93DF93182F882389F02F
:100D900080EF90E09F938F9381E892E19F938F93F0
:100DA000E091E003F091E10309950F900F900F900F
:100DB0000F9080914406823308F044C084EF91E0A4
:100DC0000E949016EC01112329F0CE010E94991681
:100DD0008823D9F3C2E0D0E026E530E080911E01FF
:100DE00090911F018217930730F02196255D3F4FA8
:100DF000C730D10598F3809144069927C89F900188
:100E0000C99F300DD89F300D11242093000111236C
:100E1000D9F068EC70E08C2F0E94C635DF93CF9339
:100E200088EF90E09F938F9381E892E19F938F9357
:100E3000E091E003F091E10309958DB79EB7069626
:100E40008DBF02C080930001112311F18091000138
:100E50006AE00E94297A892F99279F938F93809126
:100E600000010E94297A99279F938F9383E091E054
:100E70009F938F9381E892E19F938F93E091E0039A
:100E8000F091E10309952DB73EB7285F3F4F2DBF85
:100E9000DF91CF911F910895CFEFD0E1DEBFCDBF9D
:100EA0008824992414B815B807EE13E002531040B3
:100EB00017FFFCCF189B06C0199B02C08DE007C02E
:100EC0008BE005C0199B02C084E101C08AE08093D9
:100ED000020181E887B93E9A8FEF88B98BE184B926
:100EE00081E085B98EE38AB987E48BB9469A84B7E5
:100EF000877F84BF8091600088618093600010923A
:100F0000600084EC99E09093DB018093DA01109209
:100F1000E3021092E20210925407109253071092CB
:100F2000E5021092E4021092E7021092E60220918C
:100F30000201243128F084EC94E0A0E0B0E004C089
:100F40008BE095E0A0E0B0E08093430190934401F2
:100F5000A0934501B09346012A3011F0243110F0DE
:100F6000289801C0289A0E94F9160E94CA160E9469
:100F700089120E941F320E943D1A81E00E94822D38
:100F80000E94DB620E948E6E0E94C27680910201F6
:100F90008C3010F4299A01C0299878940E94942CDE
:100FA00080912202826080932202109225020E9488
:100FB000F94084EF91E00E9490168C01809122020A
:100FC00080FD05C0C8010E9499168823B9F38DE100
:100FD00091E09F938F93C1E8AC2EC2E1BC2EBF92EB
:100FE000AF92E091E003F091E103099580EA9FE080
:100FF0000E9490168C01C0E0D0E00F900F900F90EF
:101000000F90B1EFEB2EB6E0FB2EA5EACA2EA6E0BC
:10101000DA2E0E94F9408091220280FD05C0C801AD
:101020000E9499168823B9F3F60180811816ACF452
:101030000BC00E94F9408091220280FD05C0C801CA
:101040000E9499168823B9F3C8010E949916882333
:1010500021F4F7018081882364F7F701808187FFFD
:1010600018C02196DF93CF9321978FE291E09F9351
:101070008F93BF92AF92E091E003F091E103099565
:101080008091A7018F5F8093A7018DB79EB70696C9
:101090008DBF2196E4E0F0E0CE0EDF1E88E090E008
:1010A000E80EF91ECC30D10508F4B3CFC0E0D0E093
:1010B0000EEE16E0F5EAEF2EF6E0FF2EF801838142
:1010C00087FD1CC0F70180811816C4F42196DF93B8
:1010D000CF93219782E391E09F938F9381E892E1F0
:1010E0009F938F93E091E003F091E103099582E0F3
:1010F0008093D8018DB79EB706968DBFF801838186
:1011000080788383219684E090E0E80EF91E085FE2
:101110001F4FCC30D10590F280E591E09F938F93E3
:10112000C1E8D2E1DF93CF93E091E003F091E103D6
:10113000099590911F068091A7010F900F900F9035
:101140000F90981728F48091FA0380618093FA0336
:1011500086E791E09F938F93DF93CF93E091E00335
:10116000F091E103099588EE93E00E9490168C01BE
:101170000E94431A0F900F900F900F90C8010E9489
:1011800099168823D9F386E991E09F938F93DF9393
:10119000CF93E091E003F091E103099580E00E9494
:1011A0009536809102010F900F900F900F908A302A
:1011B00011F0843110F0289801C0289A80ED97E052
:1011C0009093DB018093DA0185E5809316048EE02D
:1011D00090E00E94C72A9927182F00278FE090E0FF
:1011E0000E94C72A080F111D1093AD010093AC0196
:1011F0008AE090E00E94C72A9927182F00278BE0E9
:1012000090E00E94C72A080F111D1093AB010093B4
:10121000AA010F5F1F4F39F08091AC019091AD0191
:101220008F5F9F4F41F41092AD011092AC0110926C
:10123000AB011092AA018091AA019091AB019F93FA
:101240008F938091AC019091AD019F938F938BE927
:1012500091E09F938F93DF93CF93E091E003F09120
:10126000E10309958DB79EB708968DBF8EEB91E08F
:101270009F938F93DF93CF93E091E003F091E1038D
:10128000099580912D060F900F900F900F90E0918F
:10129000E003F091E10382FF07C08AEC91E09F93A5
:1012A0008F93DF93CF9308C086ED91E09F938F9348
:1012B00081E892E19F938F9309950F900F900F9083
:1012C0000F900E94811F88E893E190933E018093E4
:1012D0003D0161E0F62EF09215048F2D0E94C206AA
:1012E000809147060E940C7688EE91E09F938F9341
:1012F000DF93CF93E091E003F091E103099580ED56
:1013000097E00E9490168C018AEF90E00E94901660
:1013100083E0809379051092A60180918A060F9050
:101320000F900F900F9084FF02C0F092AE01809159
:10133000B001882311F04798FECF8091DE01882309
:1013400009F4EBC180911001882309F4E6C11092E1
:10135000DE0180911404882319F00E948D0602C0DA
:101360000E94FE430E94F940209102012A3011F0B0
:10137000243110F0289801C0289A8091D602882341
:1013800031F08091D60281508093D6020EC08091B8
:101390006F00806280936F001092500710924F0789
:1013A0008091FA0388608093FA0380913D019091C7
:1013B0003E01019790933E0180933D0180913D0154
:1013C00090913E01892B21F0809123028823C9F15D
:1013D00080913D0190913E01892BD9F40E94AC2D62
:1013E00085E090E090933E0180933D018091B305AC
:1013F0009091B40501969093B4058093B3058091C4
:10140000FA0381608093FA0380917A058260809369
:101410007A0580910801909109018F5F9F4FC1F477
:101420008091D5028823A1F088EA91E69093DB01B0
:101430008093DA0180E890E090930901809308019D
:1014400007C02A3011F0243110F0289801C0289AE2
:101450000E9494778091DE01882309F05EC180911B
:101460000E01882311F00E9410170E94CD120E94D5
:101470001B0EC8010E949916882309F44AC10C5E0C
:101480001F4F80912302882349F08091FA038260E4
:101490008093FA0380917A0582600FC08091DA010F
:1014A0009091DB01892B59F480913D0190913E018F
:1014B000079728F080917A058D7F80937A05809137
:1014C000D602882361F08091AE01882341F010920A
:1014D000AE0188E893E19093DB018093DA0180917B
:1014E0000501882321F08150809305012EC080934F
:1014F00020041092AC021092AB021092AA02109239
:10150000A9021092A8021092A7028091D602882305
:10151000E1F480910801909109018F5F9F4FA9F438
:101520002091AE01223089F088E99AE39093DB01A3
:101530008093DA0180E09CE0909309018093080198
:10154000222319F082E08093AE0180919C01893CB6
:1015500048F0815080939C018091FA038B7F8093A7
:10156000FA033FC0809130088823F9F08091FA0394
:1015700084608093FA0389E08093AD038091080131
:10158000909109018F5F9F4F81F48091D50288234C
:1015900061F088E99AE39093DB018093DA0180E0BF
:1015A00098EA90930901809308011092A403109285
:1015B000A3031092A2031092A1031092A003109211
:1015C0002308109262081092610810926408109229
:1015D00063088FEF9FEF9093600880935F081092ED
:1015E0009C0180910001282F332780911E0190914A
:1015F0001F0182179307CCF48091A0028062809330
:10160000A00280910801909109018F5F9F4FC1F462
:1016100080E797E19093DB018093DA0180E093E02B
:1016200090930901809308010BC08091DA01909199
:10163000DB01892B29F48091A0028F7D8093A00289
:101640000E94756784E08093D9018091A00281FD9A
:1016500005C05AEA852E55E0952E12C08091AF0143
:101660008F5F8093AF01813359F41092AF01809165
:10167000A8019091A90101969093A9018093A801D6
:101680000894811C911CF2E78F16FBE09F0609F07D
:1016900040C0882499242091AC013091AD012F5F86
:1016A0003F4F3093AD012093AC018091AA019091FE
:1016B000AB0101969093AB018093AA01832F9927E8
:1016C000682F8EE090E00E94CF2A8091AC0190912B
:1016D000AD019070682F8FE090E00E94CF2A80913A
:1016E000AA019091AB01892F9927682F8AE090E099
:1016F0000E94CF2A8091AA019091AB019070682F2F
:101700008BE090E00E94CF2A84E190E00E94901646
:101710008C010E94C5670E94A56E8091D901882323
:1017200009F005CE0E94FC6202CE1F920F920FB606
:101730000F9211248F939F93EF93FF938091070152
:101740008823E1F48091CA019091CB010196909396
:10175000CB018093CA01FC01E153FB4FE081ED30E6
:1017600019F08A3A910539F41092CB011092CA010E
:1017700081E080930701E093C60004C01092CB0182
:101780001092CA01FF91EF919F918F910F900FBE20
:101790000F901F9018951F920F920FB60F92112461
:1017A0002F933F934F935F936F937F938F939F9369
:1017B000AF93BF93CF93EF93FF9390E08091B001ED
:1017C000813029F48091C6008093CE00CCC08091F6
:1017D000B001823029F48091C60080932304C3C0F5
:1017E0008091C6008093C2015091D0015A3A10F006
:1017F0009093D1018091C2018D3009F065C0809134
:10180000D101823009F060C09093D101852F9927D2
:101810008D5D9B4FFC01329740812091CC0130912E
:10182000CD01241B3109DC0111978C91281B310952
:10183000C9019F709093CD018093CC0146E09695AD
:1018400087954A95E1F7982F935C9093CE012F737B
:101850003070235C2093CF018081981729F48C91FC
:10186000281711F491E006C090E08091BF018F5FCE
:101870008093BF01C091C101CC2309F074C09923AA
:1018800009F471C081E08093C101580F5093BE01EB
:101890005150E52FFF27ED5DFB4F8DE08083809158
:1018A0002504823509F05FC00E94811F88E190E025
:1018B0002CE00FB6F894A895809360000FBE20939B
:1018C0006000C093D8014FC02091D101822F992789
:1018D00081309105F9F0823091051CF4892B21F0BB
:1018E00040C0029711F13DC08091C201833239F4AA
:1018F0008091C101882319F481E08093D101809106
:10190000C2018093230481E08093D0018091C201C1
:10191000992722C02F5F2093D101E52FFF27ED5D8E
:10192000FB4F8091C201808309C0E52FFF27ED5D49
:10193000FB4F8091C20180835A3A20F45F5F50933D
:10194000D00102C01092D1012091C2018091CC013E
:101950009091CD01820F911D9093CD018093CC0188
:1019600002C01092D101FF91EF91CF91BF91AF9141
:101970009F918F917F916F915F914F913F912F91A7
:101980000F900FBE0F901F901895AC01A0E0B0E033
:101990009D01A817B90748F4EFECF4E08191280FF6
:1019A000311D1196A417B507C8F33F70FD01E1532F
:1019B000FB4FC90156E0969587955A95E1F7835CF0
:1019C00080831196FD01E153FB4F2F733070822FFE
:1019D000835C8083A053BB4F8DE08C9310920701F2
:1019E0008091CF048093C6000895A0E0B0E0EBEFB3
:1019F000FCE00C94A27A2C859D850E85BB2483E2A5
:101A00008093CF049F599093D0042093D10433E066
:101A1000E32EF12C002309F49EC0CF84D888BE01A8
:101A20006D5E7F4FA989BA890150109709F493C060
:101A30001097B9F0F601EB0DF11DB3949081119759
:101A400091F4002349F1FB016E5F7F4FDB01C08001
:101A5000D1806E5F7F4F0D90BC91A02DBB240150B3
:101A600002C090E019C01097B9F0F601EB0DF11D1E
:101A7000B3944081119791F4002341F1FB016E5F13
:101A80007F4FDB01C080D1806E5F7F4F0D90BC9196
:101A9000A02DBB24015002C040E018C01097B1F047
:101AA000F601EB0DF11DB3941081119781F4002321
:101AB00071F0FB013296DB01CD90DC90BF016E5FCF
:101AC0007F4FA081B181BB24015001C010E0F7011C
:101AD000E153FB4F892F86958695835C808308941C
:101AE000E11CF11CF701E153FB4F892F992783700B
:101AF000907024E0880F991F2A95E1F755279A01E5
:101B000094E0369527959A95E1F7822B835C808344
:101B10000894E11CF11CF701E153FB4F4F7050702A
:101B2000440F551F440F551F812F992726E0969586
:101B300087952A95E1F7842B835C80830894E11CC8
:101B4000F11CF701E153FB4F1F73135C10830894E2
:101B5000E11CF11C6ACFC7010E94C50CE9E00C949E
:101B6000BE7AA3E07A2F4091BE014650442309F487
:101B700058C0E72FFF27ED5DFB4F80818D537F5FBE
:101B8000E72FFF27ED5DFB4F20812D537F5FE72F70
:101B9000FF27ED5DFB4F30813D537F5FE72FFF2730
:101BA000ED5DFB4F60816D537F5F9927880F991F13
:101BB000880F991F522F52955F70582B822F9927AB
:101BC0008F709070F4E0880F991FFA95E1F7232F3A
:101BD00026952695282B832F992783709070E6E011
:101BE000880F991FEA95E1F7682B41504F3FC9F0E4
:101BF000EA2FFF27ED5DFB4F5083AF5F41504F3F12
:101C000081F0EA2FFF27ED5DFB4F2083AF5F41504E
:101C10004F3F39F0EA2FFF27ED5DFB4F6083AF5F49
:101C2000A5CF86E294E09093BD018093BC01A350C0
:101C3000A093BB010895A2E0B0E0E1E2FEE00C94C5
:101C4000A87A8091C101882309F457C40E94B10D7C
:101C500080912404823609F023C3809125049927BA
:101C60008037910509F4AFC081379105C4F48A36F5
:101C7000910509F480C28B36910544F48B349105AB
:101C800071F18636910509F45FC10AC38D3691055D
:101C900009F469C08E36910509F44DC001C384373B
:101CA000910541F1853791054CF48137910509F48F
:101CB00091C08337910509F4DFC0F2C287379105DF
:101CC00009F41BC2883791052CF48537910509F476
:101CD000D7C1E6C28937910509F46DC1E1C2E0912F
:101CE000BC01F091BD01808191819093900180931E
:101CF0008F01D6C28091BE01A091BC01B091BD01FF
:101D0000853140F080E1EEEFF3E00D9001928A958D
:101D1000E1F70DC08D919D910D90BC91A02D809308
:101D2000FE039093FF03A0930004B093010480EF9F
:101D30008093B9014BC0809107018823E1F38DE4C2
:101D400090E09F938F9388E996E09F938F9381E033
:101D50008F938F938EE48F930E94F50C8DB79EB76F
:101D600007968DBF9DC2A091BC01B091BD011C9191
:101D7000113081F48DE4E8E9F6E00D9001928A9546
:101D8000E1F70E94D12B19838091FA038F7E809313
:101D9000FA0301C01982809107018823E1F381E0F1
:101DA00090E09F938F93CE0101969F938F9381E054
:101DB0008F938F938DE48F930E94F50CADB7BEB7D0
:101DC0001796ADBF6DC281E08093C4018FEF809301
:101DD000050166C2E091BC01F091BD01E0818E2F4A
:101DE0008A508A3058F48983882311F481E003C033
:101DF000863010F085E0898361E00EC08E2F84511B
:101E00008A3070F48983882311F481E003C086301E
:101E100010F085E0898360E089810E94512C12C016
:101E2000E983EF3F19F40E94342C89838981882348
:101E300011F481E003C0863010F085E08983898148
:101E40000E94E52A809107018823E1F387E790E06B
:101E50009F938F9380E296E09F938F9381E090E031
:101E60009F938F93CE0101969F938F9382E08F93E0
:101E700081E08F9381E577C12091BC013091BD0154
:101E8000D9018C918150853008F045C0F9018181DC
:101E9000883509F040C08091D5028823E1F52F5F95
:101EA0003F4F87E7E0E2F6E0D9010D9001928A9575
:101EB000E1F7F90182910E944E2B809161069927EA
:101EC000AA27BB27BC01CD0124EC39E040E050E05B
:101ED0000E940A7ADC01CB018093870190938801EC
:101EE000A0938901B0938A01809162069927AA275D
:101EF000BB27BC01CD010E940A7ADC01CB01809393
:101F0000830190938401A0938501B09386010E9480
:101F1000342C898301C01982809107018823E1F361
:101F200081E090E09F938F93CE0101969F938F93D2
:101F300081E08F938F9383E58F930E94F50C8DB78B
:101F40009EB707968DBF26C0E091BC01F091BD0100
:101F5000E0818E2F8150853018F48E2F0E94E52A63
:101F60000E94342C8983809107018823E1F381E06A
:101F700090E09F938F93CE0101969F938F9381E082
:101F80008F938F9386E48F930E94F50CADB7BEB705
:101F90001796ADBF8091D502882329F46EE670E0D4
:101FA00089810E94C63580E00E94C2068091470662
:101FB0000E940C7675C1E091BC01F091BD01808159
:101FC000992787FD909590936A078093690781818F
:101FD000992787FD909590936C0780936B0782817A
:101FE000992787FD909590936E0780936D07838165
:101FF000992787FD90959093700780936F07848150
:10200000992787FD9095909372078093710785813A
:10201000992787FD90959093740780937307868125
:10202000992787FD90959093760780937507878110
:10203000992787FD909590937807809377078085FF
:10204000992787FD909590937A07809379078185EA
:10205000992787FD909590937C0780937B078285D5
:10206000992787FD909590937E0780937D078385C0
:10207000992787FD90959093800780937F0710C1E3
:10208000E091BC01F091BD0180810E9478318A838A
:10209000882319F481E0898301C0198280910701A6
:1020A0008823E1F388E090E09F938F9386EE96E09B
:1020B0009F938F9321E030E03F932F938091BC0159
:1020C0009091BD019F938F933F932F93CE010296E2
:1020D0009F938F933F932F93CE01820F931F9F93D4
:1020E0008F9384E08F9381E08F9385E58F930E9497
:1020F000F50CEDB7FEB773963CC08091BB018930FB
:1021000008F4CEC02091BC013091BD012F5F3F4F3C
:1021100088E0A6EEB6E0F90101900D928A95E1F70C
:10212000D9018E910E94CE308A83882319F481E0F0
:10213000898301C01982809107018823E1F321E09E
:1021400030E03F932F93CE0102969F938F933F935E
:102150002F93CE01820F931F9F938F9382E08F93D3
:1021600081E08F9387E58F930E94F50CEDB7FEB762
:102170003B96EDBF95C08091D502882309F090C0B1
:102180000E94BF758983823019F0843009F088C0BD
:1021900020E430E0F8948091C1008F738093C100F7
:1021A0008091C9008F738093C9008091C100877EA0
:1021B0008093C1008091C900877E8093C90080917F
:1021C000C80087FF03C08091CE00F9CF8091C00086
:1021D00087FF03C08091C600F9CFE091BC01F09168
:1021E000BD01E081E13021F482E08093B0012EC096
:1021F000E43611F421E830E081E08093B001832FD0
:1022000099278093CD002093CC008091CD008093BE
:10221000C5008091CC008093C4008091CA008F7D5E
:102220008093CA008091CA008F7E8093CA008091FB
:10223000C9008B7F8093C9008091CA00846080931D
:10224000CA008091CA0082608093CA008091CA004F
:10225000877F8093CA008091C200877F8093C200ED
:102260008091C9008E7F8093C9008091C1008861F0
:102270008093C1008091C90088618093C9008091DA
:10228000C10080688093C1008091C90080688093FC
:10229000C90010926E0010926F0010927000789436
:1022A0008091250499278436910509F4BBC08536B1
:1022B0009105ACF48136910509F46FC08236910521
:1022C0002CF48B34910509F45DC00FC18236910561
:1022D00009F470C08336910509F47FC006C18C36BD
:1022E000910509F4EDC08D3691054CF487369105C2
:1022F00009F4F8C08836910509F4B2C0F6C08437F5
:10230000910529F08637910509F4E8C0EEC0809167
:10231000BE01A091BC01B091BD01803140F080E1CF
:10232000EEEFF3E00D9001928A95E1F70DC08D91EB
:102330009D910D90BC91A02D8093FE039093FF037F
:10234000A0930004B0930104809107018823E1F376
:102350001F92809104018F9384E58F930E94F50C66
:102360008AEF8093B9018FEF8093050180EA9FE0A7
:102370000E9490169093B2018093B1010F900F903C
:102380000F90B3C0E091BC01F091BD0180819181BB
:102390009093900180938F01A8C0E091BC01F091CF
:1023A000BD01808180930601803298F08FE1809397
:1023B00006010FC0A091BC01B091BD018BE0E6E128
:1023C000F4E00D9001928A95E1F780911F048093CB
:1023D000BB058FEF8093050188C08091B501909176
:1023E000B601892B89F4E091BC01F091BD01E08137
:1023F000EE2351F08AE0E89FC00111240E9490165C
:102400009093F1038093F003E091BC01F091BD0142
:1024100090818AE0989FC00111249093B601809327
:10242000B50115C08FEF80930501E091BC01F091DB
:10243000BD0190818AE0989FC00111249093B8015A
:102440008093B701892B19F081E08093C60180EA5F
:102450009FE00E9490169093B2018093B10145C015
:102460008FEF80930501E091BC01F091BD01908157
:1024700097FD08C082E08093C3011092B4011092CE
:10248000B3011AC0909580911B02892B80931B0287
:1024900091818AE0989FC00111249093B4018093A8
:1024A000B30184E08093C30180EA9FE00E9490160C
:1024B0009093B2018093B10181E08093C70115C070
:1024C0008FEF80930501E091BC01F091BD01808107
:1024D00080931C0281E08093C80107C081E0809353
:1024E000C50103C081E08093C9011092C10110921F
:1024F000BD011092BC011092BB01E3E0CE5F0C94D1
:10250000C47A982F8091C00085FFFCCF9093C600BD
:1025100008950F931F9388E18093C1008091C000BC
:1025200082608093C0008091C10080688093C10068
:102530008091C10080648093C10000E010E00093AE
:10254000C5008AE290E08093C4008091B701909129
:10255000B8010E9490169093F3038093F2038CEDE0
:1025600090E00E9490169093220480932104109290
:10257000F40386E58093F50381E08093F8038BE014
:102580008093F6031092F7031093BD010093BC01F2
:102590001092BB011F910F910895A0E1B0E0E3ED0F
:1025A000F2E10C94A57A80910701882309F4C1C255
:1025B0008091B1019091B2010E949916882361F037
:1025C0001092B4011092B3011092B8011092B701A9
:1025D0001092B6011092B5018091B3019091B401AF
:1025E000892B41F08091CD049091CE040E949916E0
:1025F000882329F48091C701882309F460C0809161
:102600000701882309F45BC08091C3010FEC15E03A
:102610008430A8F00E94971F80E590E09F938F93ED
:102620001F930F9381E08F938F9388E48F930E9481
:10263000F50C2DB73EB7295F3F4F2DBF34C0109228
:102640001D0280E194E09F938F938AE89FE19F931E
:102650008F93E091E003F091E103099584E190E02C
:102660009F938F931F930F9381E090E09F938F939D
:1026700083EC91E09F938F9382E08F9381E08F931F
:1026800088E48F930E94F50C8091C301982F8F5F8F
:102690008093C3012DB73EB7215F3F4F2DBF9430CC
:1026A00010F01092C3018091B3019091B4010E9487
:1026B00090169093CE048093CD041092C701809120
:1026C000C801882351F180910701882331F10E94CC
:1026D000971F80E590E09F938F938FEC95E09F93F9
:1026E0008F9321E030E03F932F9380E291E09F931E
:1026F0008F933F932F938CE192E09F938F9383E08E
:102700008F9381E08F938CE48F930E94F50C10924D
:10271000C8018DB79EB70F968DBF8091C5018823E4
:10272000D1F0809107018823B1F08AE090E09F9377
:102730008F9384EF93E09F938F9381E08F938F9398
:1027400086E58F930E94F50C1092C5012DB73EB718
:10275000295F3F4F2DBF8091C9018823D9F0809117
:1027600007018823B9F08BE090E09F938F9386E177
:1027700094E09F938F9381E08F93809104018F93D6
:1027800087E48F930E94F50C1092C9018DB79EB714
:1027900007968DBF80912104909122040E94991682
:1027A000882309F461C080910701882309F45CC083
:1027B00080913C069927880F991F880F991F7C01EB
:1027C0000027F7FC0095102F809130039091310382
:1027D000A0913203B0913303BC01CD01A801970150
:1027E0000E947E7A30930F0420930E048091280378
:1027F00090912903A0912A03B0912B03BC01CD0134
:10280000A80197010E947E7A30931104209310044E
:102810008091B502809312048091B40280931304D6
:1028200088E090E09F938F938EE094E09F938F9346
:1028300081E08F9383E08F938BE68F930E94F50C5A
:10284000809114042DB73EB7295F3F4F2DBF8530CF
:1028500018F086E08093140483E690E00E949016BE
:1028600090932204809321048091B7019091B80144
:10287000892B41F08091F2039091F3030E94991605
:10288000882321F48091C601882339F180910701C2
:10289000882319F10E94B03482E490E09F938F93D3
:1028A00089E795E09F938F9381E08F938F9384E4E2
:1028B0008F930E94F50C1092C6018DB79EB70796B4
:1028C0008DBF8091B7019091B801009731F00E94BF
:1028D00090169093F3038093F2038091B501909149
:1028E000B601892B09F4B8C08091F0039091F103EF
:1028F0000E949916882309F4AFC0809107018823AC
:1029000009F4AAC080913C069927880F991F880F67
:10291000991F7C010027F7FC0095102F8091300350
:1029200090913103A0913203B0913303BC01CD01EA
:10293000A80197010E947E7A3093E3032093E2037B
:102940008091280390912903A0912A03B0912B0331
:10295000BC01CD01A80197010E947E7A3093E50366
:102960002093E403209118083091190840911A0827
:1029700050911B08DA01C90163E0880F991FAA1F53
:10298000BB1F6A95D1F7820F931FA41FB51F820F3B
:10299000931FA41FB51F2091430130914401409122
:1029A000450150914601BC01CD010E947E7A3093D1
:1029B000E7032093E6038091F8029091F902A09139
:1029C000FA02B091FB0249E0B595A79597958795D6
:1029D0004A95D1F78093E8038091F4029091F50233
:1029E000A091F602B091F70239E0B595A7959795B9
:1029F00087953A95D1F78093E903809100039091F0
:102A00000103A0910203B091030329E0B595A795B6
:102A1000979587952A95D1F78093EA038EE090E009
:102A20009F938F9382EE93E09F938F9381E08F9398
:102A30008F9383E48F930E94F50C8091B501909160
:102A4000B6010E9490169093F1038093F0032DB786
:102A50003EB7295F3F4F2DBF809106018F3F71F137
:102A6000992704E0880F991F0A95E1F7805F9D4F31
:102A700040E150E0BC01CE0101960E945D7880E10A
:102A800090E09F938F93CE0101969F938F9381E067
:102A900090E09F938F9386E091E09F938F9382E0E5
:102AA0008F9381E08F9381E48F930E94F50C8FEFD9
:102AB000809306018DB79EB70B968DBF8091BB05A5
:102AC0008823D1F0809107018823B1F081E090E064
:102AD0009F938F938BEB95E09F938F9381E08F93E0
:102AE0008F9382E48F930E94F50C1092BB052DB753
:102AF0003EB7295F3F4F2DBF8091C4018823C9F0A5
:102B0000809107018823A9F084E390E09F938F933D
:102B10008FE497E09F938F9381E08F938F9380E56D
:102B20008F930E94F50C1092C4018DB79EB7079643
:102B30008DBFE6E0C05F0C94C17A1F920F920FB672
:102B40000F9211242F933F935F936F937F938F93F3
:102B50009F93AF93BF93EF93FF9320E08091D901B0
:102B6000882329F08091D90181508093D9018091E7
:102B7000C003882319F081508093C0038091E10144
:102B800081508093E1018F3F09F05BC089E0809321
:102B9000E1018091DF019091E00101969093E001C5
:102BA0008093DF0180910F018F5F817080930F010F
:102BB000882319F481E08093DE01349903C081E019
:102BC0008093E2018091DA019091DB01892B21F160
:102BD0008091DA019091DB010B9750F08091DA013E
:102BE0009091DB010A979093DB018093DA0104C096
:102BF0001092DB011092DA018091DA019091DB01F1
:102C0000209108013091090182239323892B11F02F
:102C100021E008C020E006C08FEF9FEF90930901EC
:102C20008093080180910201222331F08A3011F44F
:102C30005A9A07C0479A05C08A3011F45A9801C0C1
:102C400047988091E201882309F45AC020919C01A1
:102C5000222309F055C08091080883FF51C086B136
:102C60009927FC01E071F07084FF13C08091DC01B2
:102C70009091DD0101969093DD018093DC018091BC
:102C8000DC019091DD01895E9340D0F12093E20157
:102C900037C08091DC019091DD01892B69F1809131
:102CA000DC019091DD018A56914030F58091DC0184
:102CB0009091DD0169E270E00E94357A8091DC013B
:102CC0009091DD01860F971F9093DD018093DC01C9
:102CD0008091DC019091DD010B9750F08091DC0137
:102CE0009091DD010A979093900180938F0104C029
:102CF000F0939001E0938F011092DD011092DC01BE
:102D0000FF91EF91BF91AF919F918F917F916F91C3
:102D10005F913F912F910F900FBE0F901F901895CC
:102D20002091DF013091E001280F391FC901019680
:102D300008952091DF013091E001821B930B892FD0
:102D400099278695807490700895CF93DF930E94A1
:102D50009016EC01CE010E9499168823D9F3DF91D9
:102D6000CF910895CF93DF930E949016EC0109C094
:102D700080911001882329F0909310018FEC8093AB
:102D80007A00CE010E949916982F882389F3DF914B
:102D9000CF9108959FB7F8945F983E9A469A809194
:102DA000B0008F708093B0008091B00083608093FA
:102DB000B0008091B1008B738093B1008091B1001D
:102DC0008B608093B1001092B2008FEF8093B300BC
:102DD0008091B00080688093B000809170008A7FFD
:102DE00080937000809170008260809370009FBF1C
:102DF00008958AE090E00E9490169093E8018093F5
:102E0000E70182E085BD83EA84BD17BC84EB88BD01
:102E100086E086BD80916E00816080936E0008958B
:102E2000A0E0B0E0E6E1F7E10C94A47A80915706C7
:102E3000E82FFF27E75BFE4F9681D08080910E013F
:102E4000A92FBB27A7FDB095CB2FDB2F813009F031
:102E5000DDC0209130033091310340913203509115
:102E60003303BD01CE010E940A7A97FF04C0615866
:102E70007F4F8F4F9F4F7B018C01F7E01595079592
:102E8000F794E794FA95D1F78D2D992787FD9095C2
:102E9000A92FB92F209128033091290340912A03AB
:102EA00050912B03BC01CD010E940A7A97FF04C008
:102EB00061587F4F8F4F9F4FE7E0959587957795A6
:102EC0006795EA95D1F7F801E701C61BD70BE80B28
:102ED000F90B2091AB033091AC03C90153E0880F8B
:102EE000991F5A95E1F7821B930BAA2797FDA0958E
:102EF000BA2FC81BD90BEA0BFB0B80914E06992702
:102F0000AA27BB27BC01CD019E01AF010E940A7A0E
:102F100097FF04C061507E4F8F4F9F4FFC01EB0124
:102F200049E0F595E795D795C7954A95D1F78091F2
:102F30006E01992736E0880F991F3A95E1F7409185
:102F40000C0150910D01209156063327841B950BDF
:102F5000B9010E94497A80910C0190910D01860F70
:102F6000971F90930D0180930C0180910C0190911B
:102F70000D0197FD0F9624E0959587952A95E1F729
:102F80009093D5018093D4018091890680FF07C07A
:102F90008091D4019091D5018C0F9D1F06C0809126
:102FA000D4019091D5018C1B9D0B9093D5018093FA
:102FB000D40180914F06282F3327220F331F220F71
:102FC000331F8091D4019091D501821793077CF033
:102FD00080915006282F3327220F331F220F331FD3
:102FE0008091D4019091D5012817390724F43093AA
:102FF000D5012093D40180910201843108F4C2C02C
:1030000080910E018F5F80930E01BEC02091280336
:103010003091290340912A0350912B03BD01CE0129
:103020000E940A7A97FF04C061587F4F8F4F9F4FCD
:103030007B018C01C7E015950795F794E794CA9535
:10304000D1F78D2D992787FD9095A92FB92F209124
:103050003003309131034091320350913303BC016E
:10306000CD010E940A7A9B01AC0197FF04C0215850
:103070003F4F4F4F5F4FB7E0559547953795279591
:10308000BA95D1F72E0D3F1D401F511F809152065A
:103090009927AA27BB27BC01CD010E940A7A97FF76
:1030A00004C061507E4F8F4F9F4FFC01EB01A9E0A0
:1030B000F595E795D795C795AA95D1F780916D01BC
:1030C000992776E0880F991F7A95E1F740910A01D8
:1030D00050910B01209156063327841B950BB901A3
:1030E0000E94497A80910A0190910B01860F971FE7
:1030F00090930B0180930A0180910A0190910B013A
:1031000097FD0F9664E0959587956A95E1F7909302
:10311000D3018093D2018091890681FF07C08091FD
:10312000D2019091D3018C0F9D1F06C08091D201D6
:103130009091D3018C1B9D0B9093D3018093D2016E
:1031400080915306282F3327220F331F220F331F5E
:103150008091D2019091D301821793077CF08091E6
:103160005406282F3327220F331F220F331F80913D
:10317000D2019091D3012817390724F43093D30159
:103180002093D20110920E01E7E0CDB7DEB70C9488
:10319000C07A1F920F920FB60F9211242F933F9374
:1031A0004F935F938F939F93EF93FF9380910201CF
:1031B0009091E301843108F04CC0992309F01CC1BF
:1031C0008091B00086FF24C08091B0008F7B8093F7
:1031D000B0008091D4019091D50187559E4F909376
:1031E000D7018093D60125E08D3D920718F08CED34
:1031F00095E005C08757914030F487E791E09093C0
:10320000D7018093D6018091D6019091D701BAC0A1
:103210008091B00080648093B00080915506282F83
:1032200033278DED96E0289FA001299F500D389FF0
:10323000500D1124CA012091E4013091E501821B57
:10324000930B9093D7018093D60181E080930E0178
:10325000D0C0992309F0D0C08091B00086FF97C0FC
:103260008091B0008F7B8093B000E091E601EE2367
:10327000F1F480915506282F33278DED96E0289F95
:10328000A001299F500D389F500D1124CA01209193
:10329000E4013091E501821B930B9093D701809359
:1032A000D6011092E5011092E401469AA2C089EA83
:1032B00093E09093D7018093D6018E2F9927833086
:1032C0009105D9F08430910534F48130910549F0AD
:1032D000029761F020C08430910591F0059799F034
:1032E0001AC08091D4019091D50104C08091D2017F
:1032F0009091D30187559E4F1DC08091E40705C072
:103300008091BD0702C08091ED079927880F991F12
:10331000880F991FEFCFFF27EE0FFF1FE15BF84FDC
:1033200020813181220F331F8091D6019091D701E6
:10333000820F931F9093D7018093D6018091D6017D
:103340009091D70155E08D3D950718F08CED95E0F3
:1033500005C08757914030F487E791E09093D701FB
:103360008093D6012091D6013091D7012C5B30405B
:103370003093D7012093D6018091E4019091E5012B
:10338000820F931F9093E5018093E40132C08091F6
:10339000B00080648093B0008CEB90E09093D701F4
:1033A0008093D6018091E4019091E50184549F4F70
:1033B0009093E5018093E4018091D801882321F066
:1033C0008091D602882321F48091D801823011F4B3
:1033D000469801C0469A8091E6018F5F8093E6018E
:1033E00090915506981728F481E080930E01109271
:1033F000E60181E08093E3012091D6013091D7016D
:1034000041E02F37340730F08FEF8093B3002F5F08
:1034100030400FC02F3F3105C9F0C0F0A9014F5F08
:1034200050404F37510550F480E88093B300205846
:1034300030403093D7012093D60112C08FEF809394
:10344000B3005093D7014093D6010AC08091D601B2
:103450008093B3001092D7011092D6011092E3012D
:10346000FF91EF919F918F915F914F913F912F919C
:103470000F900FBE0F901F90189510927C008FEC4C
:1034800080937A000895CF93DF931092ED0183E04B
:1034900090E00E94C72AC82FDD27C531D10508F06A
:1034A0002A97C7BD84E690E00E94B216809114016D
:1034B000909115018052934010F4C0E0D0E0CA3FD3
:1034C000D105F8F4C7BD82E390E00E94B21685E210
:1034D00094E09F938F9381E892E19F938F93E09183
:1034E000E003F091E1030995809114019091150199
:1034F0000F900F900F900F908052934010F02196F4
:10350000DECFC093CC056C2F83E090E00E94CF2AE1
:1035100080912D0680FF0AC08091CC058A508B3E99
:1035200028F08091F90380648093F903C7BD8CE291
:1035300091E00E94B216DF91CF910895EF92FF9231
:103540001F93CF9310E080ED97E00E9490167C01CE
:10355000CCE8133019F4CB3008F0C9E010E08091CA
:10356000FD019091FE018C5F934024F48091130142
:1035700081500AC08091FD019091FE0187509440D6
:1035800034F0809113018F5F8093130101C011E02B
:103590008091FB019091FC018C5F934024F4809119
:1035A000120181500AC08091FB019091FC0187506B
:1035B000944034F0809112018F5F8093120101C01A
:1035C0001F5F8091F9019091FA018C5F934024F480
:1035D0008091110181500AC08091F9019091FA0106
:1035E00087509440C4F0809111018F5F8093110146
:1035F00013C087E294E09F938F9381E892E19F93B9
:103600008F93E091E003F091E10309950F900F9003
:103610000F900F905FC01F5F82E18093280280911E
:1036200022028E7F8093220285EA8093BC008091E3
:1036300013018A3040F48091F90381608093F9038B
:103640008AE08093130180911301863F40F08091BE
:10365000F90381608093F90385EF809313018091D2
:1036600012018A3040F48091F90382608093F9035B
:103670008AE08093120180911201863F40F0809190
:10368000F90382608093F90385EF809312018091A2
:1036900011018A3040F48091F90384608093F9032A
:1036A0008AE08093110180911101863F40F0809162
:1036B000F90384608093F90385EF80931101809171
:1036C0002802882339F0C7010E949916882309F03F
:1036D00090CFF5CF109210018FEC80937A008091FB
:1036E00010018823E1F3CA3020F48AE090E00E94C0
:1036F000B216C15009F02DCF86E490E00E94B216B8
:10370000CF911F91FF90EF9008951F920F920FB6E7
:103710000F921124EF92FF920F931F932F933F93D9
:103720004F935F936F937F938F939F93AF93BF93C9
:10373000EF93FF9380910602282F332744275527C4
:103740008F5F80930602F9012231310508F0B4C37E
:10375000E25CFF4F0C94D07A8091780090917900D0
:1037600046C080917800909179002CC180917800BA
:1037700090917900909309028093080257C180913B
:10378000390390913A032091780030917900821B9F
:10379000930B9093BD058093BC058091BC059091DF
:1037A000BD0590931302809312025EC18091780050
:1037B0009091790020913B0330913C03821B930B45
:1037C0009093CB058093CA058091CA059091CB0553
:1037D000909315028093140271C380910C02909112
:1037E0000D022091780030917900820F931F909301
:1037F0000D0280930C0281E062C380910A029091D5
:103800000B022091780030917900820F931F9093E2
:103810000B0280930A0284E052C380911E019091B2
:103820001F019C01220F331F280F391F8091780040
:103830009091790063E070E00E94357A260F371F7F
:10384000369527953695279530931F0120931E01B5
:1038500085E035C3809178009091790040913503DF
:1038600050913603841B950B9093F4018093F301E0
:103870008091F3019091F401029704F122E04E3E11
:10388000520784F4209107022B5F209307022550F2
:103890008091A1029091A202845F914018F4215F6F
:1038A0002093070280910702853684F14F5F5F4FB6
:1038B0005093360340933503845626C08091F3011C
:1038C0009091F4018F5F9F4F0CF532E04732530720
:1038D000ECF0209107022550209307022B5F809186
:1038E000A1029091A202845F914018F42F5020937E
:1038F0000702809107028C394CF44150504050939C
:103900003603409335038C598093070281E08093FE
:10391000F20180917800909179009093C305809393
:10392000C2058091F3019091F4019C01442737FD79
:103930004095542F8091F0029091F102A091F202F3
:10394000B091F302820F931FA41FB51F8093F00262
:103950009093F102A093F202B093F3022091F0024F
:103960003091F1024091F2025091F30257FF04C0EE
:1039700021503C4F4F4F5F4F6AE055954795379523
:1039800027956A95D1F78091F0029091F102A0916C
:10399000F202B091F302821B930BA40BB50B809340
:1039A000F0029093F102A093F202B093F3022EC1C1
:1039B00080910A0290910B02209178003091790059
:1039C000820F931F90930B0280930A0210920502BC
:1039D00078C2809102018A3071F4809178009091D0
:1039E00079002091080230910902820F931F0196FD
:1039F0009695879517C0409108025091090284312D
:103A000058F02091780030917900240F351F8FEF06
:103A100097E0821B930B06C080917800909179000B
:103A2000840F951F9093FA018093F90186E047C2B5
:103A30008091390390913A03209178003091790078
:103A4000821B930B9093BD058093BC058091BC05B0
:103A50009091BD052091120230911302820F931FA5
:103A60009093F8018093F70187E029C28091780054
:103A70009091790020913B0330913C03821B930B82
:103A80009093CB058093CA058091CA059091CB0590
:103A90002091140230911502820F931F9093F6012A
:103AA0008093F5010BC220910C0230910D028091A0
:103AB000780090917900280F391F30930D022093E0
:103AC0000C02809102018A3019F4220F331F04C0C6
:103AD000220F331F220F331F30930D0220930C024D
:103AE00020910C0230910D02C90137FD079603E0C9
:103AF000959587950A95E1F79093FE018093FD01D6
:103B000080910E0290910F02820F931F97FD0196F4
:103B10009595879590930F0280930E02209145030F
:103B200030914603821B930B90931D0180931C01DF
:103B3000209103023091040280911C0190911D019B
:103B4000280F391F37FF02C02F5F3F4F359527954C
:103B500030930402209303024ECE20910A0230914A
:103B60000B028091780090917900280F391F3093D3
:103B70000B0220930A02809102018A3019F4220F6D
:103B8000331F04C0220F331F220F331F30930B0249
:103B900020930A0220910A0230910B02C90137FDDD
:103BA0000796F3E095958795FA95E1F79093FC01D8
:103BB0008093FB018091100290911102820F931F5C
:103BC00097FD019695958795909311028093100229
:103BD0002091430330914403821B930B90931B016C
:103BE00080931A01209101023091020280911A0102
:103BF00090911B01280F391F37FF02C02F5F3F4FE5
:103C000035952795309302022093010283E057C136
:103C10001092060281E0809310018091E901909159
:103C2000EA0101969093EA018093E901809178007E
:103C30009091790090931501809314018091140163
:103C400090911501AA27BB272091160230911702E7
:103C50004091180250911902280F391F4A1F5B1F0B
:103C600020931602309317024093180250931902C2
:103C700080911A028F5F80931A02823108F41EC16C
:103C80008091160190911701A0911801B09119012E
:103C90007C018D0163E0EE0CFF1C001F111F6A9573
:103CA000D1F7E81AF90A0A0B1B0BE20EF31E041FE8
:103CB000151F8091ED01992787FD9095A92FB92FA8
:103CC000BC01CD0126EC34E240E050E00E940A7ACB
:103CD000DC01CB01E81AF90A0A0B1B0BD801C7015A
:103CE0000496A11DB11DB7FF05C0D801C7010B96F1
:103CF000A11DB11D23E0B595A795979587952A95A8
:103D0000D1F78093160190931701A0931801B093F7
:103D100019018091C4059091C5057C010027F7FC2D
:103D20000095102F8091160190911701A091180114
:103D3000B0911901E81AF90A0A0B1B0BE092D002A4
:103D4000F092D1020093D2021093D3022091EE019F
:103D50003091EF014091F0015091F10157FF04C003
:103D6000215F3F4F4F4F5F4F84E055954795379503
:103D700027958A95D1F78091EE019091EF01A0915E
:103D8000F001B091F101821B930BA40BB50B809352
:103D9000EE019093EF01A093F001B093F1018091B7
:103DA000EE019091EF01A091F001B091F1018E0D23
:103DB0009F1DA01FB11F8093EE019093EF01A09370
:103DC000F001B093F1018091EE019091EF01A0918B
:103DD000F001B091F101B7FF03C00F96A11DB11D15
:103DE00014E0B595A795979587951A95D1F72091E9
:103DF000D0023091D102281B390BC90137FF03C013
:103E0000309521953F4FAC01F3E0440F551FFA95D3
:103E1000E1F721383105C4F08091EB019091EC017C
:103E20009C01E3E0220F331FEA95E1F7281B390BD1
:103E3000240F351F37FF02C0295F3F4F73E03595D0
:103E400027957A95E1F717C08091EB019091EC01ED
:103E50009C0165E0220F331F6A95E1F7281B390B9F
:103E6000240F351F37FF02C0215E3F4F45E03595D7
:103E700027954A95E1F73093EC012093EB0180916F
:103E8000160290911702A0911802B0911902B7FF83
:103E900003C00196A11DB11DB595A795979587956E
:103EA0008093160290931702A0931802B093190200
:103EB00089E080931A0202C01092060282E0809389
:103EC00005028091050280937C0080910602882380
:103ED00019F08FEC80937A00FF91EF91BF91AF9131
:103EE0009F918F917F916F915F914F913F912F9112
:103EF0001F910F91FF90EF900F900FBE0F901F90AA
:103F0000189590E2EFECF5E08FE49193815087FFF4
:103F1000FCCF089590911D02903540F4E92FFF27C2
:103F2000E153FA4F80839F5F90931D020895AF92F3
:103F3000BF92CF92DF92FF920F931F93CF93DF93A5
:103F400020911B0220FF0AC080911C02882311F0DF
:103F5000815002C08091200180931C0221FF0CC07F
:103F600090911C0280912001981719F410921C0264
:103F700003C09F5F90931C02822F992780FF04C08B
:103F800081FF02C010921C020E94811F80911C02BE
:103F9000282F33279AE8C92E9FE1D92EC091E0033C
:103FA000D091E1038A3098F481E180931D023F9320
:103FB0002F938EE594E09F938F93DF92CF92FE0133
:103FC00009952DB73EB72A5F3F4F2DBF11C080E145
:103FD00080931D023F932F9383E694E09F938F93EA
:103FE000DF92CF92FE0109958DB79EB706968DBFE1
:103FF00020911C02822F9927AA27BB27FC014197F9
:1040000010F00C94CC28E05BFF4F0AE8C02E0FE1C3
:10401000D02EC091E003D091E1030C94D07A10929D
:104020001D0288E694E09F938F930AE81FE1DF92D8
:10403000CF92FE01099584E180931D020F900F90AD
:104040000F900F9082E690E09F938F9386E590E02B
:104050009F938F931F921F92809102016AE00E94AA
:10406000297A892F99279F938F93809102010E942B
:10407000297A99279F938F9388E794E09F938F9352
:10408000DF92CF92E091E003F091E103099588E29D
:1040900080931D02EDB7FEB73E96EDBF89E996E02D
:1040A0009F938F930E94342C99279F938F938DE831
:1040B00094E09F938F93DF92CF92E091E003F09191
:1040C000E10309958091FA032DB73EB7285F3F4F72
:1040D0002DBF84FF06C08CE380931D028BE994E022
:1040E000D2C09091F903992351F08CE380931D0283
:1040F000892F99279F938F9388EA94E03BC19091F1
:1041000023029923B1F08CE380931D02892F992714
:104110009F938F938FEB94E09F938F931F930F93B5
:10412000E091E003F091E1030995EDB7FEB7369613
:1041300079C49091AD03992371F08CE380931D02B3
:10414000892F99279F938F9384ED94E09F938F936A
:104150001F930F93D9C480913D0190913E01069722
:1041600010F00C94D5288CE380931D0285EE94E02A
:10417000A5C7809108081AE8C12E1FE1D12EC09171
:10418000E003D091E10380FF6BC010921D0280918B
:10419000D0029091D102A091D202B091D302BC0181
:1041A000CD0125E030E040E050E00E947E7A3F9370
:1041B0002F9382EF94E09F938F93DF92CF92FE0133
:1041C000099584E180931D028DB79EB706968DBF39
:1041D0008091CC029091CD02A091CE02B091CF02FD
:1041E000BC01CD0125E030E040E050E00E947E7A45
:1041F0003F932F938FEF94E09F938F93DF92CF9213
:10420000E091E003F091E103099588E280931D02BB
:10421000EDB7FEB73696EDBF809114019091150170
:104220009F938F938CE095E09F938F93DF92CF9233
:10423000E091E003F091E10309958CE380931D0286
:104240002DB73EB72A5F3F4F2DBF87B599279F9364
:104250008F9389E195E09F938F93DF92CF928EC0E9
:1042600010921D0286E295E09F938F93DF92CF928A
:10427000FE01099584E180931D020F900F900F902D
:104280000F9085E395E09F938F93DF92CF921AC7AB
:1042900010921D028EE395E09F938F930AE81FE131
:1042A000DF92CF92FE01099584E180931D020F9069
:1042B0000F900F900F908091300390913103A09157
:1042C0003203B0913303B7FF04C081509C4FAF4F0E
:1042D000BF4FCAE0B595A79597958795CA95D1F731
:1042E000BF93AF939F938F938BE495E09F938F93AE
:1042F0001F930F93E091E003F091E103099588E2A9
:1043000080931D02EDB7FEB73896EDBF809128036C
:1043100090912903A0912A03B0912B03B7FF04C009
:1043200081509C4FAF4FBF4FFAE0B595A795979539
:104330008795FA95D1F7BF93AF939F938F938AE5B3
:1043400095E09F938F931F930F93E091E003F0917B
:10435000E10309958CE380931D022DB73EB7285FDA
:104360003F4F2DBF8091C5079091C6079F938F93B4
:1043700089E695E09F938F931F930F93E091E0035D
:10438000F091E10309958DB79EB706968DBF0DC7D5
:10439000E1E0FE2EC1E0D0E001E517E09F2D96950B
:1043A00084E1989FC001112480931D02F80182814D
:1043B00093819F938F932196DF93CF932197808151
:1043C00091819F938F93DF93CF9388E795E09F939D
:1043D0008F938AE89FE19F938F93E091E003F091A0
:1043E000E10309952DB73EB7245F3F4F2DBF32E063
:1043F000F30E22960C5F1F4F88E08F1578F6D5C616
:1044000010921D0280912206E82FFF27EE0FFF1F5A
:10441000E15BF84F808191819F938F93809121067A
:10442000E82FFF27EE0FFF1FE15BF84F808191819E
:104430009F938F938AE895E09F938F93DF92CF921B
:10444000FE01099584E180931D02EDB7FEB7389611
:10445000EDBF80912406E82FFF27EE0FFF1FE15BE1
:10446000F84F808191819F938F9380912306E82F4D
:10447000FF27EE0FFF1FE15BF84F8081918181588C
:104480009F4F9F938F938AE995E09F938F93DF923D
:10449000CF92E091E003F091E103099588E28093E7
:1044A0001D022DB73EB7285F3F4F2DBF80912606D6
:1044B000E82FFF27EE0FFF1FE15BF84F808191810E
:1044C00081589F4F9F938F9380912506E82FFF2758
:1044D000EE0FFF1FE15BF84F8081918181589F4F64
:1044E0009F938F938AEA95E09F938F93DF92CF9269
:1044F000E091E003F091E10309958CE380931D02C4
:104500008DB79EB708968DBF80912806E82FFF27AC
:10451000EE0FFF1FE15BF84F8081918181589F4F23
:104520009F938F9380912706E82FFF27EE0FFF1FA1
:10453000E15BF84F8081918181589F4F9F938F93CA
:104540008AEB95E063C210921D028AEC95E09F937E
:104550008F930AE81FE1DF92CF92FE0109958091C7
:1045600002010F900F900F900F908A3009F09DC0BC
:1045700084E180931D0280914503909146039C0144
:1045800097FF02C0295F3F4F287F821B930B9F93A9
:104590008F93809145039091460397FD079673E0B2
:1045A000959587957A95E1F79F938F932091450391
:1045B0003091460337FF02C0295F3F4F63E03595D6
:1045C00027956A95E1F78091FD019091FE01821B8C
:1045D000930B9F938F9388ED95E09F938F931F93F9
:1045E0000F93E091E003F091E103099588E2809355
:1045F0001D022DB73EB7265F3F4F2DBF809143036D
:10460000909144039C0197FF02C0295F3F4F287F90
:10461000821B930B9F938F9380914303909144034C
:1046200097FD079653E0959587955A95E1F79F93E7
:104630008F93209143033091440337FF02C0295FD9
:104640003F4F43E0359527954A95E1F78091FB016F
:104650009091FC01821B930B9F938F9389EE95E0C1
:104660009F938F931F930F93E091E003F091E103E9
:1046700009958CE380931D028DB79EB70A968DBF76
:1046800080914103909142039F938F9380914103C6
:10469000909142032091F9013091FA01821B930B12
:1046A0009F938F938AEF95E0ADC08B3019F08431E2
:1046B00008F4ADC084E180931D0280914503909180
:1046C00046039C0197FF02C0215F3F4F207F821B62
:1046D000930B97FD0196959587959F938F93809166
:1046E00045039091460397FD0F9624E09595879595
:1046F0002A95E1F79F938F932091450330914603CC
:1047000037FF02C0295F3F4FC3E035952795CA9513
:10471000E1F78091FD019091FE01821B930B9F9325
:104720008F9388E096E09F938F931F930F93E09170
:10473000E003F091E103099588E280931D022DB713
:104740003EB7265F3F4F2DBF8091430390914403B6
:104750009C0197FF02C0215F3F4F207F821B930B7C
:1047600097FD0196959587959F938F93809143032D
:104770009091440397FD0F96A4E095958795AA958F
:10478000E1F79F938F93209143033091440337FFC8
:1047900002C0295F3F4FF3E035952795FA95E1F781
:1047A0008091FB019091FC01821B930B9F938F934F
:1047B0008AE196E09F938F931F930F93E091E0031C
:1047C000F091E10309958CE380931D028DB79EB7AC
:1047D0000A968DBF809141039091420397FD019607
:1047E000959587959F938F93809141039091420374
:1047F0002091F9013091FA01821B930B9F938F93C3
:104800008CE296E09F938F931F930F9303C18D309B
:1048100009F0CBC484E180931D0280911301992794
:104820009F938F93809145039091460397FD0F9638
:1048300074E0959587957A95E1F79F938F932091F2
:1048400045033091460337FF02C0295F3F4F63E0C5
:10485000359527956A95E1F78091FD019091FE01CC
:10486000821B930B9F938F938BE396E09F938F9381
:104870001F930F93E091E003F091E103099588E223
:1048800080931D022DB73EB7265F3F4F2DBF80910D
:10489000120199279F938F93809143039091440332
:1048A00097FD0F9654E0959587955A95E1F79F935C
:1048B0008F93209143033091440337FF02C0295F57
:1048C0003F4F43E0359527954A95E1F78091FB01ED
:1048D0009091FC01821B930B9F938F938FE496E042
:1048E0009F938F931F930F93E091E003F091E10367
:1048F00009958CE380931D028DB79EB70A968DBFF4
:104900008091110199279F938F93809141039091FA
:10491000420397FD0196959587959F938F9380917C
:104920004103909142032091F9013091FA01821BD9
:10493000930B9F938F9383E696E09F938F931F93A0
:104940000F93E091E003F091E1030995EDB7FEB715
:104950003A9668C010921D0287E796E09F938F9366
:10496000DF92CF92FE01099584E180931D020F90A2
:104970000F900F900F9080913B0390913C039F9379
:104980008F938091F5019091F6019F938F9384E826
:1049900096E09F938F93DF92CF92E091E003F091A6
:1049A000E103099588E280931D022DB73EB7285F89
:1049B0003F4F2DBF8091390390913A039F938F937E
:1049C0008091F7019091F8019F938F9383E996E08E
:1049D0009F938F93DF92CF92E091E003F091E103F8
:1049E00009958CE380931D028DB79EB708968DBF05
:1049F00080913503909136039F938F938091F301BB
:104A00009091F4019F938F9382EA96E09F938F9306
:104A1000DF92CF92E091E003F091E1030995EDB7C9
:104A2000FEB73896EDBFC1C310921D0280911E01E2
:104A300090911F016AE070E00E94497A9F938F93E2
:104A400080911E0190911F016AE070E00E94497AF6
:104A50007F936F9381EB96E09F938F93DF92CF923A
:104A6000FE01099584E180931D022DB73EB7285FB2
:104A70003F4F2DBF8091A8089091A9086AE070E08F
:104A80000E94357A9F938F938091A8089091A908EE
:104A90006AE070E00E94357A7F936F9385EC96E030
:104AA0009F938F93DF92CF92E091E003F091E10327
:104AB000099588E280931D028DB79EB708968DBF39
:104AC0008091AA089091AB089F938F9389ED96E00F
:104AD0009F938F93DF92CF92E091E003F091E103F7
:104AE00009958CE380931D02EDB7FEB73696EDBFB6
:104AF0008091AC089091AD089F938F9389EE96E0DA
:104B00009F938F93DF92CF92E091E003F091E103C6
:104B100009952DB73EB72A5F3F4F4FC110921D0236
:104B20008BEF96E09F938F93DF92CF92FE010995D2
:104B300084E180931D020F900F900F900F90809151
:104B40004F07909150079F938F9384E097E09F9336
:104B50008F93DF92CF92E091E003F091E10309950A
:104B600088E280931D028DB79EB706968DBF809117
:104B7000D60299279F938F9384E197E09F938F9319
:104B8000DF92CF92E091E003F091E10309958CE38D
:104B900080931D02EDB7FEB73696EDBF80914E07AC
:104BA000992701979F938F9384E297E0A9CF109262
:104BB0001D0284E397E09F938F93DF92CF92FE01D3
:104BC000099584E180931D020F900F900F900F9034
:104BD00080918F01909190019F938F938CE397E048
:104BE0009F938F93DF92CF92E091E003F091E103E6
:104BF000099588E280931D028DB79EB706968DBFFA
:104C00008091C5079091C6079F938F938AE497E0A0
:104C10009F938F93DF92CF92E091E003F091E103B5
:104C200009958CE380931D02EDB7FEB73696EDBF74
:104C30008091EE029091EF029F938F9388E597E029
:104C40005FCFC7EDCC2EC2E0DC2E20E030E0E901E2
:104C5000B3E0FB2EC0931D02F60181916F019927ED
:104C60009F938F9389010F5F1F4F1F930F9386E6CA
:104C700097E09F938F938AE89FE19F938F93E091B2
:104C8000E003F091E10309952DB73EB7285F3F4F50
:104C90002DBFFA9464969801F7FEDCCF86C2ABED87
:104CA000CA2EA2E0DA2EC0E0D0E08E01F3E0FF2EA3
:104CB00000931D02F60181916F0199279F938F93B5
:104CC0002596DF93CF9383E797E09F938F938AE8AE
:104CD0009FE19F938F93E091E003F091E1030995A9
:104CE0002DB73EB7285F3F4F2DBFFA940C5E1F4F84
:104CF0002497F7FEDDCF59C210921D0280E897E09D
:104D00009F938F930AE81FE1DF92CF92FE010995EE
:104D100084E180931D020F900F900F900F9080916F
:104D20006E0199279F938F9388E897E09F938F93C5
:104D3000DF92CF92E091E003F091E103099588E2E0
:104D400080931D028DB79EB706968DBF8091D401CA
:104D50009091D50197FD03969595879595958795A3
:104D60009F938F9386E997E09F938F931F930F9361
:104D7000E091E003F091E10309958CE380931D023B
:104D8000EDB7FEB73696EDBF8091500699279F93F9
:104D90008F9380914F0699279F938F9384EA97E092
:104DA0009F938F931F930F93E091E003F091E103A2
:104DB00009952DB73EB7285F3F4F2DBFF6C1109222
:104DC0001D0282EB97E09F938F937AE8A72E7FE1F5
:104DD000B72EDF92CF92FE0109950F900F900F90A2
:104DE0000F90CEEED6E000E010E062E0F62E802FCD
:104DF0008C5E80931D028B8D99278F7790709F9387
:104E00008F938B8999278F7790709F938F938B8542
:104E100099278F7790709F938F938B8199278F77A6
:104E200090709F938F9382EC97E09F938F93BF92A4
:104E3000AF92E091E003F091E10309958DB79EB741
:104E40000C968DBFFA940C5E1F4FA096F7FECFCF45
:104E5000ACC110921D0283ED97E09F938F935AE8A7
:104E6000A52E5FE1B52EDF92CF92FE0109950F903E
:104E70000F900F900F90CEEED6E000E010E042E0F1
:104E8000F42E802F8C5E80931D028F8D992787FDD5
:104E900090959F938F938F89992787FD90959F93E6
:104EA0008F938F85992787FD90959F938F938F81FF
:104EB000992787FD90959F938F9382EE97E09F931C
:104EC0008F93BF92AF92E091E003F091E1030995D7
:104ED000EDB7FEB73C96EDBFFA940C5E1F4FA0965F
:104EE000F7FECFCF62C110921D0283EF97E09F9330
:104EF0008F930AE81FE1DF92CF92FE01099584E1CA
:104F000080931D020F900F900F900F9080910907D2
:104F1000881F8827881F97E0899FC00111248D96DC
:104F20009F938F9380910107881F8827881F96E0A1
:104F3000899FC00111248D969F938F938091F906CC
:104F4000881F8827881F95E0899FC00111248D96AE
:104F50009F938F938091F106881F8827881F992738
:104F6000880F991F880F991F8D969F938F9382E0CA
:104F700098E09F938F93DF92CF92E091E003F091BE
:104F8000E103099588E280931D022DB73EB7245FA7
:104F90003F4F2DBF80912907881F8827881F9BE0DE
:104FA000899FC00111248D969F938F938091210733
:104FB000881F8827881F9AE0899FC00111248D9639
:104FC0009F938F9380911907881F8827881F99E0E6
:104FD000899FC00111248D969F938F938091110713
:104FE000881F8827881F992723E0880F991F2A95F3
:104FF000E1F78D969F938F9386E198E09F938F932F
:10500000DF92CF92E091E003F091E10309958CE308
:1050100080931D028DB79EB70C968DBF809131078E
:10502000881F8827881F9CE0899FC00111248D96C6
:105030009F938F938AE298E09F938F93DF92CF9212
:10504000E091E003F091E103099580913907EDB714
:10505000FEB73696EDBF87FF12C080E480931D0235
:105060008BE398E09F938F93DF92CF92E091E003E0
:10507000F091E10309950F900F900F900F908091A0
:10508000410787FF12C084E480931D028EE398E0FD
:105090009F938F931F930F93E091E003F091E103AF
:1050A00009950F900F900F900F908091490787FFFF
:1050B0007CC088E480931D0281E498E09F938F93E5
:1050C0001F930F93E091E003F091E10309950F9096
:1050D0000F900F900F9069C010921D0284E498E029
:1050E0009F938F93DF92CF92FE01099584E1809385
:1050F0001D020F900F900F900F908091AA01909138
:10510000AB019F938F9382E598E09F938F93DF92FB
:10511000CF92E091E003F091E103099588E280935A
:105120001D022DB73EB72A5F3F4F2DBF8091AC01C6
:105130009091AD019F938F938FE598E09F938F930C
:10514000DF92CF92E091E003F091E103099589E4C9
:1051500080931D028DB79EB706968DBF8CE698E0B2
:105160009F938F93DF92CF92E091E003F091E10360
:10517000099580911B020F900F900F900F9083FF65
:1051800014C01092AD011092AC0160E070E08EE0AE
:1051900090E00E94E02A09C080912001281719F4AC
:1051A00021502093200110921C0210921B02DF91CB
:1051B000CF911F910F91FF90DF90CF90BF90AF9054
:1051C0000895F999FECF92BD81BDF89A80B59927CF
:1051D0000895F999FECF1FBA92BD81BD60BD0FB68B
:1051E000F894FA9AF99A0FBE08954AEA20E030E05E
:1051F0002617370740F4FC018191480F2F5F3F4F7E
:1052000026173707C8F3842F99270895EAEA40E064
:1052100050E04617570778F49C01F999FECF32BD4C
:1052200021BDF89A80B5E80F4F5F5F4F2F5F3F4F6A
:105230004617570790F38E2F9927089581E08093A2
:10524000230682E08093220683E08093210684E097
:105250008093240685E08093250686E080932606C9
:1052600087E08093270688E08093280689E0809372
:1052700029068AE080932A068BE080932B068CE037
:1052800080932C06089588E5809320068091020182
:10529000843150F08AE080934006109264068BE1DE
:1052A00080933C068EE40AC083E08093400680E24F
:1052B000809364068EE180933C0685E580936106C9
:1052C0008093620680E2809363068AE680932D06CF
:1052D00082E280938A0664E0609347061092830618
:1052E0001092800648E040933A0656EE50933B06F3
:1052F00030E430933D069EE190932E068FEF80932D
:1053000030062FE02093310690932F06109233063B
:1053100040933406309335061092360620933206B9
:105320001092490610924A0610924B0610924C06B3
:10533000109266061092670610926806109269062F
:1053400090E890934D0632E330934E0682E08093CE
:10535000890620934F0650935006609355068DE7BB
:10536000809358068093590680935A06909351066D
:1053700025E52093520686E4809353068CED8093B6
:1053800054068CE380935606109257068FE580935F
:105390006A0683EF80936C068AEA80936E06809398
:1053A0006F0684E180936B0680936D0630935B06F5
:1053B0009AE590935C0630935D06109288068EEF16
:1053C0008093700684E680937106909372069093A2
:1053D0007306909374068BE480937506209376068B
:1053E000809377061092780686E080937906409342
:1053F0007A0690937B068AE280937C0685EF809301
:105400007D068CE880937E0685E080937F0610926F
:1054100081061092820681E2809344068DE2809399
:1054200045069093460610928406109285061092C7
:10543000860686E98093870690935E0687E38093CD
:105440005F060895CF93DF930E9443298AE08093FB
:10545000370680E18093380626E0209339069AE5E6
:1054600090933E0688E780933F0690934106809391
:1054700042062093430680E2809348068CE38093A3
:1054800060068BE480936506ABE8B6E08CE0E1E271
:10549000F1E0ED01019009928A95E1F767E770E08C
:1054A000CD018B5690400E94F52880939706DF919E
:1054B000CF910895CF93DF930E94432988E0809392
:1054C000370630E13093380626E02093390694E61B
:1054D00090933E0688E780933F0690934106809321
:1054E0004206209343063093480686E48093600684
:1054F00080936506ABE8B6E08CE0E7E2F1E0ED0111
:10550000019009928A95E1F767E770E0CD018B562B
:1055100090400E94F52880939706DF91CF910895DF
:10552000CF93DF930E94432926E0209337068AE039
:105530008093380684E08093390694E690933E0683
:1055400088E780933F06909341068093420620931C
:10555000430680E18093480686E48093600680934A
:105560006506ABE8B6E08CE0EFE2F1E0ED0101901A
:1055700009928A95E1F767E770E0CD018B5690407C
:105580000E94F52880939706DF91CF910895F999AD
:10559000FECF92BD81BDF89A80B599270895F999FB
:1055A000FECF1FBA92BD81BD60BD0FB6F894FA9AC6
:1055B000F99A0FBE089561EE78E20E9498780895F6
:1055C00049EE58E20E94D2780895EF92FF920F932D
:1055D0001F93CF93C82F8150853008F0C3E088E730
:1055E000C89F800111248CEEE82E8FEFF82EE00E7C
:1055F000F11E67E770E0C7010E940629682F980135
:105600002D593F4F8FB39927AC014270507081FDE7
:10561000F9CF32BD21BDF89A80B5861711F0CA01C5
:1056200021C08FB399279C012270307081FDF9CF82
:10563000F2BCE1BCF89A80B5883511F0C90112C0FE
:1056400088E7C89FC0011124449721EE38E248E75B
:1056500050E0BC0180E296E00E9473780E94B66739
:1056600081E090E0CF911F910F91FF90EF9008950E
:10567000282F863010F025E003C0882309F421E0AC
:10568000F999FECF1FBA82E090E092BD81BD20BDA6
:105690000FB6F894FA9AF99A0FBE0895CF93C82FCF
:1056A00080912006883509F044C0C63010F0C5E06E
:1056B00003C0CC2309F43DC00E947E7767E770E009
:1056C00080E296E00E94F5288093970688E7C89FBD
:1056D000C001112429EE38E248E750E060E276E0AC
:1056E00044970E94B07829EE38E24CE050E061E245
:1056F00076E080E590E00E94B0786CE070E081E2B6
:1057000096E00E94F528282FF999FECF1FBA8CE564
:1057100090E092BD81BD20BD0FB6F894FA9AF99A37
:105720000FBE8C2F0E94382B0E94B66781E090E05C
:1057300002C080E090E0CF9108956DE470E088EEC3
:1057400093E00E940629482F8FB399279C0122706D
:10575000307081FDF9CF85E394E092BD81BDF89A68
:1057600080B5841779F48FB399279C01227030702B
:1057700081FDF9CF88EE93E092BD81BDF89A80B5A6
:10578000813011F0C901089521EE38E24EE450E075
:1057900068EE73E088E996E00E94737881E090E01B
:1057A0000895809198068130A9F46DE470E088E94D
:1057B00096E00E94F5288093E50629EE38E24EE453
:1057C00050E068E976E088EE93E00E94B07881E0EE
:1057D00090E0089580E090E00895CF93DF9381E01A
:1057E00080939806E8E9F6E08FE01586168617861E
:1057F000108A8150349687FFF8CF80E48093A50605
:105800008093A6061092A7068093A8068093A90607
:1058100090EC9093AA061092AB068093AC0680930E
:10582000AD061092AE069093AF069093B0068093AB
:10583000B1061092B2068093B3069093B406A9E91C
:10584000B6E087E0E5E3F1E0ED01019009928A9589
:10585000E1F76DE470E0CD0101970E94F528809397
:10586000E506DF91CF910895F999FECF82E090E0AF
:1058700092BD81BDF89A80B5282F863078F023E05C
:10588000322FF999FECF1FBA82E090E092BD81BD20
:1058900030BD0FB6F894FA9AF99A0FBE822F992765
:1058A00008951F93CF93C82F162F863010F0C5E0B0
:1058B00003C0882309F4C1E08C2F99278230910519
:1058C00041F08330910544F4019731F40E94222A7B
:1058D00005C00E945A2A02C00E94902A1123E1F0BA
:1058E0006CE070E080E590E00E940629282FF9998D
:1058F000FECF8CE590E092BD81BDF89A80B582170D
:1059000059F421EE38E24CE050E060E570E081E2CD
:1059100096E00E94737802C00E941E298C2F0E947C
:105920004E2BCF911F910895DF92EF92FF920F932C
:105930001F93CF93FF24DF2CEF2C81E090E00E9497
:10594000C72A883511F031E0E32E6CE070E080E585
:1059500090E00E940629C82FF999FECF8CE590E0CF
:1059600092BD81BDF89A80B58C1711F421E0D22E3A
:10597000C1E001E010E0EE2029F48C2F0E94E52A1E
:105980008823C9F591E0F92E1F930F9384E798E0DF
:105990009F938F9381E892E19F938F93E091E0032F
:1059A000F091E10309952DB73EB72A5F3F4F2DBF18
:1059B0000230110549F0033011054CF40130110596
:1059C00031F40E94222A05C00E945A2A02C00E9475
:1059D000902ADD2059F021EE38E24CE050E060E5FD
:1059E00070E081E296E00E94737802C00E941E2956
:1059F0008C2F0E944E2BCF5F0F5F1F4FC63008F4D5
:105A0000BACFFF2019F083E00E94382B0E94342C7B
:105A1000C82F0E94E52A8C2F99279F938F938AE99C
:105A200098E09F938F9301E812E11F930F93E09109
:105A3000E003F091E103099581E090E00E94C72A1C
:105A40002DB73EB72A5F3F4F2DBF8F3F21F00E94F9
:105A50009D2B882399F483EB98E09F938F931F935A
:105A60000F93E091E003F091E10309950E94ED2B83
:105A70000E94D12B0F900F900F900F90EE2029F0E5
:105A800068E581E090E00E94CF2A10921F0690E026
:105A9000E5EAF6E0CFE08081349618160CF49F5FBB
:105AA000C150C7FFF8CF90931F06892F99279F9366
:105AB0008F9389E996E09F938F9384ED98E09F936D
:105AC0008F931F930F93E091E003F091E103099509
:105AD0008DB79EB708968DBF85EF98E09F938F9303
:105AE0001F930F93E091E003F091E10309950F906C
:105AF0000F900F900F90CF911F910F91FF90EF900B
:105B0000DF900895982F2FB7F8943998389A88B174
:105B1000836088B98091B9008C7F8093B9008AE254
:105B20008093B8001092280210922602109225024B
:105B3000992379F0EEEEF6E08BE01082118212826A
:105B4000138214821582168217828150389687FF3D
:105B5000F4CF78942FBF08951092280284E980939F
:105B6000BC0080E88093BC001092BD001092BA0087
:105B70001092BB001092B9001092B800109224024B
:105B800080E00E94822D1092BB0085E88093BC00CB
:105B90008091220282608093220208951F920F92C8
:105BA0000FB60F9211242F933F934F935F938F93D0
:105BB0009F93EF93FF9380912802282F3327442748
:105BC00055278F5F80932802F9012731310508F0AE
:105BD000C2C2EF59FF4F0C94D07A81E08093240227
:105BE00009C0809126028C3090F4809126028F5F4C
:105BF0008093260280912602E82FFF27EE0FFF1FD9
:105C0000EE0FFF1FE856F94F8585181654F780915F
:105C100026028C3070F01092210210922002109215
:105C2000260285E08093280280912502880F8D5AF4
:105C300004C080912602880F8E5A8093BB0085E8AD
:105C40007FC280912602E82FFF2783E0EE0FFF1F1F
:105C50008A95E1F7E251F94F81818093BB0085E895
:105C60008093BC0080912602E82FFF27EE0FFF1FD4
:105C7000EE0FFF1FEE0FFF1FE251F94F808180FFF3
:105C800091C080912602E82FFF27EE0FFF1FEE0F35
:105C9000FF1FEE0FFF1FE251F94F8281882329F089
:105CA00080911F06873008F46CC280912002909189
:105CB0002102892B09F065C280911E0290911F027A
:105CC000892B09F05EC26EC08091260221E030E08F
:105CD00002C0220F331F8A95E2F780911E02909135
:105CE0001F0228233923232B79F080912602E82FE5
:105CF000FF27EE0FFF1FEE0FFF1FEE0FFF1FE251FA
:105D0000F94F80E184830DC080912602E82FFF27A0
:105D1000EE0FFF1FEE0FFF1FEE0FFF1FE251F94FB7
:105D2000148280912602E82FFF2753E0EE0FFF1F19
:105D30005A95E1F7E251F94F8481282F332743E048
:105D4000220F331F4A95E1F780912602E82FFF27A3
:105D500093E0EE0FFF1F9A95E1F7E251F94F828130
:105D60008770822B8093BB0085E88093BC002091D4
:105D7000260281E090E002C0880F991F2A95E2F781
:105D8000209120023091210282239323892B51F00C
:105D900086EE96E090932C0280932B0288E080930D
:105DA0002D02EFC184E089C1E0912B02F0912C0219
:105DB00081918093BB0085E88093BC00F0932C0216
:105DC000E0932B0280912D02815080932D02882335
:105DD00009F4D7C183E071C18091B900803351F5D6
:105DE00080912902882329F4809126028F5F809375
:105DF000290280912602E82FFF2783E0EE0FFF1F84
:105E00008A95E1F7E251F94F838199278F77907056
:105E10008F3791057CF480912602E82FFF27EE0F43
:105E2000FF1FEE0FFF1FEE0FFF1FE251F94F83819F
:105E30008F5F83831092280284E98093BC008AE0FC
:105E400090E090933E0180933D01809126028F5F08
:105E500080932602109228026DC18091B90080348F
:105E6000C9F180912502E82FFF27EE0FFF1FEE0FEB
:105E7000FF1FEE0FFF1FE251F94F83818F7783835E
:105E8000809125028F5F80932502809125028C30BE
:105E9000A0F01092250210921F0210921E02809113
:105EA0002A028F5F80932A028C3038F010922A02E7
:105EB000809122028D7F8093220280912202816054
:105EC000809322021092280284E98093BC001092F1
:105ED000240273C080912502E82FFF27EE0FFF1FD9
:105EE000EE0FFF1FEE0FFF1FE251F94F8381806815
:105EF000838380912502E82FFF27EE0FFF1FEE0F0F
:105F0000FF1FEE0FFF1FE251F94F808180FF2FC06E
:105F100080912502E82FFF2753E0EE0FFF1F5A95CF
:105F2000E1F7E251F94F84819927009751F04097AA
:105F3000D9F586EE96E090932C0280932B0288E0B0
:105F400031C080912502992743E0880F991F4A9517
:105F5000E1F78D50994F90932C0280932B029091F2
:105F6000250280912A029817E1F483E01BC08091FA
:105F70002502992733E0880F991F3A95E1F78D5054
:105F8000994F90932C0280932B028091220281FDE5
:105F900006C09091250280912A02981711F482E0A0
:105FA00001C081E080932D0280912D02813011F497
:105FB00085E801C085EC8093BC0080912902809324
:105FC000230210922902DDC0E0912B02F0912C02F5
:105FD0008091BB00808380912B0290912C020196CE
:105FE00090932C0280932B0280912D0281508093FC
:105FF0002D02823010F085EC5DC0813011F485E80F
:1060000059C08091220281FF2DC08091A00280FDA5
:106010001DC080912502E82FFF2723E0EE0FFF1F10
:106020002A95E1F7E251F94F86818A3F79F4809110
:106030002502E82FFF2793E0EE0FFF1F9A95E1F767
:10604000E251F94F8081816080830CC080912502EC
:10605000E82FFF2783E0EE0FFF1F8A95E1F7E2515B
:10606000F94F1082809125028F5F809325028091E5
:1060700025028C30A0F01092250210921F0210927F
:106080001E0280912A028F5F80932A028C3038F0A2
:1060900010922A02809122028D7F80932202109218
:1060A000280284E98093BC00809122028160809361
:1060B000220265C08093BC0086E08093280261C004
:1060C00088E9BBCD80912702880F805FB6CD809193
:1060D000270299278130910561F0823091051CF4E7
:1060E000892B21F04EC0029739F04BC080911301EB
:1060F000A4CD80911201A1CD809111019ECD80E8A7
:106100009CCD1092280284E98093BC001092240256
:106110008AE090E090933E0180933D0180912702B8
:10612000823088F4809127028F5F8093270282E17A
:1061300080932802809122028E7F8093220285EA3A
:106140008093BC001EC010922702809122028160C1
:106150008093220216C01092280284E98093BC002A
:10616000809122028160809322028AE090E09093E5
:106170003E0180933D01109226021092250210925A
:106180002402FF91EF919F918F915F914F913F91E9
:106190002F910F900FBE0F901F9018951F93CF93C4
:1061A000DF93182F8091D502882321F48091B901C3
:1061B000882319F081E090E097C01D3008F092C06C
:1061C0001123B1F0E12FFF2723E0EE0FFF1F2A95E7
:1061D000E1F7E251F94F35978081359688230CF02D
:1061E00081C03897808180FD03C083E090E07CC04F
:1061F0008091E606823019F084E090E075C067E097
:1062000070E086EE96E00E94F5289091ED068917E1
:1062100019F085E090E068C080ED97E00E9490164C
:10622000EC018091220280FD05C0CE010E949916EA
:106230008823B9F3112319F48FEF90E00BC0212FBD
:1062400033272150304081E090E002C0880F991F31
:106250002A95E2F79093210280932002A1E0B0E01A
:10626000EEEEF6E040E050E06BE0CD01042E02C01F
:10627000880F991F0A94E2F72091200230912102A1
:1062800082239323892B11F01182128261504F5F78
:106290005F4F389667FFE9CF1092260210922802CE
:1062A000809122028E7F8093220285EA8093BC0037
:1062B0008091220280FD05C0CE010E94991688239C
:1062C000B9F38091200290912102892B29F0CE010F
:1062D0000E949916882311F3809120029091210247
:1062E000009711F082E090E0DF91CF911F91089527
:1062F0000F931F93CF93DF93982F8091D50288231C
:1063000021F48091B901882319F081E090E092C0D6
:106310009D30A0F4992319F486E090E08BC0C92F3A
:10632000DD27FE0133E0EE0FFF1F3A95E1F7E25162
:10633000F94F35978081359687FD03C082E090E064
:1063400079C03897808180FD03C083E090E072C0FF
:1063500080ED97E00E9490168C018091220280FDD2
:1063600005C0C8010E9499168823B9F3219721E03E
:1063700030E0C90102C0880F991FCA95E2F79093D7
:106380001F0280931E02D901EEEEF6E040E050E0DD
:106390006BE0CD01042E02C0880F991F0A94E2F72A
:1063A00020911E0230911F0282239323892B11F02A
:1063B0001182128261504F5F5F4F389667FFE9CFBD
:1063C000109225021092E6061092ED061092280215
:1063D000809122028E7F8093220285EA8093BC0006
:1063E0008091220280FD05C0C8010E949916882371
:1063F000B9F380911E0290911F02892B29F0C801E8
:106400000E949916882311F38091E606823019F0D4
:1064100084E090E00FC067E070E086EE96E00E94B6
:10642000F5289091ED06891719F085E090E002C0FB
:1064300080E090E0DF91CF911F910F910895CF936D
:10644000DF9380E022E83FEFC3E8D7E0EFE4F7E036
:10645000DF01853020F411961C921E9202C0318318
:1064600020831982188222968F5F129632968A3183
:1064700080F3109242031092410310924403109251
:1064800043031092460310924503DF91CF91089584
:106490001F920F920FB60F9211240F931F932F93F9
:1064A0003F934F935F936F937F938F939F93AF939C
:1064B000BF93CF93DF93EF93FF9380918A0682FD82
:1064C000D3C0409186005091870080912F02909117
:1064D0003002481B590B8091860090918700909361
:1064E000300280932F02CA018D549440A091310252
:1064F000B0913202835F9A4178F4809131028093A7
:106500004E07149714F01092410181E090E09093AF
:106510003202809331020FC2AD30B1050CF00BC2D4
:10652000CA018B5F9040845B914008F078C08091F5
:106530003F0190914001481B590BFD01EA0FFB1FE1
:10654000E15BF84F80819181FA01E81BF90BCF01E3
:10655000F7FF03C0909581959F4F06975CF480915B
:10656000D602883C20F48091D602865F01C088EC78
:106570008093D602FD01EA0FFB1FE15BF84F80819B
:1065800091819C01220F331F280F391F240F351FC3
:1065900037FF02C02D5F3F4FE901D595C795D595CF
:1065A000C795CA0101968C179D0714F4219706C060
:1065B00041505040C417D5070CF421968091D60263
:1065C000833CE0F08D010A0F1B1FF801E15BF84FDF
:1065D000808191819E01281B390BC90163E070E025
:1065E0000E94497ACB01880F991F860F971F0D577C
:1065F000184FD80111969C938E9307C0AA0FBB1F0A
:10660000AD57B84F11961C921E92E0913102F09155
:106610003202EE0FFF1FE15BF84FD183C083209160
:106620003102309132022F5F3F4F3093320220937C
:10663000310280910201843108F07DC1253031059D
:1066400011F45D9A01C05D988091310290913202FF
:106650008630910511F45C9A01C05C98079711F49B
:106660005B9A69C15B9867C1409186005091870031
:106670008091330290913402481B590B809186001F
:10668000909187009093340280933302CA018D5415
:10669000944060919D02835F9A4108F07AC06093B4
:1066A0002E0280912E02843008F453C090914E0740
:1066B00080912E02981709F04CC050919E025B30D9
:1066C00008F43FC01092410110929D0240E05F31FA
:1066D000C0F0E42FFF27EE0FFF1F9F0127593D4F0A
:1066E000DF01A15BB84F8D919C91D9018D939C9353
:1066F000DF01AD57B84F8D919C91ED57FD4F9183C0
:106700008083E42FFF27EE0FFF1F9F01215B384F8F
:10671000DF01AB5CBD4F8D919C91D90111969C938B
:106720008E93DF01A15BBD4F8D919C91ED57F84F8A
:1067300091838083842F8F5F482F8D3040F2809328
:106740009D0280919E028F3FB9F08F5F80939E02E1
:1067500013C080919E02853620F08AE080939E02CD
:1067600002C010929E02809102018A3011F08431A1
:1067700010F0289A01C0289881E080939D028091B2
:10678000D502882309F0D7C080912E0280934E074E
:10679000D2C06D3008F0A7C0CA018B5F9040845B07
:1067A000914008F082C080913F0190914001481BC8
:1067B000590BE62FFF27EE0FFF1FEB5CFD4F80818B
:1067C0009181FA01E81BF90BCF0105960B97B0F404
:1067D00080919E028A3120F08091D602865F05C0AA
:1067E0008B3028F08091D6028E5F8093D602809104
:1067F000D602893C18F088EC8093D602E62FFF275A
:10680000EE0FFF1FEB5CFD4F808191819C01220FF9
:10681000331F280F391F240F351F37FF02C02D5F8C
:106820003F4FE901D595C795D595C795CA01019602
:106830008C179D0714F4219706C041505040C4178F
:10684000D5070CF421968091D6028E3BD8F0E62F26
:10685000FF27EE0FFF1FDF01AB5CBD4F8D919C91B9
:106860009E01281B390BC90163E070E00E94497A40
:10687000CB01880F991F860F971FE15BFD4F918316
:10688000808308C0E62FFF27EE0FFF1FE15BFD4F5F
:106890001182108280919D02E82FFF27EE0FFF1FCB
:1068A000EB5CFD4FD183C08309C0809102018A3027
:1068B00011F0843110F0289A01C0289880910201CB
:1068C000843188F480919D02853011F45D9A05C071
:1068D0005D98863011F45C9A05C05C98873011F49D
:1068E0005B9A01C05B9880919D02843120F48F5F98
:1068F00080939D0220C08431F1F4809102018A309E
:1069000011F0843110F0289A01C028988EE180930C
:106910009D022CE0C3E8D7E0A9E6B2E0EFE4F7E09F
:106920008D919D919183808332961982188222964F
:10693000215027FFF5CFFF91EF91DF91CF91BF91CC
:10694000AF919F918F917F916F915F914F913F9107
:106950002F911F910F910F900FBE0F901F901895C0
:10696000EF92FF920F931F9380913C069927880F17
:10697000991F880F991F7C010027F7FC0095102FA5
:106980008091300390913103A0913203B091330391
:10699000BC01CD01A80197010E947E7A30937C054D
:1069A00020937B058091280390912903A0912A03CD
:1069B000B0912B03BC01CD01A80197010E947E7A02
:1069C00030937E0520937D0580910C0890910D08F1
:1069D00097FD039695958795959587959093800556
:1069E00080937F0580911C0890911D0897FD039668
:1069F00095958795959587959093820580938105C8
:106A000080914103909142032091F9013091FA0164
:106A1000821B930B90938405809383058091D00211
:106A20009091D102A091D202B091D302BC01CD01CC
:106A300025E030E040E050E00E947E7A3093860509
:106A4000209385058091F3019091F401909388053E
:106A50008093870580918F019091900190938C0590
:106A600080938B0580911E0190911F0190938E055C
:106A700080938D058091D6029927909390058093FD
:106A80008F058091C5079091C607909392058093DA
:106A900091058091EF069927909394058093930533
:106AA0008091F7069927909396058093950580919C
:106AB000FF06992790939805809397058091070783
:106AC000992790939A05809399058091D40190918C
:106AD000D5019093A4058093A3058091A808909177
:106AE000A9089093A8058093A7058091AC08909180
:106AF000AD089093AA058093A9058091CC0290914E
:106B0000CD02A091CE02B091CF02BC01CD0125E013
:106B100030E040E050E00E947E7A3093AC05209354
:106B2000AB058091EE029091EF029093B2058093B5
:106B3000B1058091AE0899279093B6058093B5056D
:106B40008091A3039091A4039093B8058093B70517
:106B50008091A1039091A2039093BA058093B90507
:106B60008091F903882321F48091FA03882321F08E
:106B700080917A05816003C080917A058E7F809331
:106B80007A051F910F91FF90EF9008951F93CF9377
:106B9000DF93182FEB018091D502882309F58091AE
:106BA00002018C3010F4299801C0299A11501F3F1E
:106BB00081F0D093DB01C093DA018091DA019091EA
:106BC000DB01892BD1F7CE018C0F9D1F0E94A516EA
:106BD000EDCF809102018C3010F4299A01C02998E0
:106BE000DF91CF911F910895CF93DF9380910201A0
:106BF0008D3011F40E949E1A10927A008091FD014E
:106C00009091FE019093D1078093D0078091FB0172
:106C10009091FC019093C1078093C0078091F90186
:106C20009091FA0190931208809311082091F50138
:106C30003091F601C901880F991F880F991F820FA3
:106C4000931F820F931F90930D0880930C0820913F
:106C5000F7013091F801C901880F991F880F991F1A
:106C6000820F931F820F931F90931D0880931C081F
:106C70008FEC80937A00A7EDB2E0C5E2D6E097E012
:106C80008991E82FFF27EE0FFF1FE15BF84F01907E
:106C9000F081E02DE158FF4F1E161F061CF0E0E0CA
:106CA000F0E005C0EF3FF10514F0EFEFF0E08C915C
:106CB000282F3327E217F30714F4815004C02E174E
:106CC0003F0714F48F5F8C939150119697FFD8CFA4
:106CD000809161069927AA27BB27BC01CD0124EC2E
:106CE00039E040E050E00E940A7ADC01CB01809359
:106CF000870190938801A0938901B0938A018091C4
:106D000062069927AA27BB27BC01CD010E940A7AF7
:106D1000DC01CB018093830190938401A0938501D2
:106D2000B0938601DF91CF910895A0E0B0E0EBE948
:106D3000F6E30C949F7A882EC0E0D0E07E016E01CD
:106D40001092F903469AD0933C03C0933B03D0932F
:106D50003A03C0933903D0933603C0933503D093DD
:106D60004603C0934503D0934403C0934303D09399
:106D70004203C093410310926B0110926A0110927A
:106D8000ED010E94F43584E690E00E94B2160E9464
:106D9000F43580912D0680FF10C0809114019091F0
:106DA0001501875B934038F480911401909115018F
:106DB0008E5E924010F40E94431A0FE18AE090E048
:106DC0000E94B2168091F9019091FA01C80FD91F63
:106DD0008091FD019091FE01E80EF91E8091FB016A
:106DE0009091FC01C80ED91E015007FFE7CF970113
:106DF000205F3F4F3695279536952795309346036C
:106E000020934503C601409696958795969587955C
:106E100090934403809343036096F5E0D695C7951D
:106E2000FA95E1F7D0934203C09341039093400356
:106E300080933F0330933E0320933D03882009F461
:106E400041C080910C0890910D0897FF03C0909568
:106E500081959F4F6CE070E00E94497A9B0170938E
:106E60003C0360933B0380911C0890911D0897FFA1
:106E700003C0909581959F4F6CE070E00E94497A25
:106E800070933A03609339038091C2059091C305D2
:106E90009093360380933503B90184E090E00E941B
:106EA000E02A6091390370913A0386E090E00E94F5
:106EB000E02A609135037091360388E090E00E94EB
:106EC000E02A65C084E090E00E94DB2A90933C03B6
:106ED00080933B0386E090E00E94DB2A90933A0384
:106EE0008093390388E090E00E94DB2A9C01909314
:106EF00036038093350380913B0390913C0381508E
:106F0000984050F48091390390913A038150984011
:106F100018F421503440D8F186E199E09F938F9383
:106F200081E892E19F938F93E091E003F091E10378
:106F3000099580910C0890910D0897FF03C09095DA
:106F400081959F4F6CE070E00E94497A70933C03FA
:106F500060933B0380911C0890911D0897FF03C02C
:106F6000909581959F4F6CE070E00E94497A7093F4
:106F70003A03609339038091C2059091C3059093C1
:106F80003603809335030F900F900F900F9010925F
:106F9000D1071092D0071092C1071092C00710922B
:106FA00012081092110884E690E00E94B2168091B7
:106FB000F5019091F6019C01220F331F220F331F20
:106FC000280F391F280F391F30930D0820930C0804
:106FD0008091F7019091F8018C01000F111F000FB3
:106FE000111F080F191F080F191F10931D08009378
:106FF0001C0880913C06C82EDD24EE24FF24442783
:1070000037FD4095542FC701B6010E940A7A4B0103
:107010005C0160933003709331038093320390934B
:1070200033039801442737FD4095542FC701B6011B
:107030000E940A7ADC01CB018093280390932903F4
:10704000A0932A03B0932B0380920C0390920D031C
:10705000A0920E03B0920F03809304039093050354
:10706000A0930603B093070310920003109201034C
:107070001092020310920303809116019091170160
:10708000A0911801B09119019093C5058093C40592
:107090001092EC011092EB011092F0021092F102AA
:1070A0001092F2021092F30200918F011091900160
:1070B0001093EF020093EE0284E690E090938C012F
:1070C00080938B0182E390E09093DB018093DA015F
:1070D000809161069927AA27BB27BC01CD0124EC2A
:1070E00039E040E050E00E940A7ADC01CB0188568A
:1070F000954CAF4FBF4F8093870190938801A09329
:107100008901B0938A01809162069927AA27BB273B
:10711000BC01CD010E940A7ADC01CB018856954C56
:10712000AF4FBF4F8093830190938401A09385015B
:10713000B09386011092480110924701C801AA2716
:1071400097FDA095BA2F20914301309144014091C1
:10715000450150914601BC01CD010E940A7ADC0133
:10716000CB018093180890931908A0931A08B09344
:107170001B081092EB021092EA0281E08093010159
:107180000E94B6678091A00284608093A0028FEF76
:10719000809398081092990880E280939A08C7ED2E
:1071A000D2E0A5E2B6E007E08D91E82FFF27EE0FD1
:1071B000FF1FE15BF84F80819181815889930150D5
:1071C00007FFF2CF84E68093D6028091D80188230E
:1071D00011F0469A579A8091450390914603805644
:1071E0009940815C9B4228F08091F90381608093F3
:1071F000F903809143039091440380569940815C48
:107200009B4228F08091F90382608093F90380917A
:107210004103909142038C5291408957954028F048
:107220008091F90384608093F90380913B039091EE
:107230003C038C529140835C914028F08091F9038B
:1072400088608093F9038091390390913A038C52BE
:107250009140835C914028F08091F9038061809394
:10726000F903809135039091360380509240835505
:10727000914028F08091F90380628093F90386E4BD
:1072800080937E01ECE0CDB7DEB70C94BB7AA3E12E
:10729000B0E0EDE4F9E30C94997A80914103909188
:1072A00042032091F9013091FA01821B930B9093D4
:1072B000120880931108809103029091040297FDB7
:1072C00007969C0113E0359527951A95E1F73093C1
:1072D000D1072093D007809101029091020297FD7F
:1072E0000796B3E095958795BA95E1F79093C10716
:1072F0008093C0073093DC072093DB079093D4077B
:107300008093D30780910C0890910D08AC01440F35
:10731000551F480F591F2091F5013091F601C90101
:10732000880F991F880F991F820F931F820F931F39
:10733000480F591F57FF02C04D5F5F4F5595479546
:107340005595479550930D0840930C0880911C0863
:1073500090911D08AC01440F551F480F591F2091F3
:10736000F7013091F801C901880F991F880F991F03
:10737000820F931F820F931F480F591F57FF02C0A0
:107380004D5F5F4F559547955595479550931D080F
:1073900040931C082091F5013091F601C901880F36
:1073A000991F880F991F820F931F820F931F9C01B3
:1073B000442737FD4095542F80912003909121035D
:1073C000A0912203B0912303820F931FA41FB51F26
:1073D0008093200390932103A0932203B09323036F
:1073E0002091F7013091F801C901880F991F880F8A
:1073F000991F820F931F820F931F9C01442737FD13
:107400004095542F80911C0390911D03A0911E0361
:10741000B0911F03820F931FA41FB51F80931C03FD
:1074200090931D03A0931E03B0931F038091E50763
:107430009091E6072091F5013091F601820F931F9C
:107440009093E6078093E5078091140890911508C2
:107450002091F7013091F801820F931F9093150846
:10746000809314088091370390913803019690938C
:107470003803809337038091C2059091C305209112
:10748000350330913603821B930B9C01442737FD53
:107490004095542F8091180390911903A0911A03DD
:1074A000B0911B03820F931FA41FB51F8093180375
:1074B00090931903A0931A03B0931B038FEC80934E
:1074C0007A00109210012091080330910903409135
:1074D0000A0350910B0329873A874B875C8729540D
:1074E0003B46414050402CF028E43BE641E050E070
:1074F0000DC089859A85AB85BC85885B9449AE4F64
:10750000BF4F4CF428EB34E94EEF5FEF2D833E8301
:107510004F83588708C089859A85AB85BC858D8344
:107520009E83AF83B887209110033091110340915F
:107530001203509113032D873E874F87588B295490
:107540003B46414050402CF028E43BE641E050E00F
:107550000DC08D859E85AF85B889885B9449AE4FF7
:10756000BF4F4CF428EB34E94EEF5FEF29833A83A9
:107570004B835C8308C08D859E85AF85B8898983E0
:107580009A83AB83BC83A0911108B0911208BB8B86
:10759000AA8BFD01CF01AA2797FDA095BA2FA09035
:1075A0000003B0900103C0900203D0900303A80E23
:1075B000B91ECA1EDB1EA0920003B0920103C09246
:1075C0000203D0920303E0901808F090190800918C
:1075D0001A0810911B08E80EF91E0A1F1B1FE092E3
:1075E0001808F092190800931A0810931B08F091DC
:1075F000BB02F98BFF2309F098C18091BA0288235E
:1076000009F093C18091080886FF8FC18091C0075F
:107610009091C107AA2797FDA095BA2FBC01CD0173
:1076200029813A814B815C810E940A7A9B01AC01DD
:1076300097FF04C02150384F4F4F5F4FBBE0559527
:10764000479537952795BA95D1F780916A01682EAD
:10765000772488249924CA01B901A40193010E94C6
:107660000A7ADC01CB018093510390935203A093DB
:107670005303B0935403B7FF04C08150904FAF4FF2
:10768000BF4F1C012D01ACE05594479437942794CB
:10769000AA95D1F72092510330925203409253039E
:1076A000509254038091D0079091D107AA2797FD5B
:1076B000A095BA2FBC01CD012D813E814F81588507
:1076C0000E940A7A97FF04C06150784F8F4F9F4FF6
:1076D000FBE09595879577956795FA95D1F7A40185
:1076E00093010E940A7ADC01CB01809355039093A9
:1076F0005603A0935703B0935803B7FF04C08150BB
:10770000904FAF4FBF4F9C01AD01ECE055954795B1
:1077100037952795EA95D1F7209355033093560373
:107720004093570350935803809151039091520313
:107730009093B8078093B7078091550390915603B3
:107740009093BC078093BB0722193309440955095C
:107750002093550330935603409357035093580397
:10776000E20EF31E041F151FE0921808F09219088C
:1077700000931A0810931B08809169018823B1F4C3
:1077800057FF04C02F5F3F4F4F4F5F4F55954795B1
:1077900037952795A21AB30AC40AD50AA092000306
:1077A000B0920103C0920203D09203032A893B895D
:1077B00079010027F7FC0095102F809155039091D7
:1077C0005603A0915703B0915803E80EF91E0A1F03
:1077D0001B1FC801B70129813A814B815C810E943E
:1077E0000A7A9B01AC0197FF04C02150384F4F4FDC
:1077F0005F4F6BE055954795379527956A95D1F77B
:1078000080916B01A82EBB24CC24DD24CA01B901D0
:10781000A60195010E940A7ADC01CB0180934903FD
:1078200090934A03A0934B03B0934C03B7FF04C05B
:107830008150904FAF4FBF4F3C014D013CE09594BC
:107840008794779467943A95D1F760924903709240
:107850004A0380924B0390924C03C801B7012D81DB
:107860003E814F8158850E940A7A97FF04C061507B
:10787000784F8F4F9F4F2BE095958795779567951C
:107880002A95D1F7A60195010E940A7ADC01CB0165
:1078900080934D0390934E03A0934F03B0935003F6
:1078A000B7FF04C08150904FAF4FBF4FAC01BD0137
:1078B0008CE075956795579547958A95D1F74093D4
:1078C0004D0350934E0360934F03709350032A89E6
:1078D0003B8937FF03C0309521953F4F2134310557
:1078E000E4F1D401C30197FE07C0B095A09590952F
:1078F00081959F4FAF4FBF4F81389105A105B105CD
:1079000084F4DB01CA0177FF07C0B095A09590957C
:1079100081959F4FAF4FBF4F81389105A105B105AC
:10792000E4F081E08093EC0218C01092BC07109242
:10793000BB071092B8071092B70710924D03109230
:107940004E0310924F03109250031092490310926D
:107950004A0310924B0310924C0380914D03909177
:107960004E03A0914F03B0915003BC01CD0124E61A
:1079700030E040E050E00E947E7AE0904903F090D1
:107980004A03E21AF30AF092CF07E092CE07809101
:10799000490390914A03A0914B03B0914C03BC0161
:1079A000CD0124E630E040E050E00E947E7ADA012A
:1079B000C90120914D0330914E038C01021B130B22
:1079C0001093C3070093C207809143019091440133
:1079D000A0914501B0914601BC01CD0128E631E0FE
:1079E00040E050E00E940A7A20911808309119086E
:1079F00040911A0850911B08261737074807590766
:107A000064F0261B370B480B590B20931808309352
:107A1000190840931A0850931B08209118083091B8
:107A2000190840911A0850911B0857FF0CC0260FE7
:107A3000371F481F591F2093180830931908409387
:107A40001A0850931B086091C0077091C1076E0D12
:107A50007F1D9B01442737FD4095542F80910403DF
:107A600090910503A0910603B0910703820F931F25
:107A7000A41FB51F8093040390930503A0930603EE
:107A8000B09307038091C0029091C102681B790BEB
:107A9000CB01AA2797FDA095BA2F29853A854B855A
:107AA0005C85820F931FA41FB51F809308039093DA
:107AB0000903A0930A03B0930B03C0908301D090F5
:107AC0008401E0908501F0908601C816D906EA0687
:107AD000FB06C4F488EA91E6A0E0B0E08C199D09A9
:107AE000AE09BF098093080390930903A0930A038A
:107AF000B0930B038093040390930503A0930603B4
:107B0000B093070322273327A9012C193D094E09F9
:107B10005F098091080390910903A0910A03B09135
:107B20000B0382179307A407B507B4F4D701C60166
:107B3000885A9146A040B04080930803909309036F
:107B4000A0930A03B0930B0380930403909305035F
:107B5000A0930603B09307036091D0077091D107FB
:107B6000600F711F9B01442737FD4095542F809172
:107B70000C0390910D03A0910E03B0910F03820F9F
:107B8000931FA41FB51F80930C0390930D03A09324
:107B90000E03B0930F038091BE029091BF02681B49
:107BA000790BCB01AA2797FDA095BA2F2D853E858D
:107BB0004F855889820F931FA41FB51F8093100310
:107BC00090931103A0931203B0931303E0908701E5
:107BD000F09088010091890110918A01E816F90658
:107BE0000A071B07C4F488EA91E6A0E0B0E08E190A
:107BF0009F09A00BB10B8093100390931103A093E6
:107C00001203B093130380930C0390930D03A0937E
:107C10000E03B0930F0322273327A9012E193F0922
:107C2000400B510B8091100390911103A09112030E
:107C3000B091130382179307A407B507B4F4D801D2
:107C4000C701885A9146A040B0408093100390939A
:107C50001103A0931203B093130380930C0390932A
:107C60000D03A0930E03B0930F0380910003909136
:107C70000103A0910203B091030380931403909336
:107C80001503A0931603B0931703809110039091EE
:107C90001103A0911203B0911303809330039093CA
:107CA0003103A0933203B093330380910803909182
:107CB0000903A0910A03B0910B03809328039093CA
:107CC0002903A0932A03B0932B0380910C03909176
:107CD0000D03A0910E03B0910F0380932C0390939A
:107CE0002D03A0932E03B0932F0380910403909152
:107CF0000503A0910603B09107038093240390939A
:107D00002503A0932603B093270380911C01909133
:107D10001D0197FD079603E0959587950A95E1F774
:107D20009093D1078093D00780911A0190911B0105
:107D300097FD079613E0959587951A95E1F790932F
:107D4000C1078093C0078091FD019091FE010F97BC
:107D500034F488E19CEF9093D1078093D007809111
:107D6000FD019091FE01079734F480E398EF909322
:107D7000D1078093D007209102012A30A9F4809185
:107D8000FD019091FE01835F934034F088EE93E013
:107D90009093D1078093D0078091FD019091FE01CF
:107DA0008A5F9340DCF014C08091FD019091FE0148
:107DB000815D974034F088EE93E09093D1078093F3
:107DC000D0078091FD019091FE01805E974034F0D4
:107DD00080ED97E09093D1078093D0078091FB01CD
:107DE0009091FC010F9734F488E19CEF9093C107C8
:107DF0008093C0078091FB019091FC01079734F4B8
:107E000080E398EF9093C1078093C0072A30A9F4CC
:107E10008091FB019091FC01835F934034F088EEE8
:107E200093E09093C1078093C0078091FB019091EC
:107E3000FC018A5F9340DCF014C08091FB019091BB
:107E4000FC01815D974034F088EE93E09093C10788
:107E50008093C0078091FB019091FC01805E974068
:107E600034F080ED97E09093C1078093C007609154
:107E70007501662309F4AFC040911C0150911D01AA
:107E80008091590390915A03481B590B50936003FA
:107E900040935F0320911C0130911D01280F391F71
:107EA00037FF02C02F5F3F4F3595279530935A0318
:107EB00020935903413851051CF080E890E005C03B
:107EC00040585F4F34F480E89FEF909360038093B5
:107ED0005F0340911A0150911B0180915B039091C7
:107EE0005C03481B590B50935E0340935D03209144
:107EF0001A0130911B01280F391F37FF02C02F5F75
:107F00003F4F3595279530935C0320935B034138B1
:107F100051051CF080E890E005C040585F4F34F4F4
:107F200080E89FEF90935E0380935D03462F552773
:107F300080915F0390916003849FB001859F700DD5
:107F4000949F700D11249B0177FF02C0215F3F4F6A
:107F5000F4E035952795FA95E1F78091D007909157
:107F6000D107820F931F9093D1078093D007809100
:107F70005D0390915E03849FD001859FB00D949F17
:107F8000B00D1124AD019D01B7FF02C0215F3F4F2D
:107F9000E4E035952795EA95E1F78091C007909147
:107FA000C107820F931F9093C1078093C0078091F0
:107FB0001C0190911D01860F971F90931D018093C6
:107FC0001C0180911A0190911B01840F951F9093C1
:107FD0001B0180931A010091D3071091D40780915F
:107FE000B7079091B807101611065CF59C0197FF32
:107FF00004C022273327281B390BC901AA2797FD64
:10800000A095BA2F20916901332744275527BC0139
:10801000CD010E940A7A9B01AC0197FF04C0215C4C
:108020003F4F4F4F5F4F76E05595479537952795D2
:108030007A95D1F78091CE079091CF07820F931F49
:1080400027C097FF03C0909581959F4FAA2797FD62
:10805000A095BA2F20916901332744275527BC01E9
:10806000CD010E940A7A9B01AC0197FF04C0215CFC
:108070003F4F4F4F5F4F66E0559547953795279592
:108080006A95D1F78091CE079091CF07821B930B11
:108090009093CF078093CE07E090DB07F090DC074A
:1080A0008091BB079091BC071E141F045CF59C01D6
:1080B00097FF04C022273327281B390BC901AA27A1
:1080C00097FDA095BA2F20916901332744275527A2
:1080D000BC01CD010E940A7A9B01AC0197FF04C04C
:1080E000215C3F4F4F4F5F4F96E055954795379531
:1080F00027959A95D1F78091C2079091C307820F77
:10810000931F27C097FF03C0909581959F4FAA2783
:1081100097FDA095BA2F2091690133274427552751
:10812000BC01CD010E940A7A9B01AC0197FF04C0FB
:10813000215C3F4F4F4F5F4F86E0559547953795F0
:1081400027958A95D1F78091C2079091C307821B2A
:10815000930B9093C3078093C2078091080887FF11
:1081600044C0B989BB2309F040C08091BA0288237A
:10817000E1F5E1E0EE16E1E0FE064CF08091D0077B
:108180009091D1078E0D9F1D805091400DC0F0E061
:10819000EF16FFEFFF0664F48091D0079091D107AE
:1081A0008E0D9F1D80509F4F9093D1078093D007D5
:1081B00021E0013012074CF08091C0079091C10777
:1081C000800F911F805091400CC03FEF003013078B
:1081D00064F48091C0079091C107800F911F805077
:1081E0009F4F9093C1078093C007E2E1CD5E0C944E
:1081F000B57A8091D502882301F58091A0028C7F09
:108200008093A002AEEFB3E0EEEEF6E09BE080914B
:10821000B901882309F48C938D9181831282915046
:10822000389697FFF4CF8091B901882359F0809157
:10823000B90181508093B90105C08091A00281608D
:108240008093A00280912402882319F010922402C6
:1082500008958093260280932802809122028E7FC7
:108260008093220285EA8093BC000895CF93DF9328
:10827000A7EDB2E0C5E2D6E057E09991E92FFF27DC
:10828000EE0FFF1FE15BF84F0190F081E02DE15808
:10829000FF4FEF3FF10521F01CF0EFEFF0E004C0DD
:1082A000F7FF02C0E0E0F0E0993111F4EC931BC05D
:1082B0004C91242F3327E217F307A9F0CF01821B3B
:1082C000930B97FD03969595879595958795242F04
:1082D000280F2C93822F9927E817F90714F42150BF
:1082E00001C02F5F2C935150119657FFC6CF80913C
:1082F0002F06883F38F0EFEFF0E0E81BF109E95274
:10830000FD4F808180937B0180917B01882329F040
:10831000843618F084E680937B0180913106883F93
:1083200038F0EFEFF0E0E81BF109E952FD4F8081F2
:108330008093790180917901882329F0843618F09F
:1083400084E68093790180913E06883F38F0EFEF14
:10835000F0E0E81BF109E952FD4F80818093740140
:10836000809174018B3010F48AE002C08F3F11F4C9
:108370008093740180916B06883F38F0EFEFF0E056
:10838000E81BF109E952FD4F80818093E707809156
:10839000E707863010F485E002C08F3F11F4809328
:1083A000E70780916D06883F38F0EFEFF0E0E81BBB
:1083B000F109E952FD4F808180930F0880910F08E9
:1083C000863010F485E002C08F3F11F480930F08CF
:1083D00080915806883F38F0EFEFF0E0E81BF10994
:1083E000E952FD4F80818093E40780915906883FD0
:1083F00038F0EFEFF0E0E81BF109E952FD4F808122
:108400008093BD0780915A06883F38F0EFEFF0E087
:10841000E81BF109E952FD4F80818093ED078091BF
:108420003006883F38F0EFEFF0E0E81BF109E95241
:10843000FD4F808180937A0180913306883F38F028
:10844000EFEFF0E0E81BF109E952FD4F80818093E6
:10845000780180913506883F38F0EFEFF0E0E81BB7
:10846000F109E952FD4F80818093760180913D06AC
:10847000883F38F0EFEFF0E0E81BF109E952FD4FDB
:1084800080818093770180913F06883F38F0EFEF3D
:10849000F0E0E81BF109E952FD4F80818093730100
:1084A00080914006883F38F0EFEFF0E0E81BF109DB
:1084B000E952FD4F80818093750180914106883F8C
:1084C00038F0EFEFF0E0E81BF109E952FD4F808151
:1084D0008093720180914206883F38F0EFEFF0E020
:1084E000E81BF109E952FD4F808180937101809171
:1084F0004806883F38F0EFEFF0E0E81BF109E95259
:10850000FD4F808180936F0180914906883F38F04C
:10851000EFEFF0E0E81BF109E952FD4F8081809315
:10852000B50280914A06883F38F0EFEFF0E0E81B93
:10853000F109E952FD4F80818093B40280914B068E
:10854000883F38F0EFEFF0E0E81BF109E952FD4F0A
:1085500080818093B30280914C06883F38F0EFEF22
:10856000F0E0E81BF109E952FD4F80818093B202EF
:1085700080916606883F38F0EFEFF0E0E81BF109E4
:10858000E952FD4F80818093B10280916706883F58
:1085900038F0EFEFF0E0E81BF109E952FD4F808180
:1085A0008093B00280916806883F38F0EFEFF0E0EA
:1085B000E81BF109E952FD4F80818093AF02809161
:1085C0006906883F38F0EFEFF0E0E81BF109E95267
:1085D000FD4F80818093AE0280914D06883F38F038
:1085E000EFEFF0E0E81BF109E952FD4F8081809345
:1085F0006E0180915106883F38F0EFEFF0E0E81B04
:10860000F109E952FD4F808180936D0180915B06F5
:10861000883F38F0EFEFF0E0E81BF109E952FD4F39
:10862000808180936C0180915E06883F38F0EFEF87
:10863000F0E0E81BF109E952FD4F808180936B0166
:1086400080915F06883F38F0EFEFF0E0E81BF1091A
:10865000E952FD4F808180936A0180916006883FD6
:1086600038F0EFEFF0E0E81BF109E952FD4F8081AF
:108670008093690180918706883F38F0EFEFF0E042
:10868000E81BF109E952FD4F80818093CC0780916E
:108690002D068093080880918A068093EC078091CC
:1086A0006506883F38F0EFEFF0E0E81BF109E9528A
:1086B000FD4F80818093680180918006883F38F06B
:1086C000EFEFF0E0E81BF109E952FD4F8081809364
:1086D0001F0880916F01282F33272F5F3F4F8CE3B6
:1086E00098E2B9010E94497A70937D0160937C0100
:1086F00080913B068093100880913A068093D507BD
:10870000909182069333C8F181E08093AD02983F47
:1087100058F0EFEFF0E0E91BF109E952FD4F8081DD
:10872000823310F41092AD0280917E012091AD024F
:10873000821799F0833070F4222319F08CED95E0C4
:1087400002C088EC90E09093DB018093DA012093E3
:108750007E0103C0815080937E0180915F089091DB
:10876000600897FF0FC08091AD02882359F0809177
:10877000F90380688093F90305C01092AD028AE086
:1087800080937E0180915F089091600897FF1DC0E3
:108790008091D5028823C9F08091AD028823A9F089
:1087A00080910801909109018F5F9F4F71F488E9D2
:1087B0009AE39093DB018093DA0180E094EA90934E
:1087C0000901809308011092AD028091AD028823C7
:1087D00069F080919F02816080939F0280916B017C
:1087E000823D48F4825E80936B0105C080919F02B8
:1087F0008E7F80939F02DF91CF910895A7E1B0E033
:10880000E4E0F4E40C94997A0E944739E090E002A5
:10881000F090E102FA82E9828091D50799270A96C1
:10882000E816F90614F49A8389838091D602843677
:1088300008F066C080919F0282FD62C0809175033E
:1088400090917603009731F001979093760380938F
:1088500075030BC01092D5029093A2028093A102DF
:108860008091A0028D7E8093A002809102018A30C7
:1088700011F0843110F0289A01C028988091A1024B
:108880009091A202895E9340C0F180914506282F05
:1088900033273A8329838091A00280618093A002CC
:1088A00080912106A82FBB27AA0FBB1FFD01ED5702
:1088B000F84F1182108280912206282F3327220F31
:1088C000331FC9018D57984FFC0111821082A15BA3
:1088D000B84F11961C921E92215B384FD901119608
:1088E0001C921E9280912406E82FFF27EE0FFF1F97
:1088F000E15BF84F11821082A9C21092D502A6C284
:108900008091D6028D3808F4A1C28091A0028F7E9A
:108910008093A0029091460682E3989FC0011124A3
:108920009093760380937503E981FA81B9978CF06F
:108930008091D502882369F08091A1029091A202D2
:10894000FFEF8F3F9F0729F001969093A20280933B
:10895000A1028091A1029091A2028F3F910509F09E
:1089600008F51092F8021092F9021092FA02109291
:10897000FB021092F4021092F5021092F60210928D
:10898000F702109261031092620310926303109237
:1089900064031092000310920103109202031092DC
:1089A000030305C08091A00282608093A0028091A1
:1089B0002306E82FFF27EE0FFF1FE15BF84F8081B2
:1089C0009181813591050CF435C12091D502222386
:1089D00009F030C180912406E82FFF27EE0FFF1F1A
:1089E000E15BF84F808191818C3491050CF4FFC0DC
:1089F000809177038F5F80937703893C08F41AC1D5
:108A0000209377031092A2021092A10230912106C6
:108A1000E32FFF27EE0FFF1FE15BF84F808191816D
:108A200087349105B4F480912206E82FFF27EE0FDA
:108A3000FF1FE15BF84F808191810190F081E02D73
:108A4000F7FF03C0F095E195FF4FE734F1050CF413
:108A500078C041E020912206A22FBB27AA0FBB1F9E
:108A6000A15BB84F8D919C9111978734910544F08B
:108A7000E32FFF27EE0FFF1FE15BF84F808191810D
:108A80008D919C918734910574F080912106E82F97
:108A9000FF27EE0FFF1FE15BF84F80819181873444
:108AA00091050CF042E0E22FFF27EE0FFF1FE15B84
:108AB000F84F808191818634910574F4809121066C
:108AC000E82FFF27EE0FFF1FE15BF84F80819181B8
:108AD000873491050CF043E0E22FFF27EE0FFF1FD4
:108AE000E15BF84F808191818A5B9F4F74F48091A4
:108AF0002106E82FFF27EE0FFF1FE15BF84F808173
:108B00009181873491050CF044E0E22FFF27EE0FAE
:108B1000FF1FE15BF84F808191818A5B9F4F74F466
:108B200080912106E82FFF27EE0FFF1FE15BF84F32
:108B300080819181863491050CF445E0842F0E9458
:108B4000382B80912206E82FFF27EE0FFF1FE15BF5
:108B5000F84F808191810190F081E02DF7FF03C0F3
:108B6000F095E195FF4F7E97BCF480912106E82FA8
:108B7000FF27EE0FFF1FE15BF84F808191818A5B39
:108B80009F4F54F481E08093140488EE93E0909317
:108B9000DB018093DA014EC00E94342C0E94E52A4A
:108BA00080E00E94C206809147060E940C76809168
:108BB000080880FF10C08091140190911501875B17
:108BC000934038F480911401909115018E5E92408B
:108BD00010F40E94431A1092D80180E00E9495364A
:108BE00081E080937A038093D801579A1AC08081DC
:108BF0009181855B9F4FE4F4809177038F5F809331
:108C00007703893CB8F02093D50220937703109224
:108C1000A2021092A10281E00E94953681E0809329
:108C20007A030E94342C68E770E00E94C63502C0C7
:108C30002093770380912306E82FFF27EE0FFF1F75
:108C4000E15BF84F808191818B5A9F4F0CF0FEC001
:108C50003091D502E0912406332309F0CCC0FF27E0
:108C6000EE0FFF1FE15BF84F80819181855B9F4F85
:108C70000CF0BEC020918306E22FFF27EE0FFF1FEE
:108C8000E15BF84F80819181855B9F4F1CF022232F
:108C900009F0AEC0809178038F5F80937803893CA0
:108CA00008F4D4C0309378038091F903882309F045
:108CB00098C080917A03882309F493C08091AD0312
:108CC000882309F08EC081E090E09093A202809307
:108CD000A10281E08093D502109261031092620399
:108CE0001092630310926403109200031092010328
:108CF00010920203109203031092FC021092FD02E4
:108D00001092FE021092FF0280913C06E82EFF2492
:108D10000027112780910C0890910D089C01442791
:108D200037FD4095542FC801B7010E940A7ADC0133
:108D3000CB018093100390931103A0931203B0937F
:108D4000130380911C0890911D089C01442737FD56
:108D50004095542FC801B7010E940A7ADC01CB016B
:108D60008093080390930903A0930A03B0930B0325
:108D70008091300390913103A0913203B09133037D
:108D800080930C0390930D03A0930E03B0930F03F5
:108D90008091280390912903A0912A03B0912B037D
:108DA0008093040390930503A0930603B0930703F5
:108DB0001092F8021092F9021092FA021092FB023D
:108DC0001092F4021092F5021092F6021092F7023D
:108DD0008091A00288608093A00284E680937B0348
:108DE00035C08CED95E09093DB018093DA012EC0C5
:108DF000109278032BC0FF27EE0FFF1FE15BF84FA7
:108E0000808191818C349105FCF020918306E22FC2
:108E1000FF27EE0FFF1FE15BF84F80819181855B9B
:108E20009F4F14F0222381F4809179038F5F809308
:108E30007903893C58F01092D50210927903109270
:108E4000A2021092A10202C0109279038091410106
:108E5000815080934101809141018F3F21F08091A9
:108E6000A00284FFA9C30E943641B09037068091CA
:108E70008403909185039C01220F331F280F391F13
:108E8000C0902106AC2DBB27AA0FBB1FFD01E15BE3
:108E9000F84F4B2D552780819181849FF001859F4C
:108EA000F00D949FF00D11242E0F3F1F37FF02C0CD
:108EB0002D5F3F4FB9017595679575956795AD57CE
:108EC000B84F80913806082F11278D919C91809F73
:108ED0007001819FF00C909FF00C11246E0D7F1D8E
:108EE0007093850360938403809186039091870338
:108EF0009C01220F331F280F391FD0902206AD2D61
:108F0000BB27AA0FBB1FFD01E15BF84F8081918158
:108F1000849FF001859FF00D949FF00D11242E0F7A
:108F20003F1F37FF02C02D5F3F4FA9015595479561
:108F300055954795AD57B84F8D919C91809F700185
:108F4000819FF00C909FF00C11244E0D5F1D5093EB
:108F50008703409386038091AD02882309F448C0BB
:108F6000CB0177FD0396DC01B595A795B595A7953F
:108F7000CA0157FD0396FC01F595E795F595E79530
:108F800080919D01682F772767FD70956A9F9001FA
:108F90006B9F300D7A9F300D11248091AF03482FC5
:108FA000552747FD50954E9FC0014F9F900D5E9FE6
:108FB000900D1124280F391F37FF02C0295F3F4F42
:108FC00093E0359527959A95E1F73093E702209342
:108FD000E6026E9F90016F9F300D7E9F300D112431
:108FE0004A9FC0014B9F900D5A9F900D11243FC086
:108FF00080918106E82FFF27E75BFE4F86818093F3
:109000009D0190819093AF03A82FBB27A7FDB0953A
:10901000A69F9001A79F300DB69F300D1124E92F18
:10902000FF27E7FDF095E49FC001E59F900DF49FB9
:10903000900D1124280F391F37FF02C0295F3F4FC1
:1090400083E0359527958A95E1F73093E7022093E1
:10905000E602A49F9001A59F300DB49F300D11240E
:10906000E69FC001E79F900DF69F900D1124281BED
:10907000390B37FF02C0295F3F4F03E03595279535
:109080000A95E1F73093E5022093E40280912406EB
:10909000E82FFF27EE0FFF1FE15BF84F80819181E2
:1090A000909581959F4F9093E3028093E2028530E3
:1090B000910514F0049705C00FEF8C3F900734F42E
:1090C00004969093E3028093E20204C01092E302BC
:1090D0001092E2028091A003882309F43EC0282F59
:1090E00033278091E6029091E70297FD079613E0FF
:1090F000959587951A95E1F7289FA001299F500D16
:10910000389F500D1124CA0157FD0F96B4E0959574
:109110008795BA95E1F79093E7028093E6028091F4
:10912000E4029091E50297FD0796A3E09595879557
:10913000AA95E1F7289FB001299F700D389F700D07
:109140001124CB0177FD0F96F4E095958795FA955C
:10915000E1F79093E5028093E4028090E60290901C
:10916000E7028091A3039091A403881A990A909230
:10917000E7028092E6020091E4021091E5028091FC
:10918000A1039091A203081B190B1093E502009311
:10919000E40280912306E82FFF27EE0FFF1FE15B1B
:1091A000F84FE080F1808FE790E0E80EF91EF09232
:1091B000E102E092E002809174019927AA2797FDCD
:1091C000A095BA2FBC01CD010E947E79DC01CB01B4
:1091D00020E030E040E251E4BC01CD010E94EC7897
:1091E000DC01CB01BC01CD010E945079DC01CB0137
:1091F00080931608809173018093EE07809172012D
:109200009927AA2797FDA095BA2FBC01CD010E94EE
:109210007E79DC01CB0120E030E040E251E4BC018A
:10922000CD010E94EC78DC01CB01BC01CD010E9494
:109230005079DC01CB018093C70780917101809345
:10924000DD078091200480FF59C080911F0881387C
:1092500008F454C080911904992787FD90952B2D0F
:109260003327829FD001839FB00D929FB00D1124B0
:109270008A0E9B1E9092E7028092E60280911A0469
:10928000992787FD9095829FF001839FF00D929F13
:10929000F00D11240E0F1F1F1093E5020093E4023E
:1092A00080911B04282F332727FD30958091E202FF
:1092B0009091E302820F931F9093E3028093E20266
:1092C00080911D04282F332727FD30958091320689
:1092D0009927289F8001299F100D389F100D112478
:1092E000109348010093470180911C0499278E1523
:1092F0009F0524F49093E1028093E0028091E002C4
:109300009091E10297FF04C01092E1021092E002F6
:109310008091080882FF02C01092EE074091E60299
:109320005091E702CA0157FD03969C013595279598
:109330003595279537FF03C0309521953F4F809194
:10934000A5029091A60282179307B4F4CA0157FFB1
:1093500003C0909581959F4F97FD039695958795AE
:10936000959587959093A6028093A50285369105E1
:1093700044F084E690E001C001979093A6028093A8
:10938000A5024091E4025091E502CA0157FD0396FF
:109390009C01359527953595279537FF03C0309566
:1093A00021953F4F8091A3029091A40282179307C9
:1093B000B4F4CA0157FF03C0909581959F4F97FD64
:1093C000039695958795959587959093A40280939C
:1093D000A3028536910544F084E690E001C0019730
:1093E0009093A4028093A3028091A00284FF08C0FE
:1093F0001092A6021092A5021092A4021092A3024B
:10940000ED2DFF27EE0FFF1FE15BF84F40915C064B
:10941000242F3327808191812817390744F48091C4
:10942000880682FF04C081E08093B90213C0ED2D4D
:10943000FF27EE0FFF1FE15BF84F842F9927209144
:109440005D06821B9109208131812817390714F4A8
:109450001092B90240912206E42FFF27EE0FFF1F62
:10946000E15BF84F50915C06852F9927222733271F
:10947000281B390B808191818217930744F48091D6
:10948000880683FF04C081E08093B80216C08091F3
:10949000B802882391F0E42FFF27EE0FFF1FE15B56
:1094A000F84F80915D069927851B910920813181B4
:1094B0008217930714F41092B802EC2DFF27EE0FD9
:1094C000FF1FE15BF84F40915C06242F332780811A
:1094D00091812817390744F48091880680FF04C0E1
:1094E00081E08093B60217C08091B602882399F07C
:1094F000EC2DFF27EE0FFF1FE15BF84F842F99271C
:1095000020915D06821B910920813181281739073E
:1095100014F41092B60240912106E42FFF27EE0FBB
:10952000FF1FE15BF84F50915C06852F992722279A
:109530003327281B390B808191818217930744F4CC
:109540008091880681FF04C081E08093B70216C035
:109550008091B702882391F0E42FFF27EE0FFF1FC1
:10956000E15BF84F80915D069927851B9109208169
:1095700031818217930714F41092B7028091B902D7
:10958000882319F48091B802811181E08093BA0296
:109590008091B602882321F48091B702882351F08C
:1095A00081E08093BB021092BA021092B90210922D
:1095B000B80202C08093BB028091BA02882321F4D2
:1095C0008091BB02882369F080915B0699272981ED
:1095D0003A818217930714F49A83898381E08093F8
:1095E000EC0280919F0299279C012470307082FFC9
:1095F0002DC08091A3039091A403909581959F4FD6
:109600009093E7028093E6028091A1039091A203D8
:10961000909581959F4F9093E5028093E40280910D
:109620008101909182019093E1028093E002809108
:1096300008088B778B66809308088091EC078C7BF9
:109640008093EC0788EC80937A011EC08091A00281
:1096500084FF1AC03093E3022093E2023093E702C2
:109660002093E6023093E5022093E4029AE590937A
:10967000160888E78093EE079093C7078093DD076D
:109680001092BA021092BB028091E0079091E1071C
:10969000A091E207B091E3072091300330913103AC
:1096A0004091320350913303820F931FA41FB51FC3
:1096B0008093E0079093E107A093E207B093E3075C
:1096C0008091E8079091E907A091EA07B091EB0734
:1096D000E0902803F090290300912A0310912B03B6
:1096E000EB82FC820D831E838E0D9F1DA01FB11F78
:1096F0008093E8079093E907A093EA07B093EB07FC
:109700008091D7079091D807A091D907B091DA0737
:10971000E0902C03F0902D0300912E0310912F0365
:10972000EF82F88609871A878E0D9F1DA01FB11F33
:109730008093D7079093D807A093D907B093DA07FF
:109740008091C8079091C907A091CA07B091CB0733
:10975000E0902403F0902503009126031091270345
:10976000EB86FC860D871E878E0D9F1DA01FB11FE7
:109770008093C8079093C907A093CA07B093CB07FB
:10978000F090BB02FF86FF2029F48091BA02882363
:1097900009F460C01092200310922103109222035A
:1097A0001092230310921C0310921D0310921E03AB
:1097B00010921F031092E0071092E1071092E20747
:1097C0001092E3071092E8071092E9071092EA0757
:1097D0001092EB071092D7071092D8071092D90772
:1097E0001092DA071092C8071092C9071092CA07A0
:1097F0001092CB078091100390911103A091120356
:10980000B091130380930C0390930D03A0930E0368
:10981000B0930F038091080390910903A0910A036C
:10982000B0910B038093040390930503A093060368
:10983000B09307031092EA011092E9011092BF025F
:109840001092BE021092C1021092C0020F85002336
:1098500009F0F8C18091BA02882309F0F3C1809120
:10986000C2059091C305815092402CF48091D5029D
:10987000882309F4E7C190909808A0903C062090B6
:109880000C0830900D0840901C0850901D081914C9
:109890000CF0E3C0BB24CC24DD24CA01B901A6012D
:1098A00095010E947E7A79018A01809161089091E8
:1098B0006208281A390AC101AA2797FDA095BA2F74
:1098C000E81AF90A0A0B1B0B6B817C818D819E8142
:1098D000A60195010E947E7A59016A018091630870
:1098E00090916408481A590AC201AA2797FDA095C9
:1098F000BA2FA81AB90ACA0ADB0A292C332427FC72
:109900003094432C532CC801B701A20191010E944D
:109910000A7A97FF04C061507E4F8F4F9F4F3B01E3
:109920004C0109E095948794779467940A95D1F750
:10993000C601B501A20191010E940A7A97FF04C0F5
:1099400061507E4F8F4F9F4F5B016C0119E0D594A2
:10995000C794B794A7941A95D1F78091A5029091D6
:10996000A602813491053CF48091A3029091A40257
:1099700081349105D4F0D401C30197FE03C0019650
:10998000A11DB11D3C014D01959487947794679476
:10999000D601C501D7FE03C00196A11DB11D5C0112
:1099A0006D01D594C794B794A79480912406E82FAD
:1099B000FF27EE0FFF1FE15BF84F8081918101903F
:1099C000F081E02DF7FF03C0F095E195FF4F7A9706
:1099D000A4F0C401B30123E030E040E050E00E9475
:1099E0007E7A39014A01C601B50123E030E040E04A
:1099F00050E00E947E7A59016A0180919A08282FCE
:109A0000332727FD3095432F532F2615370548055B
:109A1000590514F439014A01992787FD90959095CD
:109A200081959F4FAA2797FDA095BA2F68167906B2
:109A30008A069B0614F43C014D012A153B054C0592
:109A40005D0514F459016A01A816B906CA06DB06B9
:109A50000CF0D0C05C016D01CDC0EA2CFF240027C2
:109A60001127CA01B901A80197010E947E7A390124
:109A70004A01C101AA2797FDA095BA2F681A790A51
:109A80008A0A9B0A6B817C818D819E81A801970146
:109A90000E947E7A59016A01C201AA2797FDA0950A
:109AA000BA2FA81AB90ACA0ADB0AD401C30197FE61
:109AB00003C00F96A11DB11D3C014D01F4E095942A
:109AC000879477946794FA95D1F7D601C501D7FEAC
:109AD00003C00F96A11DB11D5C016D01E4E0D5949A
:109AE000C794B794A794EA95D1F78091A502909175
:109AF000A602813491053CF48091A3029091A402C6
:109B000081349105A4F0C401B30123E030E040E0CA
:109B100050E00E947E7A39014A01C601B50123E076
:109B200030E040E050E00E947E7A59016A01809165
:109B30002406E82FFF27EE0FFF1FE15BF84F80811F
:109B400091810190F081E02DF7FF03C0F095E19540
:109B5000FF4F7A97A4F0C401B30123E030E040E066
:109B600050E00E947E7A39014A01C601B50123E026
:109B700030E040E050E00E947E7A59016A0189E1BC
:109B800080938D0121E262167104810491042CF00E
:109B900070E2672E712C812C912C30EE63163FEF12
:109BA00073063FEF83063FEF930644F460EE662EA4
:109BB0006FEF762E6FEF862E6FEF962E41E2A41692
:109BC000B104C104D1042CF050E2A52EB12CC12C5B
:109BD000D12C50EEA5165FEFB5065FEFC5065FEF1F
:109BE000D50644F440EEA42E4FEFB42E4FEFC42E12
:109BF0004FEFD42E8091100390911103A091120386
:109C0000B091130386199709A809B9098093100325
:109C100090931103A0931203B09313038091080350
:109C200090910903A0910A03B0910B038A199B0933
:109C3000AC09BD098093080390930903A0930A031C
:109C4000B0930B038091E9019091EA018F3F910558
:109C500009F008F4C4C56F85662309F04EC58091EC
:109C6000BA02882309F049C58091EC02882309F0E3
:109C700044C570916406788B772309F43EC58091C2
:109C8000E0079091E107A091E207B091E307B7FFE9
:109C900004C081509F4FAF4FBF4FE92EFA2E0B2FBC
:109CA000112707FD1A95E092E007F092E107009373
:109CB000E2071093E3078091E8079091E907A091EC
:109CC000EA07B091EB07B7FF04C081509F4FAF4F39
:109CD000BF4F892F9A2FAB2FBB27A7FDBA95898B32
:109CE0009A8BAB8BBC8B8093E8079093E907A0938A
:109CF000EA07B093EB0780913C06A82EBB24CC2446
:109D0000DD242091200330912103409122035091C2
:109D10002303C601B5010E940A7A97FF04C061506F
:109D20007F4F8F4F9F4F672E782E892E992487FC67
:109D30009A94609220037092210380922203909261
:109D4000230320911C0330911D0340911E03509169
:109D50001F03C601B5010E940A7A97FF04C0615033
:109D60007F4F8F4F9F4F272E382E492E552447FC6B
:109D70005A9420921C0330921D0340921E0350926D
:109D80001F038091180390911903A0911A03B091B9
:109D90001B03B7FF04C081509F4FAF4FBF4F892FA8
:109DA0009A2FAB2FBB27A7FDBA95809318039093EA
:109DB0001903A0931A03B0931B03D801C701861996
:109DC0009709A809B90980936D0390936E03A09336
:109DD0006F03B093700320916306E22EFF240027E7
:109DE0001127BC01CD01A80197010E947E7A59017B
:109DF0006A0120937C0330937D0340937E0350934C
:109E00007F0389899A89AB89BC8982199309A4093E
:109E1000B5098093710390937203A0937303B09379
:109E20007403BC01CD01A80197010E947E7A2093A2
:109E30008003309381034093820350938303D601C0
:109E4000C501D7FE04C081509F4FAF4FBF4F892F30
:109E50009A2FAB2FBB27A7FDBA959093BF02809393
:109E6000BE0257FF04C021503F4F4F4F5F4FBB27EB
:109E700057FDBA95A52F942F832F9093C1028093FD
:109E8000C0028091A5029091A60281349105DCF474
:109E90008091A3029091A40281349105A4F4809151
:109EA0002406E82FFF27EE0FFF1FE15BF84F8081AC
:109EB00091810190F081E02DF7FF03C0F095E195CD
:109EC000FF4F7A97E4F0809198088F3FC1F480911A
:109ED000BE029091BF0297FD01969595879590934C
:109EE000BF028093BE028091C0029091C10297FD93
:109EF0000196959587959093C1028093C0028091B9
:109F0000D7079091D807A091D907B091DA07B7FF8A
:109F100004C081509F4FAF4FBF4F892F9A2FAB2F57
:109F2000BB27A7FDBA958093D7079093D807A09336
:109F3000D907B093DA078091C8079091C907A0911B
:109F4000CA07B091CB07B7FF04C081509F4FAF4FF6
:109F5000BF4F892F9A2FAB2FBB27A7FDBA958093B0
:109F6000C8079093C907A093CA07B093CB07809105
:109F7000300390913103A0913203B09133032F81CC
:109F8000388549855A85281B390B4A0B5B0B209372
:109F90006503309366034093670350936803809191
:109FA000280390912903A0912A03B0912B03EB84FD
:109FB000FC840D851E85E81AF90A0A0B1B0BE0923A
:109FC0006903F0926A0300936B0310936C03209370
:109FD0006D0330936E0340936F0350937003E092D0
:109FE0007103F092720300937303109374038091D2
:109FF0000C0390910D03A0910E03B0910F03821BEF
:10A00000930BA40BB50B80930C0390930D03A093BB
:10A010000E03B0930F038091040390910503A09168
:10A020000603B09107038E199F09A00BB10B809313
:10A03000040390930503A0930603B0930703888954
:10A040008823E1F02091EA023091EB0221383105BA
:10A050004CF080914103909142030196909342030A
:10A060008093410320583F4F4CF4809141039091DD
:10A070004203019790934203809341031092EB02B5
:10A080001092EA0281E090E0909389038093880324
:10A09000E0906D03F0906E0300916F0310917003D8
:10A0A000D801C70117FF07C088279927DC018E193F
:10A0B0009F09A00BB10B81509240A040B04034F0FA
:10A0C00084E090E0909389038093880380918E03CD
:10A0D00090918F03A0919003B09191032091E0079C
:10A0E0003091E1074091E2075091E307821B930B07
:10A0F000A40BB50B815E914BAF4FBF4F8F539C4963
:10A10000A040B04028F08091990889310CF4FFC03C
:10A1100021E0E21620E1F20620E0020720E012072B
:10A120000CF473C080918A03882309F46AC0D801B3
:10A13000C70117FF07C088279927DC018E199F09DF
:10A14000A00BB10B9C01AD01B7FF04C021503E4FE5
:10A150004F4F5F4FF9E05595479537952795FA95FD
:10A16000D1F78091880390918903820F931F909378
:10A17000890380938803D801C70117FF03C007969E
:10A18000A11DB11DE3E0B595A79597958795EA9533
:10A19000D1F780937C0390937D03A0937E03B093CB
:10A1A0007F0389589341A040B04064F088E893E170
:10A1B000A0E0B0E080937C0390937D03A0937E03A6
:10A1C000B0937F0320917C0330917D0340917E0307
:10A1D00050917F0357FF04C021503F4F4F4F5F4FB7
:10A1E000232F342F452F552747FD5A958091BE02C6
:10A1F0009091BF02820F931F9093BF028093BE0283
:10A2000006C081E080938A0302C010928A0340E076
:10A21000E41640EFF4064FEF04074FEF14070CF07D
:10A2200073C080918B03882309F46AC0D801C701E9
:10A2300017FF07C088279927DC018E199F09A00BFB
:10A24000B10B9C01AD01B7FF04C021503E4F4F4FF1
:10A250005F4F69E055954795379527956A95D1F7F2
:10A260008091880390918903820F931F90938903B3
:10A2700080938803D801C70117FF03C00796A11D6B
:10A28000B11D23E0B595A795979587952A95D1F7A8
:10A2900080937C0390937D03A0937E03B0937F0310
:10A2A00088579C4EAF4FBF4F64F488E79CEEAFEFEA
:10A2B000BFEF80937C0390937D03A0937E03B093C4
:10A2C0007F0320917C0330917D0340917E03509168
:10A2D0007F0357FF04C021503F4F4F4F5F4F232F45
:10A2E000342F452F552747FD5A958091BE029091F6
:10A2F000BF02820F931F9093BF028093BE0211C0D2
:10A3000081E080938B030DC010928B030AC01092E2
:10A3100089031092880384E690E090938C018093E7
:10A320008B016889262F33278091880390918903B8
:10A330002817390724F43093890320938803109158
:10A340009908112379F0212F332727FD309580912B
:10A350008803909189032817390724F430938903DF
:10A360002093880340916D0350916E0360916F03B9
:10A3700070917003413851056105710574F0809149
:10A380004503909146032091880330918903820F01
:10A39000931F909346038093450340585F4F6F4F40
:10A3A0007F4F74F480914503909146032091880378
:10A3B00030918903821B930B90934603809345034E
:10A3C00081E090E09093890380938803C0907103AB
:10A3D000D0907203E0907303F0907403D701C6012C
:10A3E000F7FE07C088279927DC018C199D09AE0963
:10A3F000BF0981509240A040B04034F084E090E02A
:10A4000090938903809388038091920390919303A2
:10A41000A0919403B09195032091E8073091E9074A
:10A420004091EA075091EB07821B930BA40BB50BED
:10A43000815E914BAF4FBF4F8F539C49A040B040BE
:10A4400018F019310CF4FFC001E0C01600E1D0068D
:10A4500000E0E00600E0F0060CF473C080918C038D
:10A46000882309F46AC0D701C601F7FE07C0882710
:10A470009927DC018C199D09AE09BF099C01AD012A
:10A48000B7FF04C021503E4F4F4F5F4F09E0559535
:10A490004795379527950A95D1F780918803909134
:10A4A0008903820F931F9093890380938803D701B8
:10A4B000C601F7FE03C00796A11DB11D13E0B595B7
:10A4C000A795979587951A95D1F7809380039093D8
:10A4D0008103A0938203B093830389589341A040E2
:10A4E000B04064F088E893E1A0E0B0E0809380039E
:10A4F00090938103A0938203B09383032091800300
:10A5000030918103409182035091830357FF04C02F
:10A5100021503F4F4F4F5F4F232F342F452F55274B
:10A5200047FD5A958091C0029091C102820F931FFE
:10A530009093C1028093C00206C081E080938C0397
:10A5400002C010928C0320E0C21620EFD2062FEF3B
:10A55000E2062FEFF2060CF073C080918D03882382
:10A5600009F46AC0D701C601F7FE07C088279927FA
:10A57000DC018C199D09AE09BF099C01AD01B7FF33
:10A5800004C021503E4F4F4F5F4FE9E0559547952E
:10A5900037952795EA95D1F78091880390918903A3
:10A5A000820F931F9093890380938803D701C6017C
:10A5B000F7FE03C00796A11DB11D73E0B595A795E1
:10A5C000979587957A95D1F780938003909381032F
:10A5D000A0938203B093830388579C4EAF4FBF4F25
:10A5E00064F488E79CEEAFEFBFEF80938003909315
:10A5F0008103A0938203B093830320918003309161
:10A600008103409182035091830357FF04C021507E
:10A610003F4F4F4F5F4F232F342F452F552747FD77
:10A620005A958091C0029091C102820F931F90931E
:10A63000C1028093C00211C081E080938D030DC0E0
:10A6400010928D030AC0109289031092880384E649
:10A6500090E090938C0180938B014889242F3327BD
:10A6600080918803909189032817390724F4309347
:10A6700089032093880380919908882379F0282FF3
:10A68000332727FD309580918803909189032817FF
:10A69000390724F430938903209388034091710390
:10A6A00050917203609173037091740341385105A6
:10A6B0006105710574F080914303909144032091EA
:10A6C000880330918903820F931F909344038093F2
:10A6D000430340585F4F6F4F7F4FCCF4809143034B
:10A6E000909144032091880330918903821B930B3E
:10A6F00090934403809343030AC01092C1021092C6
:10A70000C0021092BF021092BE021092EC02809121
:10A71000EE07882341F41092C1021092C0021092F9
:10A72000BF021092BE028091E0079091E107A091D4
:10A73000E207B091E30780938E0390938F03A09379
:10A740009003B09391038091E8079091E907A0915D
:10A75000EA07B091EB078093920390939303A09341
:10A760009403B0939503109220031092210310924A
:10A7700022031092230310921C0310921D031092C7
:10A780001E0310921F0310921803109219031092C7
:10A790001A0310921B031092E0071092E107109227
:10A7A000E2071092E3071092E8071092E90710926F
:10A7B000EA071092EB071092D7071092D807109271
:10A7C000D9071092DA071092C8071092C9071092A1
:10A7D000CA071092CB071092EA011092E901E090AB
:10A7E000E202F090E302C701F7FE04C08827992730
:10A7F0008E199F0904973CF08091080884FD03C0DE
:10A8000082E380937B0310913906A12EBB24CC24D4
:10A81000DD24B701882777FD8095982F9701F7FEF3
:10A8200004C0222733272E193F09442737FD4095BE
:10A83000542F0E940A7A9B01AC01C601B5010E9407
:10A840000A7A97FF04C061507E4F8F4F9F4F59E0A7
:10A8500095958795779567955A95D1F79B01812FA7
:10A8600099278E9DD0018F9DB00D9E9DB00D112416
:10A87000CD01B7FD03969595879595958795280FFA
:10A88000391F8091C2029091C302280F391F4427BB
:10A8900037FD4095542F209361033093620340931A
:10A8A0006303509364038091000390910103A0918E
:10A8B0000203B0910303821B930BA40BB50B80938F
:10A8C000000390930103A0930203B0930303815507
:10A8D000934CA040B04064F080E593ECA0E0B0E081
:10A8E0008093000390930103A0930203B0930303AA
:10A8F0008091000390910103A0910203B0910303A2
:10A90000805B9C43AF4FBF4F64F480EB9CE3AFEFA1
:10A91000BFEF8093000390930103A0930203B093D1
:10A92000030300918F011091900117FDFAC08091EF
:10A93000080883FFF6C080918E01815080938E01BC
:10A94000882309F0F2C08DE080938E01809130035E
:10A9500090913103A0913203B0913303B7FF04C04B
:10A9600081509E4FAF4FBF4F39E0B595A795979552
:10A9700087953A95D1F77C0197FF04C0F094E19454
:10A98000F108F3948091280390912903A0912A0360
:10A99000B0912B03B7FF04C081509E4FAF4FBF4F04
:10A9A00029E0B595A795979587952A95D1F79C01AC
:10A9B00097FF03C0309521953F4FE216F3060CF444
:10A9C0007901B701F7FE02C06D5F7F4F2B015594EF
:10A9D0004794559447940894411C511C6090180862
:10A9E0007090190880901A0890901B0820914301DC
:10A9F000309144014091450150914601C401B30199
:10AA00000E947E7A59016A013093C6072093C507D8
:10AA1000021B130BC801845E9D4F68E671E00E9423
:10AA2000497A9C01245B304080918B0190918C018C
:10AA3000009731F0019790938C0180938B011BC09C
:10AA400009E1E016F104BCF48091EA029091EB0276
:10AA5000820F931F9093EB028093EA0280917B0315
:10AA6000882349F0815080937B03882321F4B0929E
:10AA7000EF02A092EE0280918B0190918C01892BC4
:10AA8000F9F480918D019927289FA001299F500DED
:10AA9000389F500D1124CA01B2010E94497ACB019E
:10AAA000AA2797FDA095BA2F680E791E8A1E9B1EB5
:10AAB000609218087092190880921A0890921B08E8
:10AAC00080917B03882369F58091EE029091EF02DB
:10AAD0002091C5073091C607821B930B845E9D4F62
:10AAE00068E671E00E94497A9C01245B30408091C5
:10AAF000770186959927289FB001299F700D389F6F
:10AB0000700D11249B0177FF02C0215F3F4FF4E0DD
:10AB100035952795FA95E1F73093C3022093C20249
:10AB200004C01092C3021092C2028091EC028823EA
:10AB300081F01092F4021092F5021092F602109237
:10AB4000F7021092F8021092F9021092FA02109293
:10AB5000FB02F090BB02FF20F1F48091EE07282F5A
:10AB60003327442755278091300390913103A091DA
:10AB70003203B0913303BC01CD010E940A7ADC019B
:10AB8000CB01BC01CD0128EF3AE240E050E00E9449
:10AB90007E7A390102C066247724E090BA02EE2062
:10ABA000F1F48091EE07282F332744275527809111
:10ABB000280390912903A0912A03B0912B03BC0193
:10ABC000CD010E940A7ADC01CB01BC01CD0128EF46
:10ABD0003AE240E050E00E947E7A290102C044241B
:10ABE00055248091C2079091C307893C91051CF0C0
:10ABF00088EC90E005C088539F4F34F488E39FEFC2
:10AC00009093C3078093C2078091CE079091CF079E
:10AC1000893C91051CF088EC90E005C088539F4F5B
:10AC200034F488E39FEF9093CF078093CE07809111
:10AC3000D0079091D107AA2797FDA095BA2F209110
:10AC40001608A22EBB24CC24DD24BC01CD01A60114
:10AC500095010E940A7A9B01AC018091C2079091F4
:10AC6000C307AA2797FDA095BA2FE7E0880F991F81
:10AC7000AA1FBB1FEA95D1F7280F391F4A1F5B1F78
:10AC800057FF04C0215C3F4F4F4F5F4F76E0559513
:10AC90004795379527957A95D1F78301020F131FB2
:10ACA0001093D1070093D0078091C0079091C107FE
:10ACB000AA2797FDA095BA2FBC01CD01A601950149
:10ACC0000E940A7A9B01AC018091CE079091CF0738
:10ACD000AA2797FDA095BA2F67E0880F991FAA1F92
:10ACE000BB1F6A95D1F7280F391F4A1F5B1F57FFFB
:10ACF00004C0215C3F4F4F4F5F4FF6E0559547959D
:10AD000037952795FA95D1F74201820E931E9092BE
:10AD1000C1078092C0078091110890911208880F96
:10AD2000991FAA2797FDA095BA2F2091C70733270F
:10AD300044275527BC01CD010E940A7A5B016C01B2
:10AD400097FF08C02FE330E040E050E0A20EB31EB2
:10AD5000C41ED51EE6E0D594C794B794A794EA958F
:10AD6000D1F78091DD07282F33274427552780917D
:10AD7000140390911503A0911603B0911703BC0121
:10AD8000CD010E940A7ADC01CB01BC01CD0120EF8C
:10AD900035E540E050E00E947E7AB501620F731FF6
:10ADA00070931208609311080150104134F080E054
:10ADB00090E19093D1078093D0078091D007909134
:10ADC000D1078050904F34F480E090EF9093D107FA
:10ADD0008093D00751E0851650E1950634F080E06D
:10ADE00090E19093C1078093C0078091C007909134
:10ADF000C1078050904F34F480E090EF9093C107EA
:10AE00008093C0076150704134F080E090E19093EE
:10AE100012088093110880911108909112088050B7
:10AE2000904F34F480E090EF9093120880931108D3
:10AE300080910001482F552780911E0190911F019C
:10AE40004817590794F420911E0130911F01098180
:10AE50001A81049FC001059F900D149F900D11242D
:10AE6000B9010E94357A7A83698329813A81220F58
:10AE7000331F220F331F3A8329834091080840FF74
:10AE8000EBC7EE2009F0E8C7FF2009F0E5C700E0B6
:10AE900010E048018091BC029091BD029093A605FC
:10AEA0008093A50520914703309148032115310572
:10AEB00009F03FC080911401909115018959934088
:10AEC00058F087B5853F20F48091ED01815011C085
:10AED00081E080939F034EC08091140190911501F1
:10AEE0008436910508F587B58B30D0F08091ED015F
:10AEF0008F5F8093ED019AE0890290011124809187
:10AF0000CC05821B87BD8CE291E09093DB0180939E
:10AF1000DA018EE591E090934803809347032AC0BD
:10AF200081E080939E0326C0F0929E03F0929F03DF
:10AF300021C08091D0029091D102A091D202B09113
:10AF4000D30264E0880F991FAA1FBB1F6A95D1F72F
:10AF50008093EE019093EF01A093F001B093F10183
:10AF60001093EC010093EB012150304030934803E3
:10AF70002093470320917A0141FF24C02233D8F463
:10AF8000809191018150809391018F3FD9F510926A
:10AF9000ED028091D0029091D102A091D202B091A5
:10AFA000D3028093CC029093CD02A093CE02B093B3
:10AFB000CF0281E004C081E08093ED0288EC8093B1
:10AFC000910120C08091470190914801820F911D0D
:10AFD000209132063327829FA001839F500D929FBC
:10AFE000500D1124CA01AA2797FDA095BA2F80936E
:10AFF000CC029093CD02A093CE02B093CF0281E019
:10B000008093ED028091300390913103A09132033F
:10B01000B0913303E0904301F09044010091450169
:10B0200010914601BC01CD01A80197010E947E7AD2
:10B0300059016A018091280390912903A0912A0364
:10B04000B0912B03BC01CD01A80197010E947E7A2B
:10B05000B901C5010E94B86F5C01CC971CF05CE39C
:10B06000A52EB12CC5010E94B26B5C0180E28093D9
:10B0700042011092CB021092CA028091ED02882305
:10B0800009F45CC58091A00299279C012071307061
:10B0900084FD54C580919F02826080939F027091CD
:10B0A000EC07872F992741E0C42ED12CC822D92242
:10B0B00080FD04C08091080881FD10C0C980DA803D
:10B0C00030939703209396033093CB022093CA02C8
:10B0D0008091A002806C8093A002A8C28091A002FF
:10B0E00081FF7AC20091810110918201C8010F96FF
:10B0F0002090E0023090E102821593050CF058C0D8
:10B1000080919E03882309F053C08091A00287FF9D
:10B1100015C08091A0028F778093A0028091D00209
:10B120009091D102A091D202B091D3028093CC022F
:10B130009093CD02A093CE02B093CF028091A00253
:10B1400080648093A002E090CC07EE20F1F0809123
:10B15000CC029091CD02A091CE02B091CF02BC0161
:10B16000CD0124E630E040E050E00E947E7A8E2D52
:10B170009927AA27BB2782179307A407B5072CF4A2
:10B18000D092CB02C092CA0210C0C101801B910BA9
:10B190000F9797FF03C0909581959F4F9093CB0297
:10B1A0008093CA028BE2809342011092C40216C1BE
:10B1B000C8010F9728163906C4F520919F03222352
:10B1C000A1F58091A00286FF15C08091A0028F7B1F
:10B1D0008093A0028091D0029091D102A091D202DE
:10B1E000B091D3028093CC029093CD02A093CE0273
:10B1F000B093CF028091A00280688093A002C10129
:10B20000801B910B0F9697FF03C0909581959F4FE0
:10B21000909581959F4F9093CB028093CA028DE2C7
:10B22000809342012093C402D9C08DE380934201F0
:10B230006091C502662371F12091C6023091C70268
:10B240004091C8025091C9028091CC029091CD02E8
:10B25000A091CE02B091CF0282179307A407B50741
:10B26000CCF48091A00280648093A002862F99275D
:10B270009093CB028093CA028AE08093C4028EE549
:10B28000809342018091A00287FFA8C08091A00214
:10B290008F7733C0662309F443C02091C6023091F2
:10B2A000C7024091C8025091C9028091CC0290918E
:10B2B000CD02A091CE02B091CF02281739074A07DC
:10B2C0005B0774F58091A00280688093A002862FAE
:10B2D0009927909581959F4F9093CB028093CA02B6
:10B2E00086EF8093C40286E7809342018091A0029A
:10B2F00086FF74C08091A0028F7B8093A002809112
:10B30000D0029091D102A091D202B091D302809349
:10B31000CC029093CD02A093CE02B093CF025EC038
:10B320008091A002807C09F459C08091C4028823D6
:10B3300079F5E090D002F090D1020091D202109104
:10B34000D302D801C70180589040A040B04020915E
:10B35000CC023091CD024091CE025091CF028217A3
:10B360009307A407B5075CF4D801C70180589F4F25
:10B37000AF4FBF4F281739074A075B075CF0809330
:10B38000CC029093CD02A093CE02B093CF0202C024
:10B390001092C4028091A0028F738093A002109239
:10B3A00097031092960371FF06C084EF91E090938B
:10B3B000DB018093DA018091D402882379F48091B3
:10B3C000D0029091D102A091D202B091D302C39742
:10B3D000A105B1051CF081E08093D4026091960331
:10B3E000709197038091CA029091CB02680F791FE8
:10B3F0007093970360939603CB0177FF04C088276F
:10B400009927861B970B855F91400CF4CEC0409125
:10B41000C402442389F18091C6029091C702209111
:10B42000CC023091CD02821B930B0996439748F4CE
:10B430008091C6029091C702A091C802B091C90242
:10B4400012C0242F332727FD3095432F532F80918F
:10B45000CC029091CD02A091CE02B091CF02820F8A
:10B46000931FA41FB51F8093CC029093CD02A0938D
:10B47000CE02B093CF0224C0809132062091CC023C
:10B480003091CD024091CE025091CF021616170690
:10B4900044F463E00E94297A280F311D411D511D9B
:10B4A00007C063E00E94297A281B3109410951092C
:10B4B0002093CC023093CD024093CE025093CF0222
:10B4C0001092970310929603E090D002F090D10270
:10B4D0000091D2021091D302D801C701805094404C
:10B4E000A040B0402091CC023091CD024091CE02DC
:10B4F0005091CF0282179307A407B5075CF4D801D7
:10B50000C70180509C4FAF4FBF4F281739074A07DC
:10B510005B0744F08093CC029093CD02A093CE02BF
:10B52000B093CF028091EC0781FF06C084E690E0E3
:10B530009093DB018093DA01809136068823A9F588
:10B540008091C502882389F54091BC025091BD02CB
:10B5500057FF02C04D5F5F4F5595479555954795ED
:10B5600080911E0190911F01209100013327489F77
:10B57000F001499FF00D589FF00D1124CF01B90142
:10B580000E94497A7093820160938101663471054B
:10B590001CF486E490E005C06739710534F086E953
:10B5A00090E0909382018093810180914703909174
:10B5B0004803892BB9F18091D0029091D102A091DA
:10B5C000D202B091D3028093CC029093CD02A0938B
:10B5D000CE02B093CF0226C08091D0029091D102CA
:10B5E000A091D202B091D30280599140A040B040C6
:10B5F0008093CC029093CD02A093CE02B093CF0261
:10B6000080913606882311F0992702C088E790E0E0
:10B610009093820180938101E980FA80F092BD02CB
:10B62000E092BC02C090BC02D090BD02E090D0027B
:10B63000F090D1020091D2021091D3022091CC025D
:10B640003091CD024091CE025091CF022E153F0590
:10B650004007510724F08091EC0780FDBBC2809128
:10B66000470390914803892B39F0C090BC02D090D9
:10B67000BD0200E010E0D7C0D801C701821B930BC8
:10B68000A40BB50B8093650390936603A0936703A7
:10B69000B0936803823000E890070FEFA0070FEF28
:10B6A000B0072CF481E090E8AFEFBFEF09C08F5FE7
:10B6B0009F47A040B04064F08FEF9FE7A0E0B0E06C
:10B6C0008093650390936603A0936703B093680328
:10B6D000009165031091660380917901282F33272B
:10B6E000442755278091650390916603A0916703D5
:10B6F000B0916803BC01CD010E940A7A97FF04C093
:10B70000615E7F4F8F4F9F4F25E095958795779589
:10B7100067952A95D1F760936503709366038093CC
:10B7200067039093680365302EEF72072FEF82074F
:10B730002FEF92072CF484E09EEFAFEFBFEF09C02C
:10B74000605074408040904064F080E094E0A0E05D
:10B75000B0E08093650390936603A0936703B09372
:10B76000680380906503909066032091EB0130910F
:10B77000EC0137FF02C0295F3F4F83E035952795E5
:10B780008A95E1F74FEF223834071CF421E83FEFA8
:10B7900005C02038310514F020E830E0C901AA279F
:10B7A00097FDA095BA2F20917B0133274427552779
:10B7B000BC01CD010E940A7A97FF04C06D5F7F4FE4
:10B7C0008F4F9F4FB2E09595879577956795BA957E
:10B7D000D1F79B015FEF613075071CF420E03FEF6C
:10B7E00006C06F3F710519F014F020E031E0809140
:10B7F000A002807C49F0C90137FD03969C01359574
:10B800002795359527950DC08091EC0780FF09C0DD
:10B81000C90137FD07969C01F3E035952795FA9508
:10B82000E1F7820E931E20917801222309F454C07F
:10B830006091F0027091F1028091F2029091F30216
:10B8400097FF04C061587F4F8F4F9F4FE7E095955A
:10B85000879577956795EA95D1F73327442755273C
:10B860000E940A7A97FF04C0615E7F4F8F4F9F4FFF
:10B8700055E095958795779567955A95D1F760939B
:10B880006503709366038093670390936803613840
:10B89000AFEF7A07AFEF8A07AFEF9A072CF480E893
:10B8A0009FEFAFEFBFEF0AC06F3F710581059105B4
:10B8B00069F064F080E091E0A0E0B0E0809365037F
:10B8C00090936603A0936703B09368038091650328
:10B8D00090916603880E991E80917601282F332758
:10B8E00080919C08992787FD9095289FF001299FBA
:10B8F000F00D389FF00D11249F01F7FF02C0215871
:10B900003F4F220F232F221F330BFFEF21383F071A
:10B910001CF420E83FEF06C02F3F310519F014F06A
:10B9200020E031E0820E931EC401AA2797FDA09566
:10B93000BA2FE090BC02F090BD029701442737FD7A
:10B940004095542FBC01CD010E940A7A97FF04C094
:10B9500061507E4F8F4F9F4F29E095958795779542
:10B9600067952A95D1F7C61AD70A8091CA02909195
:10B97000CB02892B09F060C01E141F040CF05CC0C0
:10B98000980117FF03C0309521953F4F2D333105A6
:10B9900040F48091E8029091E9028C159D0574F5C0
:10B9A00026C02C53304085E0369527958A95E1F7DF
:10B9B0002031310510F02FE030E04091E802509145
:10B9C000E90210161106E4F480E190E0821B930B6B
:10B9D000489F9001499F300D589F300D1124B4E0CD
:10B9E00036952795BA95E1F72C153D0520F5809100
:10B9F0007F0190918001C816D906F4F06C011CC03B
:10BA0000205F3F4F80917F0190918001829F800154
:10BA1000839F100D929F100D11249801A4E036957C
:10BA20002795AA95E1F74C155D0514F06A0104C04D
:10BA3000C216D30608F06901C601AA2797FDA09592
:10BA4000BA2FFDE0880F991FAA1FBB1FFA95D1F7E7
:10BA50009501442737FD4095542FBC01CD010E942C
:10BA60007E7A2093690330936A0340936B0350936B
:10BA70006C03C0906903D0906A0380919803909101
:10BA800099039C01220F331F280F391F2C0D3D1DD8
:10BA900037FF02C02D5F3F4FA9015595479555953A
:10BAA0004795509399034093980380912E06282F31
:10BAB0003327220F331F220F331F241735076CF44F
:10BAC00080911008282F3327220F331F220F331F96
:10BAD000205530404217530724F0309399032093A8
:10BAE00098038091EC0780FF14C080919803909197
:10BAF000990329813A818217930724F0309399039F
:10BB00002093980340919803509199035A83498355
:10BB100061C029813A812E193F0937FF02C02D5F8C
:10BB20003F4F3595279535952795609198037091EE
:10BB30009903620F731F7A8369834CC08091360624
:10BB4000882301F56091BC027091BD0277FF02C0AD
:10BB50006D5F7F4F759567957595679540911E014F
:10BB600050911F0180910001282F3327649FC0014D
:10BB7000659F900D749F900D1124B9010E94497A20
:10BB8000CB0101C09927909382018093810180911C
:10BB9000810190918201873491051CF486E490E044
:10BBA00005C08639910534F086E990E090938201D2
:10BBB0008093810189819A8190939903809398035E
:10BBC0008091A002806C8093A00280919F028D7F63
:10BBD00080939F028091A00299279C01227030706F
:10BBE00081FF2BC180919A0390919B03A0919C03AC
:10BBF000B0919D030097A105B10521F08091D40279
:10BC00008130B1F4E981FA81CF01AA2797FDA0958F
:10BC1000BA2F1EE0880F991FAA1FBB1F1A95D1F7D4
:10BC200080939A0390939B03A0939C03B0939D03EE
:10BC30008091D402813019F482E08093D402E980AB
:10BC4000FA80C701AA2797FDA095BA2F950144272E
:10BC500037FD4095542FBC01CD010E940A7ADC01CA
:10BC6000CB018093690390936A03A0936B03B09315
:10BC70006C03B7FF04C08150904EAF4FBF4F7C01A3
:10BC80008D01FDE015950795F794E794FA95D1F7A6
:10BC9000E0926903F0926A0300936B0310936C03C4
:10BCA0006091A1027091A2022FE0603A720750F5F4
:10BCB00080919A0390919B03A0919C03B0919D0366
:10BCC0009C01AD01EAE05695479537952795EA9591
:10BCD000D1F7821B930BA40BB50BA8019701F4E0DD
:10BCE000220F331F441F551FFA95D1F7820F931F60
:10BCF000A41FB51F80939A0390939B03A0939C036A
:10BD0000B0939D0360547F4118F580919A03909100
:10BD10009B03A0919C03B0919D039C01AD01ECE0BD
:10BD20005695479537952795EA95D1F7821B930B42
:10BD3000A40BB50BA801970172E0220F331F441F1B
:10BD4000551F7A95D1F7820F931FA41FB51F38C0D6
:10BD50008091EB019091EC018091EB019091EC01CD
:10BD600097FF03C0909581959F4F8436910584F588
:10BD70008091D0029091D1022091CC023091CD02DD
:10BD8000821B930B81509F4F8F5F914008F58091EC
:10BD90009A0390919B03A0919C03B0919D039C01F9
:10BDA000AD016EE056954795379527956A95D1F781
:10BDB000821B930BA40BB50B8E0D9F1DA01FB11FF3
:10BDC00080939A0390939B03A0939C03B0939D034D
:10BDD00080919A0390919B03A0919C03B0919D0345
:10BDE0005EE0B695A795979587955A95D1F790936C
:10BDF000BD028093BC0240913406442399F055273C
:10BE00009C01BA010E94497AC901861B970B909345
:10BE1000E9028093E802260F371F309380012093B8
:10BE20007F011FC01092E9021092E8028FEF93E0A9
:10BE30009093800180937F0114C01092D4021092DD
:10BE40009A0310929B0310929C0310929D033093CF
:10BE5000BD022093BC0205C08091A002806C80933B
:10BE6000A0022091D507822F9927880F991F880F4C
:10BE7000991F889669817A818617970714F09A83AB
:10BE80008983709110087D8B872F9927880F991FC0
:10BE9000880F991F80559040A981BA818A179B0706
:10BEA00014F49A83898380912302882341F480913A
:10BEB000AE088F3F21F48091AD038823E9F0809193
:10BEC000A1029091A2020297C097B0F4E981FA8191
:10BED0001E161F068CF481E090E09093A2028093DE
:10BEE000A102E22EFF24EE0CFF1CEE0CFF1C8701CA
:10BEF000085D1F4F1A83098329813A8130938A058F
:10BF0000209389058091610390916203A09163035E
:10BF1000B091640312E0880F991FAA1FBB1F1A95E6
:10BF2000D1F70091110810911208081B190B213A42
:10BF300031058CF0C90137FD0196959587958017DD
:10BF400091070CF48C01909581959F4F0817190764
:10BF50006CF48C010BC00135110514F000E510E004
:10BF60003FEF003B130714F400EB1FEF4D89242F24
:10BF70003327220F331F220F331FC90169817A81B2
:10BF8000861B970B801791070CF48C0189819A818D
:10BF9000821B930B081719070CF48C018091D007B2
:10BFA0009091D1076091E6027091E702861B970B92
:10BFB0009093DF078093DE07D090EE072091F80280
:10BFC0003091F9024091FA025091FB02DD2041F0DC
:10BFD000661A770AC301AA2797FDA095BA2F04C055
:10BFE000AA2797FDA095BA2F280F391F4A1F5B1F5C
:10BFF0002093F8023093F9024093FA025093FB0227
:10C000008091F8029091F902A091FA02B091FB029E
:10C0100081509A4FA040B04064F080E09AEFA0E0D9
:10C02000B0E08093F8029093F902A093FA02B093E3
:10C03000FB028091F8029091F902A091FA02B0916E
:10C04000FB0280509640AF4FBF4F64F480E096E013
:10C05000AFEFBFEF8093F8029093F902A093FA023A
:10C06000B093FB02C09043062091DE073091DF07BA
:10C0700078E0E72EEC1498F08C2D9927829FA00190
:10C08000839F500D929F500D1124CA0157FD0796B2
:10C090007C0163E0F594E7946A95E1F712C08C2D7A
:10C0A00086959927829FB001839F700D929F700D96
:10C0B0001124CB0177FD03967C01F594E794F59468
:10C0C000E794A0907C01B0907D019501442737FD55
:10C0D0004095542F8091F8029091F902A091FA02B4
:10C0E000B091FB02BC01CD010E947E7AE20EF31EEC
:10C0F00090906801692D772788279927980117FF65
:10C1000004C022273327201B310B37FF02C02F5FCB
:10C110003F4F35952795A981BA812A0F3B1F4427A8
:10C1200037FD4095542F0E940A7A97FF04C0615C46
:10C130007F4F8F4F9F4F26E0959587957795679511
:10C140002A95D1F79B016E157F050CF47B01309584
:10C1500021953F4FE216F3060CF479018091C00758
:10C160009091C1076091E4027091E502861B970BE4
:10C170009093BF078093BE072091F4023091F5029F
:10C180004091F6025091F702DD2041F0461A570A1D
:10C19000C201AA2797FDA095BA2F04C0AA2797FD30
:10C1A000A095BA2F280F391F4A1F5B1F2093F40256
:10C1B0003093F5024093F6025093F7028091F40217
:10C1C0009091F502A091F602B091F70281509A4F3A
:10C1D000A040B04064F080E09AEFA0E0B0E080932F
:10C1E000F4029093F502A093F602B093F7028091C7
:10C1F000F4029091F502A091F602B091F7028050FE
:10C200009640AF4FBF4F64F480E096E0AFEFBFEFD2
:10C210008093F4029093F502A093F602B093F70294
:10C220002091BE073091BF0748E04C1598F08C2D47
:10C230009927829FB001839F700D929F700D1124EA
:10C24000CB0177FD07966C01B3E0D594C794BA95FE
:10C25000E1F712C0C6948C2D9927829FD001839F4D
:10C26000B00D929FB00D1124CD01B7FD03966C0166
:10C27000D594C794D594C7949501442737FD40952C
:10C28000542F8091F4029091F502A091F602B091A2
:10C29000F702BC01CD010E947E7AC20ED31E692D29
:10C2A000772788279927980117FF04C0222733276B
:10C2B000201B310B37FF02C02F5F3F4F359527956D
:10C2C000E981FA812E0F3F1F442737FD4095542FF7
:10C2D0000E940A7A97FF04C0615C7F4F8F4F9F4F87
:10C2E000E6E09595879577956795EA95D1F79B0157
:10C2F0006C157D050CF46B01309521953F4FC216EE
:10C30000D3060CF469018091D507282E3324509070
:10C3100084066EEE862E66E0962E55EAA52E56E031
:10C32000B52E4BE0442E3FEE632E37E0732ED50141
:10C330002C9112160CF029C1203429F4E981FA81DC
:10C34000FF8BEE8B1FC049815A81CA01AA2797FD36
:10C35000A095BA2F332727FD3095432F532FBC01CB
:10C36000CD010E940A7A97FF04C0615C7F4F8F4F16
:10C370009F4F26E095958795779567952A95D1F7F4
:10C380007F8B6E8BF5012181203439F42E893F8912
:10C390002E0D3F1D3F8B2E8B2AC0203C39F44E8939
:10C3A0005F894E195F095F8B4E8B21C0C701AA2799
:10C3B00097FDA095BA2F332727FD3095432F532F94
:10C3C000BC01CD010E940A7A97FF04C0615C7F4FD7
:10C3D0008F4F9F4FB6E09595879577956795BA955E
:10C3E000D1F7AE89BF89A60FB71FBF8BAE8BF50102
:10C3F0002281203439F42E893F892C0D3D1D3F8B3D
:10C400002E8B2AC0203C39F44E895F894C195D0976
:10C410005F8B4E8B21C0C601AA2797FDA095BA2F2E
:10C42000332727FD3095432F532FBC01CD010E94A8
:10C430000A7A97FF04C0615C7F4F8F4F9F4FA6E041
:10C440009595879577956795AA95D1F7AE89BF8918
:10C45000A60FB71FBF8BAE8BF5012381203439F4B3
:10C460002E893F89200F311F3F8B2E8B2AC0203C05
:10C4700039F44E895F89401B510B5F8B4E8B21C075
:10C48000C801AA2797FDA095BA2F332727FD30951D
:10C49000432F532FBC01CD010E940A7A97FF04C09D
:10C4A000615C7F4F8F4F9F4FF6E09595879577950D
:10C4B0006795FA95D1F7AE89BF89A60FB71FBF8BD5
:10C4C000AE8BF301808191812E893F89821793077A
:10C4D00064F4B901680F791F77FF02C06F5F7F4F67
:10C4E000759567957F8B6E8B1DC0552049F44E89DD
:10C4F0005F89440F551F481B590B5F8B4E8B12C031
:10C5000051E0551578F4252D33276E897F89861BD8
:10C51000970BB9010E94497AAE89BF89A60FB71F50
:10C52000BF8BAE8BC101880F991F880F991FEE89B1
:10C53000FF898E179F0764F4FD898F2F9927880F35
:10C54000991F880F991F2E893F892817390714F0E2
:10C550009F8B8E8B8E899F8997FD039695958795E6
:10C5600095958795F4018183880F991F880F991FEE
:10C570002E893F89281B390BC901880F8283EE89D8
:10C58000FF89D301ED93FC9303C0F4011182128261
:10C590004A9422E030E0620E731E44E050E0A40EA4
:10C5A000B51E68E070E0860E971E47FEC0CEE2E141
:10C5B000C95E0C94B57A84B1806A84B93D9A82E5EB
:10C5C0008CBD1DBC459A81E0809322088AEA809345
:10C5D000330883E8809334088AE08093350810920A
:10C5E00037081092360810923908109238081092C5
:10C5F0009B0810925708089530912208332309F0C0
:10C6000085C00DB407FE82C084E08093D901459AAD
:10C610002EB58091B00399278130910589F0823041
:10C6200091051CF4892B21F03EC00297B9F03BC064
:10C63000309356082093B1032138A9F581E008C052
:10C64000253549F48091B103820F8093B10382E0D4
:10C650008093B00328C03093B00325C08091560862
:10C66000E82FFF27E858F74F20838F5F8093560805
:10C670009091B1038032A0F0291769F480E2A8E715
:10C68000B8E0E8E5F8E00D9001928A95E1F781E0E5
:10C690008093570802C0309357081092B00303C02C
:10C6A000920F9093B10320913208223208F028C0F3
:10C6B000459800000000000000000000000000009D
:10C6C000000000000000000000000000000000006A
:10C6D000000000000000000000000000000000005A
:10C6E0000000E0912B08F0912C08E20FF11D8081F1
:10C6F0008EBD809154089081890F8093540803C0A7
:10C7000081E0809322082F5F209332080895EF92F2
:10C71000FF920F931F9380913C069927880F991FD2
:10C72000880F991F7C010027F7FC0095102F80913E
:10C73000300390913103A0913203B0913303BC01D7
:10C74000CD01A80197010E947E7A3093370820938B
:10C7500036088091280390912903A0912A03B09173
:10C760002B03BC01CD01A80197010E947E7A309372
:10C770003908209338082091180830911908409101
:10C780001A0850911B08DA01C90163E0880F991F4C
:10C79000AA1FBB1F6A95D1F7820F931FA41FB51F55
:10C7A000820F931FA41FB51F2091430130914401B4
:10C7B0004091450150914601BC01CD010E947E7A15
:10C7C00030933F0820933E088091410390914203AB
:10C7D0002091F9013091FA01821B930B9093450847
:10C7E00080934408E0913703F09138038091E50786
:10C7F0009091E607BF010E94497A9B01220F331FE7
:10C80000220F331F260F371F260F371F37FF02C097
:10C810002D5F3F4F359527953595279530933B08EC
:10C8200020933A088091140890911508BF010E9446
:10C83000497A9B01220F331F220F331F260F371F08
:10C84000260F371F37FF02C02D5F3F4F35952795C5
:10C850003595279530933D0820933C081092380376
:10C86000109237031092E6071092E5071092150810
:10C87000109214088091350899278D30910509F49C
:10C880008EC08E3091055CF48B30910509F4B6C0F2
:10C890008C3091050CF037C10A9761F0E7C18F30F9
:10C8A000910509F4B3C18F3091050CF482C1409712
:10C8B000A9F1DCC18091B502809348088091B4024F
:10C8C000809349088091B30280934A088091B20214
:10C8D00080934B088091B10280934C088091B00204
:10C8E00080934D088091AF0280934E088091AE02F4
:10C8F00080934F088091A002809350088091A002FD
:10C90000837F8093A0020E94342C809351088091F1
:10C9100085068093520880919F02A6C18091A80845
:10C920009091A90890934908809348088091AC0899
:10C930009091AD0890934B0880934A0880911E0116
:10C9400090911F0180934C088091000180934D08C5
:10C950008091420180934E088091080880934F088F
:10C960008091EC07809350089091B2039093510806
:10C97000E92FFF27A3E0EE0FFF1FAA95E1F7E25191
:10C98000F94F878180935208858180935308892FBE
:10C990008F5F6CE00E94297A9093B20367C1809107
:10C9A00070068093480880917106809349088091B1
:10C9B000720680934A088091730680934B08809199
:10C9C000740680934C088091780680934D0880917E
:10C9D000790680934E0880917A0680934F08809163
:10C9E0007D068093500880917B068093510880914A
:10C9F0007C068093520880917E0636C1F89480911F
:10CA00002306E82FFF27EE0FFF1FE15BF84F019091
:10CA1000F081E02DE038F1051CF0EFE7F0E006C012
:10CA20002FEFE138F20714F4E1E8FFEFE093480854
:10CA300080912406E82FFF27EE0FFF1FE15BF84FE0
:10CA40000190F081E02DE038F1051CF0EFE7F0E017
:10CA500006C06FEFE138F60714F4E1E8FFEFE0936A
:10CA6000490880912206E82FFF27EE0FFF1FE15BA8
:10CA7000F84F0190F081E02DE038F1051CF0EFE770
:10CA8000F0E006C08FEFE138F80714F4E1E8FFEFBB
:10CA9000E0934A0880912106E82FFF27EE0FFF1F41
:10CAA000E15BF84F0190F081E02DE038F1051CF0DA
:10CAB000EFE7F0E006C02FEFE138F20714F4E1E809
:10CAC000FFEF7894E0934B088091D70280934C0855
:10CAD0008091D80280934D088091D90280934E08AE
:10CAE0008091DA0280934F088091DB028093500896
:10CAF0008091DC02809351088091DD02809352087E
:10CB00008091DE02B1C080911404863018F010923A
:10CB1000140485E08093480880917F06809349083B
:10CB20008091D0029091D102A091D202B091D30213
:10CB3000BC01CD0125E030E040E050E00E947E7A6B
:10CB400030934B0820934A088091CC029091CD02FB
:10CB5000A091CE02B091CF02BC01CD0125E030E022
:10CB600040E050E00E947E7A30934D0820934C08BC
:10CB70008091750680934E088091760680934F08C9
:10CB800080917706809350088091D6028093510857
:10CB900080914F07909150078093520880918905AA
:10CBA00090918A0597FD039695958795959587951C
:10CBB0005BC01092480886E58093490881E0809325
:10CBC0004A088AE180934B088091020180934C08C7
:10CBD0008091F90380934D088091FA0380934E0869
:10CBE0001092F90380718093FA038091FB03809384
:10CBF0004F088091FC03809350088091FD0380933F
:10CC00005108809181068093520830C0809155066A
:10CC100080934808809189068093490880916E012D
:10CC200080934A0880914E0680934B0880914F066E
:10CC300080934C088091500680934D0880916D013F
:10CC400080934E088091520680934F08809153063E
:10CC50008093500880915406809351088091AE08CB
:10CC6000809352088091B3058093530880915708B0
:10CC7000882309F42DC18AEF80939C0181E0809381
:10CC80008E014091590850915A08CA0181509E4F17
:10CC90008F5F9340B0F420915B0830915C08C9012C
:10CCA00081509E4F8F5F934060F480912D0685FFE9
:10CCB00008C05093A4034093A3033093A20320938E
:10CCC000A10380915F089091600821E08936920766
:10CCD00024F49093900180938F0120916908309102
:10CCE0006A088091DA019091DB018217930720F4A2
:10CCF0003093DB012093DA01809158089927883618
:10CD0000910509F464C08936910524F487369105AC
:10CD100031F0E6C08936910509F48AC0E1C08091FE
:10CD20006B088093980880916C0880939A08809192
:10CD30006D088093990880916E0880938D01809191
:10CD40006F0880939C088091700880939D0180916A
:10CD500071088093AF03809172088093A003809143
:10CD6000AD028823F9F0209173083091740837FDE3
:10CD700019C03093EF022093EE0290915706992349
:10CD800089F08FE0989FC0011124281B390BC9013D
:10CD900088599E4F68E671E00E94497A9093EF02AD
:10CDA0008093EE022091AB033091AC038091750823
:10CDB00090917608280F391F37FF02C02F5F3F4F31
:10CDC000359527953093AC032093AB0389C08091B0
:10CDD0006B0880932D0880916C0880932E088091B9
:10CDE0006D0880932F0880916E08809330088091A1
:10CDF0006F08809331088091790590917008892B94
:10CE00008093790590917A059370809171088C7068
:10CE1000982B90937A05809172088093AD0380914E
:10CE20007308809392018091740880939B0858C086
:10CE300080916B088093230880916C08809324086C
:10CE400080916D088093250880916E088093260854
:10CE500080916F089091700890932808809327081C
:10CE6000809171089091720890932A088093290804
:10CE700080917308992787FD9095909382078093FE
:10CE80008107809174088093C50280917508909104
:10CE900076089C01442737FD4095542FDA01C901DB
:10CEA00063E0880F991FAA1FBB1F6A95D1F7820FF5
:10CEB000931FA41FB51F820F931FA41FB51F80933C
:10CEC000C6029093C702A093C802B093C90208C0DB
:10CED0001092A4031092A3031092A2031092A10334
:10CEE0001F910F91FF90EF90089580912208882361
:10CEF00009F43BC0459883E398E090932C08809315
:10CF00002B089091AE03E92FFF27ED56FE4F9F5F50
:10CF10009093AE03808180933508993010F0109281
:10CF2000AE03109222080E94876381E0809332084A
:10CF300000000000000000000000000000000000F1
:10CF400000000000000000000000000000000000E1
:10CF500000000000000000000000000000000000D1
:10CF600080913308809354088EBD089587B18C60FA
:10CF700087B9429843981092B40380E880939F0148
:10CF80001092B30380939E0108958091B90381505C
:10CF90008093B9038F3F09F0FAC089E08093B90309
:10CFA0008091A002992780739070892B21F4809141
:10CFB000FA0380FF1DC080916E06882351F0809196
:10CFC000BC03882319F484E08093B40381E0809348
:10CFD000BC0380916F068823B9F08091BD0388233C
:10CFE00019F484E08093B30381E08093BD030CC007
:10CFF0001092BC031092BD0380916A068093BA031D
:10D0000080916C068093BB038091BC03882309F058
:10D0100040C080918806282F332724FF07C08091C5
:10D02000D502882319F425FD4DC04EC090916B06A2
:10D03000983F50F08091E7078D3D30F08091BA0322
:10D0400088230CF43FC040C0983F48F08091E70728
:10D05000853029F48091BA038823B4F133C08091DC
:10D06000B40381508093B4038F3F79F58091E70733
:10D0700086958093B40380919F01813011F480E8FC
:10D0800001C0869580939F0180919F019091BA0382
:10D0900017C08091B40381508093B4038F3FA9F4EB
:10D0A00089E08093B40380919F01813011F480E87E
:10D0B00001C0869580939F0180919F0190916E069B
:10D0C000892311F0429A01C042988091BD038823C0
:10D0D00009F041C09091880697FF07C08091D50262
:10D0E000882319F496FD50C034C090916D06983F86
:10D0F00050F080910F088D3D30F08091BB03882364
:10D100000CF442C026C0983F48F080910F0885304B
:10D1100029F48091BB038823E4F036C08091B303E7
:10D1200081508093B3038F3F91F580910F088695CE
:10D130008093B30380919E01813011F480E801C097
:10D14000869580939E0180919E019091BB038923D7
:10D15000D9F4439808958091B30381508093B30329
:10D160008F3FA9F489E08093B30380919E018130C1
:10D1700011F480E801C0869580939E0180919E0104
:10D1800090916F06892311F0439A0895439808956A
:10D190004FB724E130E0F8948091C9008F778093F5
:10D1A000C9008091C9008F7B8093C9008091C9001C
:10D1B0008F7D8093C9005A9A52985B9A539A832F15
:10D1C00099278093CD002093CC008091C800826085
:10D1D0008093C80080E18093C9008091CA008F7756
:10D1E0008093CA008091CA008F7B8093CA0080918F
:10D1F000CA008F7D8093CA008091CA008F7E809381
:10D20000CA008091CA00877F8093CA008091C900BC
:10D210008B7F8093C9008091CA0084608093CA008C
:10D220008091CA0082608093CA008091C80087FF05
:10D2300003C08091CE00F9CF8091C90080688093AF
:10D24000C9004FBF0895A0E0B0E0E9E2F9E60C9410
:10D25000A37A482F00E010E08091A001813061F4B2
:10D260001092A00184E48093C0031092C203109234
:10D27000C1031092C30325C28091C003882319F40F
:10D2800021E030E001C098019091C103992371F42D
:10D29000232B11F081E010C084E48093C0039093AD
:10D2A000C2039093C1039093C303F4C1913069F416
:10D2B000232B09F0E5C182E08093C1038091C20372
:10D2C0008F5F8093C20383E0E3C19230D1F4232BBC
:10D2D00009F0D6C183E08093C0034093C3039091CB
:10D2E000C203923039F41092C40347FF03C081E0B7
:10D2F0008093C40383E08093C1039F5F9093C20334
:10D30000C9C1933009F0BCC1232B09F0B9C1909376
:10D31000C00382E08093C1038091C2038F5F80933A
:10D32000C2032091C303822F9927782F6627842F69
:10D330009927682B792B80914706813051F47370BF
:10D34000CB018050924063E070E00E94497AEB018B
:10D3500019C0823069F47770CB018050944066E048
:10D3600070E00E94497AEB012695269526950CC01F
:10D37000EB01D370C856D140CE01D7FD0196EC0128
:10D38000D595C79526952695022F11270F701070F9
:10D390000F5F1F4F0D30110508F06BC102301105F2
:10D3A00019F404E010E005C00430110511F402E0A6
:10D3B00010E06801C00ED11EF601E15BF84F8081DC
:10D3C00091819E01281B390BC90137FF03C090953D
:10D3D00081959F4F069794F48091D602883C30F453
:10D3E0008091D602865F8093D60208C088EC809335
:10D3F000D60280916F008F7D80936F00F601E15B14
:10D40000F84F808191819C01220F331F280F391F13
:10D410002C0F3D1F37FF02C02D5F3F4F7901F59460
:10D42000E794F594E794CE0101968E159F0524F4B8
:10D430000894E108F10808C0CE010197E816F90642
:10D440001CF40894E11CF11C0630110509F0D1C050
:10D45000C536D1050CF4A8C09091BF03E92FFF2772
:10D46000E356F74FE081ED3729F48091BE038095B4
:10D470008093BE03963061F48091BE03882311F03F
:10D48000E338B9F0882309F08BC0ED3791F088C0FC
:10D49000993009F085C08091BE03882329F48091DA
:10D4A000A608833831F07CC08091A6088D3709F03A
:10D4B00077C080919E088D3739F480919F0883381A
:10D4C000B1F483E89FEF0FC0833889F480919F08FF
:10D4D000833829F410925A071092590708C08D37E3
:10D4E00031F48DE790E090935A078093590780912B
:10D4F000A008992787FD909590935C0780935B0720
:10D500008091A108992787FD909590936607809355
:10D5100065078091A208992787FD909590936807E9
:10D52000809367078091BF038930D1F58091A4086B
:10D530008D3749F480915F0790916007059690932D
:10D54000600780935F078091A5088D3749F480912B
:10D550005F079091600705979093600780935F073E
:10D5600080915F079091600783589F4F1CF483E878
:10D570009FEF09C080915F07909160078E379105FA
:10D5800034F08DE790E09093600780935F0780917F
:10D59000A308992787FD909590936407809363076C
:10D5A0001092BF031092BE03CA30D1055CF4809183
:10D5B000BF038F5F8093BF03E82FFF27E356F74F2A
:10D5C00083E880838091BF038A3011F41092BF03F7
:10D5D0008FEFCC39D8076CF48091BF03E82FFF2779
:10D5E000E356F74F8DE780838091BE03809580934B
:10D5F000BE038091D602843BD0F0F601E15BF84F88
:10D6000080819181F701E81BF90BCF0163E070E0A5
:10D610000E94497ACB01880F991F860F971F23E834
:10D6200037E0C20ED31EF6019183808307C023E842
:10D6300037E0C20ED31EF6011182108205301105AB
:10D6400040F4000F111F015B184FF801F182E082D6
:10D6500021C00530110529F4D0935E07C0935D0702
:10D6600019C007301105B1F4D0936207C093610768
:10D6700011C00231110570F081E08093A0010AC051
:10D6800081E08093A0011092C2031092C40384E44D
:10D690008093C0038091C203803198F08091C403CD
:10D6A000882331F48091A001882311F480934101F3
:10D6B0001092C2031092C4031092C10384E48093B9
:10D6C000C003E8E0CDB7DEB70C94BF7ACF93FC017E
:10D6D00097FF05C0CFEFF095E195FF4F01C0C1E086
:10D6E00028E631E0CF01B9010E94497AFC018B356F
:10D6F000910554F08B5590408A35910538F484EBB0
:10D7000090E08E1B9F0BFC0141E00DC0CF01855BBB
:10D7100090408A35910518F4E45BF04003C02E1B5D
:10D720003F0BF9014FEFEE0FFF1FE25DF64F259122
:10D7300034918C2F992787FD9095289FB001299FC0
:10D74000700D389F700D1124842F992787FD9095B7
:10D75000689FA001699F500D789F500D1124CA0148
:10D76000CF9108952AE530E0281B390BC9010E94AA
:10D77000666B0895CF93DF9380E00E949E71809145
:10D780001E0190911F016AE070E00E94497A9F9308
:10D790008F9380911E0190911F016AE070E00E94BA
:10D7A000497A7F936F938CEF99E09F938F93C1E9B0
:10D7B000D1E7DF93CF93E091E003F091E103099586
:10D7C0002DB73EB7285F3F4F2DBF80919C01882326
:10D7D00061F186E00E949E718091920199279F934A
:10D7E0008F9380912708909128086AE070E00E944A
:10D7F000357A7F936F938FED90E09F938F93809115
:10D80000C5079091C6079F938F9385E09AE09F93F9
:10D810008F93DF93CF93E091E003F091E1030995BB
:10D820008DB79EB70C968DBF12C086E00E949E7188
:10D8300083E19AE09F938F93DF93CF93E091E0038E
:10D84000F091E10309950F900F900F900F90809148
:10D85000AD038823F9F086E00E949E718091AD03AC
:10D8600099279F938F938AE19AE09F938F93DF93F9
:10D87000CF93E091E003F091E10309952DB73EB716
:10D880002A5F3F4F2DBF8091D502882319F08FE486
:10D890008093A60180E10E949E718091A8019091E1
:10D8A000A9016CE370E00E94357A9F938F93809179
:10D8B000A8019091A9016CE370E00E94357A7F93F2
:10D8C0006F938091AC089091AD089F938F9386E2FF
:10D8D0009AE09F938F93C1E9D1E7DF93CF93E091D3
:10D8E000E003F091E1030995809108082DB73EB758
:10D8F000265F3F4F2DBF80FF29C08AE10E949E71A5
:10D900008091420199279F938F938091D0029091AB
:10D91000D102A091D202B091D302BC01CD0124E684
:10D9200030E040E050E00E947E7A3F932F9383E303
:10D930009AE09F938F93DF93CF93E091E003F09170
:10D94000E10309958DB79EB708968DBFDF91CF9102
:10D950000895CF93DF9380E00E949E7180910D0720
:10D96000992787FD90959F938F938091050799271D
:10D9700087FD90959F938F938091FD06992787FD52
:10D9800090959F938F938091F506992787FD9095A9
:10D990009F938F938AE39AE09F938F93C1E9D1E796
:10D9A000DF93CF93E091E003F091E103099580E1EB
:10D9B0000E949E712DB73EB7245F3F4F2DBF8091CF
:10D9C0002D07992787FD90959F938F938091250729
:10D9D000992787FD90959F938F9380911D07992795
:10D9E00087FD90959F938F9380911507992787FDC9
:10D9F00090959F938F938AE49AE09F938F93DF9300
:10DA0000CF93E091E003F091E103099580911F0627
:10DA10002DB73EB7245F3F4F2DBF853098F480E18E
:10DA20000E949E718AE59AE09F938F93DF93CF9334
:10DA3000E091E003F091E10309950F900F900F90B2
:10DA40000F9018C08730B0F488E10E949E718FED6E
:10DA500090E09F938F938BE69AE09F938F93DF9351
:10DA6000CF93E091E003F091E10309958DB79EB764
:10DA700006968DBFDF91CF9108950F931F9380E09D
:10DA80000E949E712AE030E08091A8089091A90838
:10DA9000B9010E94357A9F938F938091A808909145
:10DAA000A908B9010E94357A7F936F9380911E0176
:10DAB00090911F01B9010E94497A9F938F938091A1
:10DAC0001E0190911F01B9010E94497A7F936F93C3
:10DAD00084E79AE09F938F9301E911E71F930F93D7
:10DAE000E091E003F091E103099580E10E949E71CD
:10DAF0008DB79EB70C968DBF8091AC089091AD0804
:10DB00009F938F938091AA089091AB089F938F93D6
:10DB100087E89AE09F938F931F930F93E091E00320
:10DB2000F091E10309958DB79EB708968DBF1F91BF
:10DB30000F9108950F931F93CF93DF9380919C01D2
:10DB4000C1E9D1E7882309F47DC080E00E949E717D
:10DB50008091240899279F938F9380912608992775
:10DB60009F938F9383E99AE09F938F938E01DF9326
:10DB7000CF93E091E003F091E10309958DB79EB753
:10DB800008968DBF80912508833031F48CE00E9487
:10DB90009E7182EA9AE005C08CE00E949E7187EA3D
:10DBA0009AE09F938F93DF93CF93E091E003F091FE
:10DBB000E10309950F900F900F900F90809123082B
:10DBC00081FF12C08CE00E949E718CEA9AE09F93C4
:10DBD0008F931F930F93E091E003F091E103099578
:10DBE0000F900F900F900F9080E10E949E71809196
:10DBF000920199279F938F938FED90E09F938F933E
:10DC00008091290890912A089F938F9380912708EB
:10DC1000909128086AE070E00E94357A7F936F93B4
:10DC200081EB9AE09F938F9381E991E79F938F9384
:10DC3000E091E003F091E10309958DB79EB70C9652
:10DC40008DBF12C082E00E949E7184EC9AE09F9387
:10DC50008F93DF93CF93E091E003F091E103099577
:10DC60000F900F900F900F90DF91CF911F910F9118
:10DC70000895CF93C82F2091C5032093C6039927F9
:10DC80008F32910509F1803391051CF44F97A1F073
:10DC90002CC08F34910501F18F38910531F5222385
:10DCA00019F481E090E038C086E0289FF00111244B
:10DCB000EC51F64F849117C086E0289FF0011124A3
:10DCC000EB51F64F84910FC086E0289FF00111249C
:10DCD000EA51F64F849107C086E0289FF001112495
:10DCE000E951F64F84918093C5039091C5038091CB
:10DCF000C6039813C0E00E94A4719091C50386E00A
:10DD0000989FF0011124E851F64F259134918C2F02
:10DD1000F901099580E090E0CF9108951092A9084B
:10DD20001092A8081092AD081092AC081092AB089F
:10DD30001092AA081092AE088AE090E00E94901615
:10DD40009093C8038093C7030895CF93DF93809186
:10DD5000C7039091C8030E949916882309F4AFC0A5
:10DD60008091C7039091C8030A969093C80380934B
:10DD7000C703E0E0F0E09F0190E05FEFAEEEB6E0B9
:10DD80004BE0ED018B8187FF0BC09F5F8D81E80F1A
:10DD9000F11D8981280F311D8E81851708F4582FB8
:10DDA0004150189647FFEDCF5093AE08232B41F515
:10DDB0002091CD033091CE034091CF035091D003F9
:10DDC000BB27A52F942F832F9093CC038093CB0355
:10DDD000AA27BB27281B390B4A0B5B0BCF01AA27AD
:10DDE000BB27280F391F4A1F5B1F2093CD03309399
:10DDF000CE034093CF035093D003E5E0F0E013C08F
:10DE00002091CB033091CC032E173F0718F4E21B6F
:10DE1000F30B02C0E0E0F0E0892F9927880F991FEB
:10DE2000E80FF91F3596F093A908E093A808EF3F93
:10DE3000F10578F480911E0190911F018E9F900151
:10DE40008F9F300D9E9F300D1124C90164E670E054
:10DE500013C0CF01969587959695879520911E01C1
:10DE600030911F01289FA001299F500D389F500D10
:10DE70001124CA0169E170E00E94357A7093AB0801
:10DE80006093AA082091C9033091CA032E0F3F1F47
:10DE90003093CA032093C9035EE02131350778F03F
:10DEA0008091AC089091AD0801969093AD08809355
:10DEB000AC0820513E403093CA032093C903DF9140
:10DEC000CF910895002422273327442751E0BB2710
:10DED000EE27FF27A0E1660F771F881F991F001C00
:10DEE000221F331F441F660F771F881F991F001CB6
:10DEF000221F331F441F2AF4050E2B1F3E1F4F1FE6
:10DF000004C0051A2B0B3E0B4F0B550FBB1FEE1F0A
:10DF1000587F556047FD5250AA95E9F6E695B795AA
:10DF20005795E695B7955795852F9B2F08952227EE
:10DF3000332741E0552768E0880F991F221F331FC0
:10DF4000880F991F221F331F1AF4240F351F02C098
:10DF5000241B350B440F551F487F456037FD425049
:10DF60006A9551F75695479556954795842F08958C
:10DF7000AA2797FF04C0809590958A1F9A1F77FF64
:10DF800004C0609570956A1F7A1F669F9001779F05
:10DF9000A001679F300D411D5A1F300D411D5A1FB2
:10DFA000889FF001999F2E0F3F1F401D511D899F93
:10DFB000300D411D5A1F300D411D5A1FCA01B901B4
:10DFC000112480CF4FB720E430E0F8948091C9004D
:10DFD0008F778093C9008091C9008F7B8093C9009F
:10DFE0008091C9008F7D8093C9005A9A52985B9A9C
:10DFF000539A832F99278093CD002093CC00809152
:10E00000C80082608093C80088E18093C900809135
:10E01000CA008F778093CA008091CA008F7B80935B
:10E02000CA008091CA008F7D8093CA008091CA0087
:10E030008F7E8093CA008091CA00877F8093CA0038
:10E040008091C9008B7F8093C9008091CA00846051
:10E050008093CA008091CA0082608093CA00809138
:10E06000C80087FF03C08091CE00F9CF8091C9001E
:10E0700080688093C9004FBF08950F931F93CF937B
:10E08000DF93482F4F5F893108F08BC080914E0796
:10E09000841720F44F5F40934E074150CB018353C8
:10E0A0009B4268E170E00E94497AA42FBB27FD01E2
:10E0B000EA0FFB1FE15BF84F808191819B01281BD8
:10E0C000390BC90137FF03C0909581959F4F069783
:10E0D00094F48091D602883C30F48091D602865F19
:10E0E0008093D60208C088EC8093D60280916F009E
:10E0F0008F7D80936F00FD01EA0FFB1FE15BF84FFE
:10E10000808191819C01220F331F280F391F260F18
:10E11000371F37FF02C02D5F3F4FE901D595C795E7
:10E12000D595C795CB0101968C179D0714F42197BF
:10E1300006C061507040C617D7070CF42196809135
:10E14000D602843BD8F08D010A0F1B1FF801E15B5A
:10E15000F84F80819181FE01E81BF90BCF0163E04C
:10E1600070E00E94497ACB01880F991F860F971F94
:10E170000D57184FF8019183808307C0AA0FBB1F6A
:10E18000AD57B84F11961C921E92E42FFF27EE0F49
:10E19000FF1FE15BF84FD183C083443011F410922C
:10E1A0004101DF91CF911F910F910895CF93DF939C
:10E1B0002091AF08822F9927807F9070409709F0B7
:10E1C0006CC02F3109F046C08091B0088093D50310
:10E1D0002091B2082093D7038091B3088093D6038F
:10E1E000822F99279093500780934F07222309F09D
:10E1F00054C080912106282F3327220F331FF901A5
:10E20000ED57F84F1182108280912206A82FBB276C
:10E21000AA0FBB1FFD01ED57F84F118210828091AC
:10E220002406E82FFF27EE0FFF1FCF018D57984FD1
:10E23000EC0119821882215B384FE901198218829A
:10E24000A15BB84F11961C921E92E15BF84F1182B0
:10E25000108223C0C22FCF70CA30F8F48091B0086A
:10E260008093D9088091B1088093D8088091B20832
:10E270008093DB088091B3088093DA086091D80816
:10E280007091D9088C2F0E943D706091DA087091CE
:10E29000DB088C2F8F5F0E943D70DF91CF91089536
:10E2A000CF93C82F8F3F49F48091D8038F3F29F433
:10E2B0001092DA031092D90332C02091DA0322239C
:10E2C00039F4CF3111F485E001C084E08093DB03A1
:10E2D0008091DB039091D9038217A0F4892F809558
:10E2E0008093D9038F3F19F48EEF8093D9038091E7
:10E2F000D903C81711F40E94D6701092DA03109255
:10E30000D9030BC0E22FFF27E155F74FC0832F5FE2
:10E310002093DA039C0F9093D903C093D803CF9135
:10E3200008959091D403933240F4E92FFF27EB54E2
:10E33000F74F80839F5F9093D4030895833218F43E
:10E340008D5F8093D403089590E2E8EBF8E08FE1CD
:10E350009193815087FFFCCF0895CF93CFB723E0EF
:10E3600031E0F8948091C9008F778093C900809143
:10E37000C9008F7B8093C9008091C9008F7D8093F5
:10E38000C9005A9A52985B9A539A832F992780937F
:10E39000CD002093CC008091C80082608093C8009B
:10E3A00088E18093C9008091CA008F778093CA006A
:10E3B0008091CA008F7B8093CA008091CA008062DE
:10E3C0008093CA008091CA0080618093CA008091C6
:10E3D000CA0088608093CA008091C90084608093DD
:10E3E000C9008091CA0084608093CA008091CA00ED
:10E3F00082608093CA008091C80087FF03C080912B
:10E40000CE00F9CF8091C90080688093C9008091C7
:10E41000C90080648093C9000E94A471CFBFCF91CE
:10E420000895282F99278F709070892B31F42095AB
:10E430008091D303822B8093D30308958091A3010D
:10E44000882309F44BC08091A00285FD04C080910F
:10E45000A601882381F082E98093B50883E2809346
:10E46000B6088091A601882309F485E58093B70852
:10E470001092A60102C08093B5088091A4018F304C
:10E4800071F48091D3030E94396E882341F081E9B1
:10E490008093B5088093B60881E38093B708109203
:10E4A000A3018091C80085FFFCCF8091C9008F7EB9
:10E4B0008093C9008091C9008E7F8093C9008091AC
:10E4C000B508882311F48EEF01C08EE78093CE004B
:10E4D0008091D3038093A4011092D30308951F92D7
:10E4E0000F920FB60F9211248F939F93EF93FF9388
:10E4F0009091A301992309F040C08091DC03882307
:10E5000061F48091B508882311F483E003C0813958
:10E5100099F481E08093DC030FC0833099F48091FB
:10E52000B508882349F09093B5088091C9008E7F83
:10E530008093C9008EEF1EC08091C90081608093D6
:10E54000C9000EC0833261F48091C9008E7F809330
:10E55000C9008FEF8093CE0081E08093A30114C0A7
:10E560008091DC03E82FFF27EB54F74F8F5F8093F8
:10E57000DC0380818093CE0007C01092DC03809181
:10E58000C90080618093C900FF91EF919F918F91A5
:10E590000F900FBE0F901F901895EF92FF920F9360
:10E5A0001F93CF93DF937C018B01EA01452B39F058
:10E5B000F80181918F01F70109952197C9F7E6E0EC
:10E5C000CDB7DEB70C94C17AEF92FF920F931F93F1
:10E5D000CF93DF937C018B01EA01452B41F0F801D9
:10E5E0000F5F1F4F8491F70109952197C1F7E6E06E
:10E5F000CDB7DEB70C94C17A0F931F93CF938C01E4
:10E60000C62F161634F480E2F8010995C1501C1685
:10E61000D4F3CF911F910F9108950F931F93CF9330
:10E620008C01C62F161634F480E3F8010995C15009
:10E630001C16D4F3CF911F910F910895A5E3B0E07C
:10E64000E4E2F3E70C94997A2E96EEADFFAD2E97A7
:10E650008824992454018091D203882321F42C9694
:10E660001FAE1EAE2C975EE4452E512C4C0E5D1E47
:10E670006F01B60105C0153239F00894C11CD11CD8
:10E68000F60114911123B9F7A601461B570B31F07F
:10E690002C968EAD9FAD2C970E94E472112309F445
:10E6A0006AC20894C11CD11CFF24FDA6FCA64FEF32
:10E6B000E42EF9A6F6010894C11CD11C149115375B
:10E6C00021F0812F80628837B1F4F0FE0AC0F20198
:10E6D00024E030E0420E531E80809180A280B380FF
:10E6E0000AC0F20142E050E0440E551E8081918143
:10E6F0004C01AA24BB24103221F489A58823D1F629
:10E700001DC0133219F458E0F52AD4CF1A3211F093
:10E710001D3291F41A3259F4F20182E090E0480E71
:10E72000591EE081ECA7EE232CF6E195ECA790E1D1
:10E73000F92AAFEDFA22BECF1B3211F419A7BACFD6
:10E740001E32C1F5F6010894C11CD11C14911A3275
:10E7500079F4F20122E030E0420E531E40815181F3
:10E760003FEF4F3F530714F44FEF5FEFE42EA2CF7C
:10E7700040E050E0812F80538A30A0F4CA0133E09A
:10E78000880F991F3A95E1F7840F951F480F591F7D
:10E79000410F511D40535040F6010894C11CD11C3B
:10E7A0001491E8CF8FEF4F3F580714F44FEF5FEF0E
:10E7B000E42E85CF103329F4F4FC7CCF90E2F92AC3
:10E7C00079CF812F81538930D8F440E050E0CA01DD
:10E7D00023E0880F991F2A95E1F7840F951F480FB2
:10E7E000591F410F511D40535040F6010894C11C60
:10E7F000D11C1491812F80538A3048F34CA75FCFEE
:10E80000183619F4A4E0FA2A55CF1C3619F4B1E0F1
:10E81000FB2A50CF133661F43E010894611C711C31
:10E82000F20122E030E0420E531E808189833CC118
:10E83000143421F0143611F0193651F5143411F452
:10E8400031E0F32AF0FE0AC0F20144E050E0440E49
:10E85000551E80809180A280B3800CC0F20182E0BE
:10E8600090E0480E591E808191814C01AA2497FCAA
:10E87000A094BA2CB7FE0AC0B094A094909480944F
:10E88000811C911CA11CB11C8DE289A70AE06FC0FC
:10E890001F3411F01F3631F41F3411F491E0F92ABE
:10E8A00008E064C0103779F4F201A2E0B0E04A0E4B
:10E8B0005B1E808191814C01AA24BB2400E1B0E45D
:10E8C000FB2A18E753C01337C1F5F20122E030E00C
:10E8D000420E531E608071806114710489F43E0100
:10E8E0000894611C711C88E289838EE6F3018183A0
:10E8F00085E78B838CE68C838D8389E28E831F82F0
:10E90000E7FC13C08E2D992787FD9095AC0160E040
:10E9100070E0C3010E946678009729F0382E3618FF
:10E92000E3140CF0C3C03E2CC1C0F30101900020E1
:10E93000E9F731973E2E3618B9C0153511F0153765
:10E9400031F4153511F4F1E0FF2A0AE00FC0183553
:10E9500019F0183709F0A0C000E1F3FE07C08114D8
:10E960009104A104B10411F020E4F22A19A6EDA645
:10E97000E7FC02C03FEDF32289E2682E712C6C0E99
:10E980007D1E81149104A104B10421F44DA54423FA
:10E9900009F47BC0802F9927AA27BB278EA79FA7A2
:10E9A000A8ABB9AB202E332490E0891690E09906ED
:10E9B00091E0A90690E0B90648F0C501B4012EA582
:10E9C0003FA548A959A90E945C7A17C0AFEF8A16E3
:10E9D0009104A104B10449F040F0C401B1010E94C6
:10E9E000357A9B014427552708C0882D602F0E9447
:10E9F000297A282F3327442755272AAB3BAB4CAB2A
:10EA00005DAB0A3059F48AA9880F880F880F9AA93C
:10EA1000990F890F382D381B832F10C0003139F41E
:10EA20008AA98295807F482D481B842F07C08AA918
:10EA3000880F880F880F582D581B852F90E02EA522
:10EA40003FA548A959A982169306A406B50608F061
:10EA500091E08AA89BA8ACA8BDA88A3010F4805D7C
:10EA600004C0895A183509F48F7DD3018E933D0176
:10EA7000992309F099CF083041F4F3FE06C08033A2
:10EA800021F080E3FD0182933F01CE010196382EF3
:10EA90003618F8E23F0E0BC0112309F46CC03E019A
:10EAA0000894611C711C1983B1E03B2E19A6032D3B
:10EAB0002DA4231827FC222489A5882311F00F5F99
:10EAC00002C0F6FC0E5F020DEF2CFF24C70180731D
:10EAD0009070892B49F48CA5801B682F2C968EADE5
:10EAE0009FAD2C970E94FC7289A5882331F041E0EC
:10EAF00050E0BE01675D7F4F0AC0E6FE0EC080E3B6
:10EB00008AA71BA742E050E0BE01665D7F4F2C96AE
:10EB10008EAD9FAD2C970E94CD72C701807390700F
:10EB2000809749F48CA5801B682F2C968EAD9FADE5
:10EB30002C970E940D73622D2C968EAD9FAD2C9755
:10EB40000E940D73832D992787FD9095AC01B30129
:10EB50002C968EAD9FAD2C970E94CD72E4FE89CD90
:10EB60002CA5201B2CA7622F2C968EAD9FAD2C9729
:10EB70000E94FC727ECDE2E1CB5C0C94B57A2FB79B
:10EB800040E0F894E0E0F0E081E280935700949157
:10EB9000E2E0F0E0809357003491E4E0F0E080930D
:10EBA000570084912FBF9E3199F4363941F4893052
:10EBB00011F441E00DC08A3059F442E009C0373900
:10EBC00039F4863011F443E003C0853009F444E0A1
:10EBD000842F992708959FB7F8948091C900877F63
:10EBE0008093C9008091C9008F7E8093C900809175
:10EBF000C9008F778093C9008091C9008F7B809373
:10EC0000C9008091C9008F7D8093C90052985A9A9B
:10EC100053985B9A9FBF08951F93CF93DF93182F4C
:10EC20008091D203882309F4A9C08091A20118170A
:10EC300009F4A4C08091D103882321F40E94BF75F8
:10EC40008093D10382ED91E09093400180933F0146
:10EC50008BEC9BE09F938F93C1E8D2E1DF93CF933E
:10EC6000E091E003F091E10309950F900F900F9070
:10EC70000F90812F99278330910539F184309105C8
:10EC80004CF48130910591F082309105DCF4892BB0
:10EC900051F036C085309105F1F085309105C4F012
:10ECA0000697E1F02DC08BEB9BE002C089EA9BE068
:10ECB0009F938F93DF93CF93E091E003F091E10373
:10ECC00009952AC080E99BE0F3CF8DE69BE0F0CF69
:10ECD0008FE59BE0EDCF87E59BE0EACF89E49BE001
:10ECE0009F938F93DF93CF93E091E003F091E10343
:10ECF000099588ED91E09093400180933F010CC00D
:10ED000088ED9BE09F938F93DF93CF93E091E00397
:10ED1000F091E103099510E00F900F900F900F9084
:10ED20008091D103843011F0823099F40E94EB7508
:10ED3000812F8150833018F40E94C8681DC01430A0
:10ED400019F40E94AD7118C01530B1F40E94E26F41
:10ED500013C0112389F08EEE9BE09F938F9381E87F
:10ED600092E19F938F93E091E003F091E103099585
:10ED70000F900F900F900F901093A201DF91CF9101
:10ED80001F9108950F931F9381E08093D2034091C8
:10ED9000A101E9EFFAE020E030E05FE484919927F7
:10EDA0002F5F3F4F829FB001839F700D929F700D28
:10EDB000112446275150319657FFF0CF4093A101BF
:10EDC000E1EDFAE020E030E057E2849199272F5FEF
:10EDD0003F4F829FB001839F700D929F700D112451
:10EDE00046275150319657FFF0CF4093A1018091B3
:10EDF000D103882321F40E94BF758093D1038091B1
:10EE0000A101833459F088E190E029E20FB6F8942B
:10EE1000A895809360000FBE209360008EE193E779
:10EE20009093E1038093E00389E09CE09F938F93AC
:10EE300001E812E11F930F93E091E003F091E103E9
:10EE400009950F900F900F900F9082E690E09F939E
:10EE50008F9386E590E09F938F931F921F928091EE
:10EE600002016AE00E94297A892F99279F938F9344
:10EE7000809102010E94297A99279F938F938FE2B4
:10EE80009CE09F938F931F930F93E091E003F09189
:10EE9000E103099589EF9AE09F938F931F930F9356
:10EEA000E091E003F091E103099581ED9AE09F93F1
:10EEB0008F931F930F93E091E003F091E103099585
:10EEC0008DB79EB746968DBF83E69CE09F938F9348
:10EED0001F930F93E091E003F091E103099583EC18
:10EEE0008093810080916F00806280936F000F900B
:10EEF0000F900F900F901F910F91089580918606AB
:10EF00008F3138F08091230887FD03C08EE1809314
:10EF1000860680913606882331F08055853618F0B4
:10EF20008FE7809336060895CF938091D20388238C
:10EF300009F46EC08091DD0381508093DD03882346
:10EF400009F04FC089E18093DD038091860680320D
:10EF500038F08091230887FD03C08FE180938606F7
:10EF60008091D602823800F58091A1029091A20290
:10EF7000885E934020F41092DF031092DE038091AC
:10EF8000DE039091DF03009739F101979093DF033F
:10EF90008093DE03419728F18091230884FF21C0EC
:10EFA00080919F0284601BC08091D602853BC8F08F
:10EFB0009091860684E1989FC0011124409620918B
:10EFC000DE033091DF032817390730F42F5F3F4FFE
:10EFD0003093DF032093DE0380919F028B7F809329
:10EFE0009F02C091A501CC2321F0C150C093A5017F
:10EFF0000FC086E98093A5018091A201843011F4AD
:10F000000E941E728091A101833411F0C093D2033B
:10F01000CF9108951F920F920FB60F9211242F9344
:10F020003F934F935F936F937F938F939F93AF9390
:10F03000BF93EF93FF932091CE008091B00188237E
:10F04000B1F02093C6008091B001823029F52F3FA6
:10F0500019F58FEF94E3ACE0B0E0C297A109B109D4
:10F06000B7FFFBCF809123048093CE0015C0909111
:10F07000A201892F8150833020F4822F0E942369BE
:10F080000BC0943021F4822F0E94117205C095307C
:10F0900019F4822F0E945071FF91EF91BF91AF91AF
:10F0A0009F918F917F916F915F914F913F912F91A0
:10F0B0000F900FBE0F901F901895FB01DC0102C04E
:10F0C00005900D9241505040D8F70895FC014150F1
:10F0D000504030F001900616D1F73197CF010895D6
:10F0E000882799270895A0E0B0E0E9E7F8E70C94B5
:10F0F000A17A6C017B01EA01590121978FEFCF3F83
:10F10000D80789F086010894C11CD11CC701089456
:10F11000E11CF11CF5010995F80180832197FFEFAF
:10F12000CF3FDF0779F7EAE0CDB7DEB70C94BD7AC1
:10F13000CF92DF92EF92FF920F931F937C016B01AE
:10F14000FB010995082FC7010196F6010995182FB3
:10F15000C8011F910F91FF90EF90DF90CF9008951D
:10F16000A0E0B0E0E6EBF8E70C94A37A8C017B0119
:10F17000EA01690121978FEFCF3FD80771F0F701BE
:10F1800021917F01C8010F5F1F4F622FF601099582
:10F190002197FFEFCF3FDF0791F7E8E0CDB7DEB76C
:10F1A0000C94BF7ACF92DF92EF92FF920F931F934E
:10F1B0006C018B017A01FA010995812F9927682F3B
:10F1C000C6010196F70109951F910F91FF90EF90ED
:10F1D000DF90CF9008955058BB27AA270ED0E0C0EB
:10F1E000D1D030F0D6D020F031F49F3F11F41EF48E
:10F1F000C6C00EF4E095E7FBBCC0E92FE2D080F377
:10F20000BA17620773078407950718F071F49EF523
:10F21000FAC00EF4E0950B2EBA2FA02D0B01B90108
:10F2200090010C01CA01A0011124FF27591B99F07C
:10F23000593F50F4503E68F11A16F040A22F232F88
:10F24000342F4427585FF3CF469537952795A795D8
:10F25000F0405395C9F77EF41F16BA0B620B730B7F
:10F26000840BBAF09150A1F0FF0FBB1F661F771FF0
:10F27000881FC2F70EC0BA0F621F731F841F48F4A5
:10F28000879577956795B795F7959E3F08F0B3CF2B
:10F290009395880F08F09927EE0F97958795089515
:10F2A00098D088F09F5790F0B92F9927B751A0F0C8
:10F2B000D1F0660F771F881F991F1AF0BA95C9F70A
:10F2C00012C0B13081F09FD0B1E008959CC0672F8B
:10F2D000782F8827B85F39F0B93FCCF386957795BA
:10F2E0006795B395D9F73EF49095809570956195A3
:10F2F0007F4F8F4F9F4F0895E89409C097FB3EF4CE
:10F3000090958095709561957F4F8F4F9F4F992372
:10F31000A9F0F92F96E9BB279395F69587957795F0
:10F320006795B795F111F8CFFAF4BB0F11F460FFB0
:10F330001BC06F5F7F4F8F4F9F4F16C0882311F008
:10F3400096E911C0772321F09EE8872F762F05C01C
:10F35000662371F096E8862F70E060E02AF09A95B7
:10F36000660F771F881FDAF7880F9695879597F9AC
:10F37000089597F99F6780E870E060E008959FEF37
:10F3800080EC089500240A9416161706180609063C
:10F39000089500240A94121613061406050608950B
:10F3A000092E0394000C11F4882352F0BB0F40F493
:10F3B000BF2B11F460FF04C06F5F7F4F8F4F9F4FD3
:10F3C000089557FD9058440F551F59F05F3F71F055
:10F3D0004795880F97FB991F61F09F3F79F08795BC
:10F3E0000895121613061406551FF2CF4695F1DF45
:10F3F00008C0161617061806991FF1CF86957105D5
:10F40000610508940895E894BB2766277727CB0108
:10F4100097F90895629FD001739FF001829FE00DDC
:10F42000F11D649FE00DF11D929FF00D839FF00D83
:10F43000749FF00D659FF00D9927729FB00DE11D2F
:10F44000F91F639FB00DE11DF91FBD01CF0111240C
:10F450000895991B79E004C0991F961708F0961B30
:10F46000881F7A95C9F780950895AA1BBB1B51E1A7
:10F4700007C0AA1FBB1FA617B70710F0A61BB70B24
:10F48000881F991F5A95A9F780959095BC01CD01C9
:10F49000089597FB092E07260AD077FD04D0E5DFF3
:10F4A00006D000201AF4709561957F4F0895F6F705
:10F4B000909581959F4F0895A1E21A2EAA1BBB1B20
:10F4C000FD010DC0AA1FBB1FEE1FFF1FA217B30730
:10F4D000E407F50720F0A21BB30BE40BF50B661F46
:10F4E000771F881F991F1A9469F76095709580950A
:10F4F00090959B01AC01BD01CF01089597FB092EAA
:10F5000005260ED057FD04D0D7DF0AD0001C38F4F2
:10F5100050954095309521953F4F4F4F5F4F08953F
:10F52000F6F790958095709561957F4F8F4F9F4F1F
:10F5300008952F923F924F925F926F927F928F9297
:10F540009F92AF92BF92CF92DF92EF92FF920F9372
:10F550001F93CF93DF93CDB7DEB7CA1BDB0B0FB67C
:10F56000F894DEBF0FBECDBF09942A883988488839
:10F570005F846E847D848C849B84AA84B984C884CF
:10F58000DF80EE80FD800C811B81AA81B981CE0FC6
:10F59000D11D0FB6F894DEBF0FBECDBFED010895AB
:0EF5A000EE0FFF1F0590F491E02D0994FFCFB0
:10F5AE005E010A010164FF01FFFFC01FC01F0101C0
:10F5BE0001737373FF03007D0000C409C409640066
:10F5CE00104661737400004E6F726D616C000045E1
:10F5DE00617379000051756164726F00006400D22E
:10F5EE000101200B050000ECFF00020406070808CD
:10F5FE00080706040200FEFCFAF9F8F8F8F9FAFC1E
:10F60E00FE000204060708086440415A4664640A74
:10F61E0002969696960840403A10FB30380132FF1B
:10F62E0003780090D0030090D0030032002064FFD6
:10F63E00FF64200B0A0D0B0C0E0B0F10FA200101AC
:06F64E000170FF010F64D2
:00000001FF
